:100000000C9448210C9479210C9479210C94792139
:100010000C9479210C9479210C9479210C947921F8
:100020000C9479210C9479210C9479210C947921E8
:100030000C9479210D945F3E0C9479210C947921D4
:100040000C9479210C94B9DA0C9479210C947921CF
:100050000C9479210C9479210C9480D70D94153E41
:100060000C9479210C94F44C0C94EA4C0C94792166
:100070000C9479210C9479210C9479210C94792198
:100080000C9479210C9479210C9479210C94792188
:100090000C9479210C9479210C9479210C94792178
:1000A0000C9479210C9479210C9479210C94792168
:1000B0000C9479210C9479210C9479210C94792158
:1000C0000C9479210C9479210C9479210C94792148
:1000D0000C9479210C9479210C9479210C94792138
:1000E0000C947921084AD73B3BCE016E84BCBFFDFE
:1000F000C12F3D6C74319ABD56833DDA3D00C77FF8
:1001000011BED9E4BB4C3E916BAAAABE0000008090
:100110003F05A84CCDB2D44EB93836A9020C50B91F
:10012000918688083CA6AAAA2ABE000000803F004B
:100130000D9438380C947E210D946F380C94877E82
:100140000C943C830C94D6870D9485370D94893795
:100150000C94137B0C94C4860C94187D0D94841617
:100160000C947B210D946F370C94D5860C94997860
:100170000C9461B50C94DC870C94307D0C94A778BA
:100180000D9483380C9401CA0C9422860C94864DED
:100190000C942C830C94837E0C94B1C50D94C037C1
:1001A0000C94A6CB0C94B0840C948F7B0C943FB52C
:1001B0000C94B07C0C9482C90C9444830D94A437A5
:1001C0000D9442380C9440830C94D09B0D9481374D
:1001D0000C94A67B0D946A370C94F5B20C94BB96E4
:1001E0000C941ECA0C946C220C9445980C94E2B1A9
:1001F0000D949A370C94AE7C0C947B7E0C94C7873C
:100200000C94D3870C94FEB10C94324D0C948A4D0F
:100210000C94388F0C94E3870C9484220C94048102
:100220000C94317E0C94047B0C94ACB10C9494CB64
:100230000C94B8A00C9438830C9494800C9441A234
:100240000D948D380C949ABE0C94527B0C9454905F
:100250000C949B7C0C94727E0C949A4D0D9479387E
:100260000D94BC370C94477D0C948F840C94F783C9
:100270000D94A0370C94FE7C0C945D840C94617BEF
:100280000C94CAB10D94B6160D94AD170C94367833
:100290000C9460250D948D370C94964D0C94BF7A78
:1002A0000C94CA8C0C94EF830C9432800C942A7DAD
:1002B0000C94F97E0C94D27A0C94A54D0D942D4A91
:1002C0000C94DCB10C94F6920C94FAA80C9412A73E
:1002D0000C9413A40C947BBE0C941F340C94EB254B
:1002E0000C9489250D9490370C94BD7B0C949A84C2
:1002F0000C94EEB10D94FD370C9425990D9414389F
:100300000C94AC7A0C94277D0C9441780C94DBBE51
:100310000C94BE860C947F4D0C9449B50D94B63761
:100320000C945D880C94BB990C94C2A00C943F88EB
:100330000C94B84D0C94CA870C9428830C94F39AAF
:100340000C94B77C0D9428380C94D58D0C94377A86
:100350000C9444B50C94817E0C94E6870C9416CBD7
:100360000C948F7C0C9461850C9430830C944C839A
:100370000D944B4A0C9404850D94B2370D9430388B
:100380000C9444840C94FABE0C9448830D944C381D
:100390000C94E8B10D9457160D940A380C94397BDF
:1003A0000C94B7CA0C9480780C94267B0C9428BECD
:1003B0000C94E9870C943AB50C94E0860C9405C72C
:1003C0000C943E800C94F4B10C94B2B10D94973817
:1003D0000C94C67C0C94D0B10C9413390C94C17C51
:1003E0000D941E380C948C800C947D7E0C94CD87DB
:1003F0000C94787A0C94D9870C9476840D94DA490D
:100400000C9424BF0C94B04D0C949DCC0C94427D64
:100410000C94CC860C942BAA0C94507A0D9496379D
:100420000C94937A0C9442880C943F7C0C949E4DCF
:100430000D94AE370C94DF830C94BC7C0C94B9946F
:100440000C94614D0C947F7E0C94E07D0C94F8210B
:100450000C94FBCA0C94857E0C9410B60C94227EEE
:100460000C94EB7A0C942FC50C942FB90C94BEB15C
:100470000C94B8B10C94BC870C94E1870C94787BF5
:100480000C94C4B10C9409BE0C94D1840C945A9A67
:100490000C9413780C94D3CB0C94B2C50C94924D5D
:1004A0000C94D0870C942D7D0C94B27C0C94179FE7
:1004B0000D94A8370C9490800C94697A0C947CAEBF
:1004C0000C94897E0C942B840C9434830C9496CADF
:1004D0000C948E4D0C941B850D9405380C944B7D1B
:1004E0000D9465380C94D6B50C94704D0C94F78A25
:1004F0000C94419D0D9456380C94D6B10C94867C86
:100500004E414E494E495459494E46CDCCCC3D0AF8
:10051000D7233C17B7D13877CC2B329595E6241FDB
:10052000B14F0A000020410000C84200401C462094
:10053000BCBE4CCA1B0E5AAEC59D7400407A10F367
:100540005A00A0724E18090010A5D4E80000E87601
:1005500048170000E40B54020000CA9A3B00000058
:10056000E1F505000080969800000040420F000071
:1005700000A08601000000102700000000E8030032
:100580000000006400000000000A000000000001FC
:1005900000000000002C76D888DC674F0823DFC1FC
:1005A000DFAE59E1B1B796E5E3E453C63AE65199B7
:1005B0007696E8E6C28426EB898C9B62ED407C6FE0
:1005C000FCEFBC9C9F40F2BAA56FA5F490055A2A97
:1005D000F75C936B6CF9676DC11BFCE0E40D47FEA3
:1005E000F520E6B500D0ED902E0300943577050098
:1005F00080841E080000204E0A000000C80C33331F
:1006000033330F986E12831141EF8D2114893BE62D
:100610005516CFFEE6DB18D1844B381BF77C1D90B6
:100620001DA4BBE424203284725E228100C9F1241F
:10063000ECA1E53D27434F4D4D554E4943415449AB
:100640004F4E0044525952554E004552524F52534C
:1006500000494E464F004543484F004572726F7245
:100660002077726974696E6720746F204545505217
:100670004F4D210A0053544F505045442E200050F6
:1006800072696E7465722073746F70706564206433
:10069000756520746F206572726F72732E204669C3
:1006A0007820746865206572726F7220616E6420B4
:1006B000757365204D39393920746F2072657374F4
:1006C0006172742E202854656D7065726174757244
:1006D000652069732072657365742E2053657420DC
:1006E00069742061667465722072657374617274D6
:1006F000696E67290A004E6F20436865636B7375E6
:100700006D2077697468206C696E65206E756D6206
:1007100065722C204C617374204C696E653A200020
:100720004E6F20436865636B73756D2077697468DD
:10073000206C696E65206E756D6265722C204C614F
:100740007374204C696E653A2000636865636B734F
:10075000756D206D69736D617463682C204C6173D5
:1007600074204C696E653A20004C696E65204E75A8
:100770006D626572206973206E6F74204C617374B2
:10078000204C696E65204E756D6265722B312C2090
:100790004C617374204C696E653A20004D313130E4
:1007A0000053657269616C20737461747573206D98
:1007B00069736D617463680A00776169740A005334
:1007C000442072656164206572726F720A00486F1E
:1007D00074656E642049646C652054696D656F753D
:1007E0007400486F74656E642049646C65205469B8
:1007F0006D656F75740A002121204B494C4C2063B4
:100800006175736564206279204B494C4C20627598
:1008100074746F6E2F70696E0A002121204B494C51
:100820004C2063617573656420627920746F6F205A
:100830006D75636820696E6163746976652074699B
:100840006D65202D2063757272656E7420636F6D07
:100850006D616E643A20007061757365004D3630CD
:1008600030002066696C616D656E745F72756E6FC5
:100870007574200066696C616D656E745F72756E6B
:100880006F757420540046696C616D656E745275A5
:100890006E6F75742054004D656469612052656DFA
:1008A0006F766564004D6564696120496E73657299
:1008B000746564004D313030305300627573793A9D
:1008C0002070617573656420666F7220696E707543
:1008D000740A00627573793A2070617573656420DB
:1008E000666F7220757365720A00627573793A20BB
:1008F00070726F63657373696E670A00506C65612F
:100900007365205265736574005052494E544552C8
:100910002048414C5445440025533A20255300704B
:100920006F7765726F6666004B494C4C45442E20CC
:10093000005072696E7465722068616C7465642E13
:10094000206B696C6C28292063616C6C6564210ADA
:10095000006563686F3A004572726F723A000A4D23
:100960006561737572656420706F696E74733A0A9D
:1009700000387838206D6573682E205A206F6666BF
:100980007365743A20005072696E74696E67204F07
:10099000626A656374002553202569002F2F616307
:1009A00074696F6E3A0073746172740070726F6D67
:1009B00070745F00656E6400486F74656E642074C7
:1009C0006F6F20636F6C640A0053656E64204D3155
:1009D000303820746F20726573756D650A00496E3A
:1009E000736572742066696C616D656E7420616EEA
:1009F000642073656E64204D3130380A005265689A
:100A000065617420446F6E65005265686561746944
:100A10006E672E2E2E005265686561740048656110
:100A20007465722054696D656F75740053656E64EA
:100A3000204D31303820746F2068656174206E6FEE
:100A40007A7A6C650A004E6F7A7A6C652050617212
:100A50006B656400706175736564005061757365E2
:100A600000726573756D656400526573756D696EAE
:100A700067004732362043616E63656C65640047EA
:100A800032362048656174696E67204E6F7A7A6CE1
:100A900065004732362048656174696E672042659B
:100AA000640057616974696E6720666F72206865BB
:100AB000617475702E0A004669786564204C656E15
:100AC000677468205072696D6500446F6E652050D0
:100AD00072696D696E67004D616E75616C20707230
:100AE000696D696E672E2E2E004C656176696E67A2
:100AF00020473236003F537065636966696564203C
:100B0000582C5920636F6F7264696E617465206F31
:100B10007574206F6620626F756E64732E0A003FD5
:100B200028522965706561742076616C7565206E48
:100B30006F7420706C61757369626C653B206D75B4
:100B40007374206265206174206C65617374203158
:100B50002E0A003F537065636966696564206E6F95
:100B60007A7A6C652074656D7065726174757265F2
:100B7000206E6F7420706C61757369626C652E0AEB
:100B8000003F5370656369666965642066696C61DE
:100B90006D656E742073697A65206E6F7420706C59
:100BA00061757369626C652E0A003F5370656369F5
:100BB00066696564207072696D65206C656E677426
:100BC00068206E6F7420706C61757369626C652E3D
:100BD0000A003F537065636966696564206E6F7AC9
:100BE0007A6C652073697A65206E6F7420706C6111
:100BF000757369626C652E0A003F52657472616399
:100C000074696F6E204D756C7469706C69657220C3
:100C10006D757374206265207370656369666965BC
:100C2000642E0A003F5370656369666965642052EB
:100C3000657472616374696F6E204D756C74697050
:100C40006C696572206E6F7420706C617573696277
:100C50006C652E0A003F53706563696669656420A0
:100C60006C6179657220686569676874206E6F745D
:100C700020706C61757369626C652E0A0043292EC1
:100C80000A003F5370656369666965642062656444
:100C90002074656D7065726174757265206E6F7415
:100CA00020706C61757369626C65202834302D008A
:100CB000473236207374617274696E672E2E2E0A65
:100CC000004F46460A0046616465204865696768CA
:100CD000742000426564204C6576656C696E6720FF
:100CE000004661696C656420746F20656E61626C9A
:100CF0006520426564204C6576656C696E670A0004
:100D00004D65736820426564204C6576656C20648F
:100D10006174613A0A00496E76616C6964206D65A0
:100D200073682E0A00206E6F7420656E746572659C
:100D3000642E0A0050726F62696E6720506F696E90
:100D4000740025532025692F256900206F66200037
:100D50004D424C2047323920706F696E7420002953
:100D60000A004A206F7574206F662072616E676595
:100D70002028302D00290A0049206F7574206F66E5
:100D80002072616E67652028302D004732384C3064
:100D9000004D6573682070726F62696E6720646FC2
:100DA0006E65004D6573682070726F62696E6720B2
:100DB000646F6E652E0A005374617274206D6573E2
:100DC000682070726F62696E67207769746820228C
:100DD000473239205331222066697273742E0A001B
:100DE0004732395332004732384C300A4732395390
:100DF0003200686173206E6F20646174612E0A0096
:100E00004D65736820426564204C6576656C696E3B
:100E100067200053206F7574206F662072616E67C3
:100E2000652028302D35292E0A004D657368207005
:100E30006F696E74206F7574206F662072616E67C3
:100E4000650A004D34323120696E636F72726563DA
:100E50007420706172616D6574657220757361676D
:100E6000650A005741524E494E4721204C6F77206A
:100E70005A204A65726B206D6179206C656164202F
:100E8000746F20756E77616E746564207061757320
:100E900065732E0A004F4646004F4E0020204D61DC
:100EA000783A2000200020204D696E3A2000536FD0
:100EB000667420656E6473746F70733A20004D32EF
:100EC000342053256C642054256C64004739322E3D
:100ED00039204525730047312046256400473932C3
:100EE0002E39205A2573004731205A30204632309F
:100EF0003000473120582573205925732046333060
:100F00003030004D34323020532569205A2573008B
:100F10004D3130362050256920532569004D32303F
:100F20003020442573004732385230585900473931
:100F3000322E39204530205A300A47315A25730065
:100F40004D31303920532569004D3139302053253A
:100F500069004D343230205330205A300020496E21
:100F600076616C69642065787472756465722000BE
:100F700047322F47332062616420706172616D6572
:100F8000746572730A00536C6565702E2E2E004DC9
:100F900065736820706F696E74206F7574206F665A
:100FA0002072616E67650A004D302053746F7000C7
:100FB0004D312053746F7000436C69636B20746F04
:100FC00020526573756D652E2E2E004E6F204D6F6D
:100FD00076652E00456E642066696C65206C6973C9
:100FE000740A00426567696E2066696C65206C69E9
:100FF00073740A004E6F206D656469610A00526562
:1010000073756D696E6720534400286E6F206669A2
:101010006C65290043757272656E742066696C6533
:101020003A20005072696E742074696D653A200030
:101030000A53746174733A2046696C616D656E740D
:1010400020757365643A20002C204C6F6E676573C1
:1010500074206A6F623A2000546F74616C20746966
:101060006D653A200053746174733A20002C204659
:1010700061696C65643A20002C2046696E6973686A
:1010800065643A20005072696E74733A200053749C
:101090006174733A2000436F6F6C696E672E2E2E59
:1010A0000048656174696E672E2E2E004520255319
:1010B000006F6B006F666600560651064A064306CF
:1010C000350644454255473A004D313133205300EF
:1010D00042656420436F6F6C696E672E2E2E00424E
:1010E00065642048656174696E672E2E2E00343069
:1010F00030205375506552204F46462E002F2F004A
:101100004D31343520533C696E6465783E206F75EF
:1011100074206F662072616E67652028302D31293A
:101120000A00205200416363656C65726174696FE7
:101130006E3A2050004D32303620580046523A0068
:1011400020466C6F773A20004D424C2041646A750E
:101150007374205A0020643A0020693A0020703AE3
:1011600000496E76616C6964206578747275646597
:10117000720A0020643A0020693A0020703A006444
:10118000697300656E0043290A0061626C65642022
:10119000286D696E2074656D702000436F6C64204B
:1011A00065787472756465732061726520004669A4
:1011B0006C616D656E742072756E6F7574206469F4
:1011C0007374616E636520286D6D293A200046694D
:1011D0006C616D656E742072756E6F757420004F52
:1011E000666673657473204170706C696564004550
:1011F00072723A20546F6F206661722100546F6FD3
:10120000206661722066726F6D2072656665726518
:101210006E636520706F696E740A00454550524FC9
:101220004D204F4B0A002E0A002028302D31302946
:10123000002076616C7565206F7574206F66207272
:10124000616E676500416476616E6365204B3D00A9
:10125000506F7765722D6C6F7373207265636F7654
:1012600065727920004D383400446F6E65207072CD
:10127000696E74696E672066696C650A004D373760
:10128000004D3331004361703A004D4541545041A7
:10129000434B00434F4F4C45525F54454D504552D0
:1012A0004154555245004348414D4245525F5445D3
:1012B0004D504552415455524500424142595354B4
:1012C000455050494E470041524353004D4F5449F9
:1012D0004F4E5F4D4F44455300544845524D414C8D
:1012E0005F50524F54454354494F4E004C4F4E4768
:1012F0005F46494C454E414D45004155544F52457E
:10130000504F52545F53445F53544154555300530C
:10131000445F57524954450052455045415400538B
:1013200044434152440050524F4D50545F53555026
:10133000504F525400454D455247454E43595F501A
:10134000415253455200434153455F4C494748542D
:101350005F4252494748544E45535300544F474704
:101360004C455F4C494748545300534F46545741EE
:1013700052455F504F574552004255494C445F50CB
:10138000455243454E54004C4556454C494E475FE7
:1013900044415441005A5F50524F42450052554E0D
:1013A0004F5554004155544F4C4556454C005052F2
:1013B000494E545F4A4F420050524F475245535393
:1013C000004155544F5245504F52545F54454D5073
:1013D00000564F4C554D45545249430045455052D7
:1013E0004F4D0042494E4152595F46494C455F546A
:1013F00052414E534645520053455249414C5F5865
:101400004F4E5F584F4646004649524D5741524550
:101410005F4E414D453A4D61726C696E20322E30FF
:101420002E375F4457372E332E3120544D3344200E
:1014300034534D444E4E20284170722032392032B0
:101440003032312032323A33343A30372920534F58
:10145000555243455F434F44455F55524C3A68747B
:101460007470733A2F2F6769746875622E636F6D9D
:101470002F496E73616E6974794175746F6D617413
:10148000696F6E2F4D61726C696E2F747265652F76
:10149000437265616C6974794477696E5F322E308E
:1014A0002050524F544F434F4C5F56455253494F73
:1014B0004E3A312E30204D414348494E455F5459F4
:1014C00050453A34303020537550655220455854B9
:1014D00052554445525F434F554E543A312055556D
:1014E00049443A63656465326132662D3431613254
:1014F0002D343734382D396231322D63353563362A
:10150000326633363766660A0043616E6E6F74204A
:101510006F70656E2073756264697220002569734F
:101520000025696D20256973002569682025696D8E
:101530002025697300256964202569682025696D67
:10154000202569730025697920256964202569684B
:101550002025696D202569730023646566696E65C1
:101560002044454641554C545F00626564004B641D
:1015700020004B6920004B702000504944204175E9
:10158000746F74756E652066696E69736865642131
:101590002050757420746865206C617374204B70E2
:1015A0002C204B6920616E64204B6420636F6E7346
:1015B00074616E74732066726F6D2062656C6F77F4
:1015C00020696E746F20436F6E666967757261740F
:1015D000696F6E2E680A00504944204175746F741B
:1015E000756E65206661696C6564212074696D653E
:1015F0006F75740A00504944204175746F74756E9C
:1016000065206661696C6564212054656D70657242
:10161000617475726520746F6F20686967680A006D
:10162000204B643A2000204B693A2000204B703A4E
:10163000200020436C617373696320504944200A81
:1016400000204E6F206F76657273686F6F740A00AA
:101650002054753A2000204B753A2000206D6178A7
:101660003A2000206D696E3A200020643A20002064
:10167000626961733A2000504944204175746F7467
:10168000756E652073746172740A0050494420417C
:1016900075746F74756E65206661696C6564212070
:1016A00054656D706572617475726520746F6F201A
:1016B000686967680A00504944204175746F747501
:1016C0006E6500504944204175746F74756E6520D5
:1016D0006661696C6564212042616420686561749B
:1016E00065722069640A004572723A207574663822
:1016F00020666F6E74206E6F7420696E6974696104
:101700006C697A65642E004572723A207574663889
:1017100020666F6E74206E6F7420696E69746961E3
:101720006C697A65642E004572723A207574663869
:1017300020666F6E74206E6F7420696E69746961C3
:101740006C697A65642E00000C0F00FE0702250309
:10175000BB017FFE08FE08FE05080806000040F0F9
:10176000C88888987810050808060000C0F888889E
:10177000888888F80505050600012030F830200526
:1017800008080600002070F820202020E005090944
:101790000600FF2070A8A8B88888702007050507F4
:1017A0000001D86C366CD80509090600FFF8A88836
:1017B00088888888A8F8050A0A0600FE205050503C
:1017C0005088A8A8887003030306000340A040FFC8
:1017D000FFFFFFFFFFFFFFFFFFFFFFFFFFFFFFFF19
:1017E000FFFFFFFFFF0000000605FF0107070602DD
:1017F0000080808080800080030303060105A0A094
:10180000A005060606000050F85050F850050909DA
:101810000600FF2070A8A07028A870200507070602
:101820000000C8C81020409898050707060000402F
:10183000A0A040A8906801030306020580808003F1
:1018400009090601FF2040408080804040200309B4
:10185000090601FF80404020202040408005070706
:1018600006000020A8702070A820050505060001CC
:101870002020F820200203030601FFC0408005015C
:1018800001060003F8020202060100C0C0050707B6
:1018900006000008101020404080050707060000E1
:1018A000708898A8C8887003070706010040C040E8
:1018B000404040E0050707060000708808102040FF
:1018C000F8050707060000F80810300888700507BB
:1018D0000706000010305090F810100507070600AA
:1018E00000F880F0080888700507070600003040FF
:1018F00080F0888870050707060000F8081010209F
:101900002020050707060000708888708888700509
:101910000707060000708888780810600205050631
:101920000100C0C000C0C00206060601FFC0C00022
:10193000C0408003050506010120408040200503CA
:1019400003060002F800F8030505060101804020A7
:101950004080050707060000708810202000200541
:1019600007070600007088B8A8B88070050707064A
:101970000000708888F8888888050707060000F04E
:101980004848704848F005070706000070888080C6
:10199000808870050707060000F04848484848F06E
:1019A000050707060000F88080F08080F80507072B
:1019B000060000F88080F0808080050707060000A0
:1019C00070888080988870050707060000888888DE
:1019D000F8888888030707060100E040404040403F
:1019E000E00507070600003810101010906005078A
:1019F000070600008890A0C0A09088050707060091
:101A000000808080808080F805070706000088D865
:101A1000A8888888880507070600008888C8A898CD
:101A20008888050707060000708888888888700500
:101A30000707060000F08888F08080800507070609
:101A4000000070888888A89068050707060000F0E5
:101A50008888F0A0908805070706000070888070CD
:101A6000088870050707060000F8202020202020A5
:101A7000050707060000888888888888700507079A
:101A80000600008888888850502005070706000057
:101A900088888888A8A8500507070600008888500D
:101AA00020508888050707060000888850202020DD
:101AB00020050707060000F80810204080F80309F9
:101AC000090601FFE080808080808080E0050707B4
:101AD000060000804040201010080309090601FF9D
:101AE000E020202020202020E00503030600052020
:101AF00050880501010600FEF80303030601058076
:101B0000402005050506000070087888780507075D
:101B10000600008080F0888888F005050506000032
:101B2000708080887005070706000008087888889C
:101B300088780505050600007088F08070050707A5
:101B4000060000304840E04040400507070600FE20
:101B5000708888887808700507070600008080F084
:101B6000888888880307070601004000C04040407D
:101B7000E00409090601FE100030101010109060FA
:101B800005070706000080808890E090880307071B
:101B9000060100C04040404040E005050506000049
:101BA000D0A8A8A8A8050505060000B0C8888888A0
:101BB000050505060000708888887005070706007F
:101BC000FEF0888888F080800507070600FE788888
:101BD0008888780808050505060000B0C880808060
:101BE00005050506000078807008F0050707060067
:101BF000002020F820202018050505060000888810
:101C00008898680505050600008888885020050525
:101C1000050600008888A8A850050505060000886C
:101C2000502050880507070600FE8888885020400D
:101C300080050505060000F8102040F80309090694
:101C400001FF204040408040404020010909060239
:101C5000FF8080808080808080800309090601FFEA
:101C60008040404020404040800503030600024879
:101C7000A890FF554E4C4F41442046494C414D459C
:101C80004E54004C4F41442046494C414D454E5422
:101C90000046494C414D454E54204348414E47452E
:101CA0000042656400456E636C6F73757265002554
:101CB00068753A25303268750025303268753A25E6
:101CC0003032687500202020202020200020202095
:101CD00020001FE0201020102010102010202010C5
:101CE000201030300840048003001FE03FF03FF038
:101CF0003FF01FE01FE03FF03FF03FF00FC00780D4
:101D000003003FFFF038007030FC3020FC102078DA
:101D1000102030102C00D02E31D02F7BD02F7BD034
:101D20002E31D02C00D020301020781020FC103024
:101D3000FC303800703FFFF03FFFF0380070318614
:101D4000302387102787902F87D02F03D020301083
:101D50002078102078102030102F03D02F87D02724
:101D600087902387103186303800703FFFF01FFFC7
:101D7000F81FFFF804104002082002082004104059
:101D8000082080104100104100082080041040000D
:101D900000001FFFF81FFFF8FFFFFF8000018E000B
:101DA000E19F01F19381399F81F99F81F99FB9F9F1
:101DB0008F28F18038018000019FFFF99174999B71
:101DC00006A99B54A99B56A99B54999FFFF9FFFF15
:101DD000FF6E6F74696669636174696F6E2000637A
:101DE000616E63656C005072696E742041626F723F
:101DF000746564004469736D6973730055492041CB
:101E0000626F72746564004D323520500A4D323471
:101E100000526573756D6500554920506175736595
:101E20000050617573696E672E2E2E007265737592
:101E30006D65004D32340052756E6F7574204469C3
:101E40007374206D6D004C6F6164206D6D00556E74
:101E50006C6F6164206D6D0046696C2E2044696171
:101E60002E004520696E206D6D5E33004164766101
:101E70006E6365204B004D333033205531204525AE
:101E8000692053256900504944204175746F747569
:101E90006E65202A005049442D44202A00504944B0
:101EA0002D49202A005049442D50202A0020082086
:101EB00046616374002008204D6178002008204DA1
:101EC000696E004F6666004F6E004175746F7465F1
:101ED0006D70005654726176204D696E00566D69C2
:101EE0006E00566D6178204500566D6178205A006D
:101EF000566D6178205900566D6178205800416D0B
:101F00006178204500416D6178205A00416D61780B
:101F1000205900416D6178205800412D547261763E
:101F2000656C00412D526574726163740041636396
:101F3000656C0056652D4A65726B00565A2D4A65D0
:101F4000726B0056592D4A65726B0056582D4A65C2
:101F5000726B00452073746570732F6D6D005A208D
:101F600053746570732F6D6D0059205374657073D1
:101F70002F6D6D00582053746570732F6D6D004187
:101F80006476616E6365642053657474696E67730B
:101F9000003F0043616E63656C00496E6974004DDB
:101FA00034323800496E697469616C697A6520451C
:101FB0004550524F4D0046696C616D656E7400541A
:101FC000656D7065726174757265005374657073C8
:101FD0002F6D6D004A65726B00416363656C6572BD
:101FE0006174696F6E0056656C6F63697479005334
:101FF000657420486F6D65204F6666736574730065
:10200000436F6E66696775726174696F6E003F0039
:102010004E65787420506F696E7400446F6E650071
:102020004E657874004C6576656C696E6720446F08
:102030006E6521004D6F7665205A00473239533264
:10204000004E65787420506F696E74002569202FEA
:102050002025750047323953310047323953320059
:10206000436C69636B20746F20426567696E00483A
:102070006F6D696E672058595A005A2056616C7509
:102080006500496E646578205900496E6465782062
:10209000580053746F72652053657474696E67736A
:1020A000004C6F61642053657474696E6773004CF3
:1020B0006576656C20436F726E657273004265646D
:1020C000205A004661646520486569676874004F5E
:1020D0006666004F6E00426564204C6576656C69EB
:1020E0006E670045646974204D657368004C6576C1
:1020F000656C20426564004D6F74696F6E003F002F
:1021000043616E63656C204F626A656374004E4F75
:10211000005945530043616E63656C204F626A65E8
:102120006374203D004D61696E00426564004E6F2E
:102130007A7A6C650046616E205370656564004371
:102140006F6E66696775726174696F6E0052657350
:10215000746F72652044656661756C7473004C6FB2
:1021600061642053657474696E67730053746F7291
:10217000652053657474696E677300507265686595
:102180006174202420436F6E6600506F7765722063
:102190004F7574616765004F6666004F6E0052753B
:1021A0006E6F75742053656E736F72004164766153
:1021B0006E6365642053657474696E6773004D6166
:1021C000696E004D37303220542564004D36303072
:1021D00020423020542564004D373032203B2564A6
:1021E000004D37303120542564004D373032004DDA
:1021F000373031004D363030204230004D61696E4D
:10220000004F6666004F6E0052756E6F75742053F6
:10221000656E736F72005075726765206D6F7265C1
:1022200000436F6E74696E756500524553554D4598
:10223000204F5054494F4E533A005052494E54206B
:102240005041555345440020204E6F7A7A6C653AD0
:1022500020005061726B696E672E2E2E00000057B1
:1022600061697420666F720066696C616D656E7479
:10227000206368616E676500746F207374617274A7
:10228000005761697420666F720066696C616D65E4
:102290006E7420756E6C6F616400004E6F7A7A6C9C
:1022A000652068656174696E6700506C656173656F
:1022B00020776169742E2E2E000050726573732092
:1022C000627574746F6E00746F2068656174206E3F
:1022D0006F7A7A6C650000496E7365727420666966
:1022E0006C616D656E7400616E64207072657373ED
:1022F00020627574746F6E00746F20636F6E746902
:102300006E7565005761697420666F720066696C4E
:10231000616D656E74206C6F61640000507265734E
:102320007320427574746F6E00746F2072657375DC
:102330006D65207072696E74000057616974206663
:102340006F72207072696E7400746F20726573759D
:102350006D652E2E2E00005761697420666F720025
:1023600066696C616D656E742070757267650000DA
:102370003E2000256C642E25696D004578747275C9
:1023800064656420546F74616C003E20004C6F6E75
:1023900067657374204A6F622054696D65003E2042
:1023A00000546F74616C205072696E742054696DB2
:1023B0006500436F6D706C65746564003A20005071
:1023C00072696E7420436F756E74003A2000313567
:1023D000300035004245443A2041544320313034E6
:1023E00047542D320052756E6177617920576174C0
:1023F00063683A204F4E004D61782054656D70003F
:10240000333135004D696E2054656D7000350045DF
:10241000313A204550434F53203130304B00505318
:10242000550047656E657269630050726F746F6323
:102430006F6C00312E3000426175640032353030EF
:10244000303000437265616C6974793344205241C5
:102450004D5053004D657368204C6576656C696E10
:102460006700457874727564657273003100746931
:102470006E796D616368696E657333642E636F6D29
:102480000034303020537550655200323032312DD7
:1024900030342D313800322E302E375F4457372EEE
:1024A000332E31004D61726C696E005072696E742A
:1024B000657220537461747300546865726D69733A
:1024C000746F727300426F61726420496E666F00B0
:1024D0005072696E74657220496E666F004D616955
:1024E0006E004D313030300053746F70205072697F
:1024F0006E7400526573756D65205072696E74005C
:10250000506F776572204F7574616765003F0042B8
:1025100061636B0053746F70005072696E74206653
:10252000726F6D204D65646961004368616E676517
:10253000204D65646961004D32310041626F7574F0
:10254000205072696E746572004368616E67652021
:1025500046696C616D656E7400436F6E6669677580
:10256000726174696F6E0054656D70657261747527
:102570007265004D6F74696F6E00486F73742053FD
:102580007461727400526573756D65205072696E66
:1025900074004E6F204D656469610043616E636530
:1025A0006C204F626A6563740054756E65005374E5
:1025B0006F70205072696E740050617573652050A1
:1025C00072696E7400496E666F2053637265656E42
:1025D000003F005374617274205072696E7400433E
:1025E000616E63656C005072696E740043616E6E5B
:1025F0006F7420656E746572207375626469723AD7
:102600002000022E2E004D61696E002100486F747B
:10261000656E6420746F6F20636F6C640042616349
:102620006B0050726F63656564004F6666004F6EA5
:1026300000536F667420456E6473746F7073004D41
:102640006F74696F6E0044697361626C65205374C6
:10265000657070657273004D383400426564204CBB
:102660006576656C696E6700486F6D65205A004736
:1026700032385A00486F6D6520590047323859008A
:10268000486F6D6520580047323858004175746FA7
:1026900020486F6D6500473238004D61696E00500B
:1026A000726568656174202420456E64005072650F
:1026B000686561742024204265640054656D70650E
:1026C00072617475726500436F6F6C646F776E0032
:1026D0005072656865617420240046616E205370F5
:1026E000656564207E00426564004E6F7A7A6C6591
:1026F000004D61696E004261627973746570205AA1
:1027000000416476616E6365204B00466C6F770014
:1027100046616E205370656564207E0042656400EA
:102720004E6F7A7A6C6500426564205A005370657A
:102730006564004D61696E00486F6D696E67204683
:1027400061696C6564006F70656E0054524947475B
:1027500045524544003A200066696C616D656E74AF
:10276000007A5F6D696E00795F6D696E00785F6DEC
:10277000696E005265706F7274696E6720656E6471
:1027800073746F70207374617475730A0020746FB2
:102790006F206C6F6E6720657874727573696F6EE9
:1027A0002070726576656E7465640A0020636F6CD4
:1027B0006420657874727573696F6E2070726576C7
:1027C000656E7465640A00000000000000000000EF
:1027D0000000005761726E696E673A20486F6D693C
:1027E0006E672042756D702044697669736F722040
:1027F0003C20310A000202040000CD430000C8431F
:102800000000C843000000410000004100000040FB
:102810000000000100000001000080005555550037
:102820000000400033333300AAAA2A004992240052
:1028300000002000C7711C0099991900D1451700AC
:10284000555515003BB11300244912001111110018
:10285000000010000F0F0F00E3380E0043790D0049
:10286000CCCC0C00C3300C00E8A20B0064210B00A0
:10287000AAAA0A00703D0A009DD80900427B0900FF
:1028800092240900DCD30800888808001042080060
:1028900000000800F0C10700878707007550070097
:1028A000711C07003EEB0600A1BC06006990060003
:1028B00066660600703E06006118060017F4050003
:1028C00074D105005BB00500B2900500627205008E
:1028D0005555050078390500B81E050005050500A9
:1028E0004EEC040087D40400A1BD040090A70400AE
:1028F00049920400C17D0400EE690400C75604003B
:10290000444404005C320400082104004110040027
:10291000000004003FF00300F8E0030026D20300AB
:10292000C3C30300CCB503003AA803000A9B03000D
:10293000388E0300C08103009F750300D069030037
:10294000505E03001D53030034480300913D030013
:102950003333030016290300381F030097150300C3
:10296000300C0300030303000BFA020049F10200DC
:10297000BAE802005CE002002DD802002DD002006F
:1029800059C80200B0C0020031B90200DAB1020039
:10299000AAAA0200A0A30200BC9C0200FA950200B1
:1029A0005C8F0200DF88020082820200457C020008
:1029B0002776020027700200436A02007C6402004E
:1029C000D05E02003F590200C8530200FFFDFCFA2E
:1029D000F8F6F4F2F0EEECEAE9E7E5E3E1E0DEDC5C
:1029E000DAD9D7D5D4D2D0CFCDCBCAC8C7C5C3C208
:1029F000C0BFBDBCBAB9B7B6B4B3B2B0AFADACAA84
:102A0000A9A8A6A5A4A2A1A09E9D9C9A99989795D5
:102A1000949392908F8E8D8B8A8988878684838207
:102A200081807F7E7D7B7A79787776757473727119
:102A3000706F6E6D6C6B6A6968676665646362610E
:102A4000605F5E5D5C5B5A595858575655545352F7
:102A50005150504F4E4D4C4B4A4A494847464645C7
:102A60004443424241403F3E3E3D3C3B3B3A393885
:102A70003837363535343332323130302F2E2E2D33
:102A80002C2B2B2A292928272726252524232322D6
:102A9000212120201F1E1E1D1C1C1B1B1A1919186A
:102AA00018171616151514131312121111100F0FF3
:102AB0000E0E0D0D0C0C0B0A0A0909080807070673
:102AC0000605050404030302020100000000CD43D3
:102AD0000000C8430000C8430000000000000000E0
:102AE0000000000053657474696E67732053746F3F
:102AF00072656400454550524F4D20496E697469B6
:102B0000616C697A65640A003B200020204D3630F4
:102B100033200020440020204D3431322053004621
:102B2000696C616D656E742072756E6F757420735B
:102B3000656E736F723A002055004C0046696C61F7
:102B40006D656E74206C6F61642F756E6C6F61645F
:102B5000206C656E677468733A0020204D39303000
:102B6000204B004C696E65617220416476616E6332
:102B7000653A0020204D343133205300506F776583
:102B8000722D4C6F7373205265636F766572793A5C
:102B90000020440020490020204D333034205000D4
:102BA00020440020490020204D3330312050005077
:102BB00049442073657474696E67733A0020460057
:102BC00020480020204D3134352053004D6174657C
:102BD0007269616C206865617475702070617261E2
:102BE0006D65746572733A00202047323920533482
:102BF000205A00204A0020204732392053332049F0
:102C00000020204D3432302053004D65736820423F
:102C10006564204C6576656C696E673A0020204DCE
:102C2000323036205800486F6D65206F66667365D8
:102C3000743A0020580020530020204D32303520B7
:102C40004200416476616E6365643A20423C6D697E
:102C50006E5F7365676D656E745F74696D655F75D2
:102C6000733E20533C6D696E5F6665656472617486
:102C7000653E20543C6D696E5F74726176656C5F71
:102C800066656564726174653E20583C6D61785F6D
:102C9000785F6A65726B3E20593C6D61785F795F41
:102CA0006A65726B3E205A3C6D61785F7A5F6A6537
:102CB000726B3E20453C6D61785F655F6A65726B43
:102CC0003E0020540020520020204D32303420504D
:102CD00000416363656C65726174696F6E2028756D
:102CE0006E6974732F7332293A20503C7072696E8A
:102CF000745F616363656C3E20523C7265747261FF
:102D000063745F616363656C3E20543C74726176EA
:102D1000656C5F616363656C3E0020204D3230312D
:102D20002058004D6178696D756D20416363656C55
:102D300065726174696F6E2028756E6974732F7384
:102D400032293A0020204D3230332058004D61782E
:102D5000696D756D206665656472617465732028A0
:102D6000756E6974732F73293A00537465707320FC
:102D700070657220756E69743A0020440020204D01
:102D80003230302053002044697361626C65640AFC
:102D90000046696C616D656E742073657474696E4C
:102DA00067733A0020204D3134392043203B2055B1
:102DB0006E69747320696E2043656C736975730A5C
:102DC0000020286D6D29002020473231202020204E
:102DD0003B20556E69747320696E206D6D00000094
:102DE000FA430000C8430000204100009642000062
:102DF000A0420000A0420000C8430000BE42E80319
:102E00000000EE020000640000004B00000024F40B
:102E1000D43050C38E20C2A24017828B7011127A18
:102E2000910D816CD90AA861E108C7586607615104
:102E300043061E4B5D05C145A7041A411104093D17
:102E40009803713931034036DB0265339102D43087
:102E50005402802E1D02632CEE01752AC501B02894
:102E6000A001102781018F2564012B244B01E02252
:102E70003401AC211F018D200D01801FFC00841E38
:102E8000ED00971DDF00B81CD200E61BC600201B1A
:102E9000BC00641AB200B219A8000A19A0006A188E
:102EA0009900D117910040178B00B5168400311698
:102EB0007E00B31579003A157300C7146F005814DB
:102EC0006A00EE1366008813630025135E00C712C4
:102ED0005B006C12570015125400C11151007011A3
:102EE0004F0021114B00D61049008D1047004610AD
:102EF000440002104200C00F4000800F3E00420F0D
:102F00003C00060F3B00CB0E3800930E37005C0EE2
:102F10003500270E3400F30D3200C10D3100900D45
:102F20003000600D2E00320D2D00050D2C00D90C47
:102F30002B00AE0C2900850C29005C0C2700350CF9
:102F400027000E0C2600E80B2400C40B2400A00B65
:102F500023007D0B23005A0B2100390B2100180B95
:102F60002000F80A1F00D90A1E00BB0A1E009D0A95
:102F70001D00800A1D00630A1C00470A1B002C0A62
:102F80001B00110A1A00F7091A00DD091900C4090B
:102F90001900AB091900920917007B091800630991
:102FA00017004C09160036091600200916000A09F8
:102FB0001500F5081500E0081400CC081400B80846
:102FC0001400A4081400900813007D0812006B0878
:102FD0001300580812004608120034081100230894
:102FE00011001208110001081100F0071000E0079D
:102FF0001000D0071000C0071000B0070F00A10795
:10300000100091070E0083070F0074070F0065077B
:103010000E0057070E0049070E003B070D002E0754
:103020000E0020070D0013070D0006070D00F9061E
:103030000C00ED060D00E0060C00D4060C00C806DE
:103040000C00BC060C00B0060C00A4060B00990690
:103050000C008D060B0082060B0077060B006C0639
:103060000B0061060A0057060B004C060A004206D8
:103070000A0038060A002E060A0024060A001A066C
:103080000A001006090007060A00FD050900F405FC
:103090000900EB050900E2050900D9050900D00582
:1030A0000900C7050900BE050900B5050800AD0502
:1030B0000800A50509009C050800940508008C057A
:1030C0000800840508007C050800740508006C05EC
:1030D0000700650508005D050700560508004E0558
:1030E00007004705070040050800380507003105BF
:1030F00007002A050700230507001C050600160522
:1031000007000F0507000805060002050700FB047D
:103110000600F5040700EE040600E8040600E204D9
:103120000700DB040600D5040600CF040600C9042E
:103130000600C3040600BD040600B7040600B1047F
:103140000500AC040600A6040600A00405009B04CC
:10315000060095040500900406008A040500850415
:103160000500800406007A0405007504050070045B
:1031700005006B04050066040500610405005C049D
:10318000050057040500520405004D0405004804DD
:103190000500430405003E0404003A04050035041C
:1031A0000500300404002C04050027040400230457
:1031B00005001E0404001A0404001604050011048E
:1031C00004000D04040009040500040404000004C4
:1031D0000400FC030400F8030400F4030400F003FB
:1031E0000400EC030400E8030400E4030400E0032B
:1031F0000400DC030400D8030400D4030400D0035B
:103200000400CC030400C8030300C503030024F436
:1032100004D9201BC40C5C0E9804C4095F02650726
:103220007101F405F900FB04B30048048700C103F1
:1032300069005803550003034500BE023A008402AA
:10324000310053022A002902250004022000E40173
:103250001C00C8011900AF01170098011400840177
:103260001300710110006101100051010E004301B3
:103270000D0036010B002B010B0020010B00150186
:1032800009000C01090003010800FB000800F3001D
:103290000800EB000700E4000600DE000600D8008E
:1032A0000600D2000600CC000500C7000500C200E1
:1032B0000500BD000400B9000400B5000400B10021
:1032C0000400AD000400A9000400A5000300A20052
:1032D00003009F0004009B0003009800030095007A
:1032E000020093000300900003008D0002008B0099
:1032F00003008800020086000200840003008100B1
:1033000002007F0002007D0002007B0002007900C5
:1033100002007700010076000200740002007200D3
:103320000100710002006F0002006D0001006C00DE
:1033300002006A00010069000200670001006600E7
:1033400001006500010064000200620001006100EC
:103350000100600001005F0002005D0001005C00F0
:1033600001005B0001005A000100590001005800F3
:1033700001005700010056000100550001005400F3
:1033800001005300000053000100520001005100F1
:103390000100500001004F0001004E0000004E00EF
:1033A00001004D0001004C0001004B0000004B00EB
:1033B00001004A00010049000100480000004800E7
:1033C00001004700010046000000460001004500E2
:1033D00000004500010044000100430000004300DC
:1033E00001004200000042000100410000004100D5
:1033F0000100400001003F0000003F0001003E00CE
:1034000000003E0001003D0000003D0001003C00C6
:1034100000003C0000003C0001003B0000003B00BD
:1034200001003A0000003A000100390000003900B4
:1034300001003800000038000000380001003700AB
:1034400000003700010036000000360000003600A2
:103450000100350000003500000035000100340097
:10346000000034000000340001003300000033008D
:103470000000330001003200000032000000320082
:103480000100310000003100000031000100300077
:10349000000030000000300001002F0000002F006D
:1034A00000002F0000002F0001002E0000002E0061
:1034B00000002E0001002D0000002D0000002D0056
:1034C00000002D0001002C0000002C0000002C004A
:1034D00000002C0001002B0000002B0000002B003E
:1034E00000002B0001002A0000002A0000002A0032
:1034F00000002A0001002900000029000000290026
:103500000000290000002900010028000000280018
:10351000000028000000280000002800010027000B
:1035200000002700000027000000270000002700FF
:1035300001002600000026000000260000002600F2
:1035400000002600010025000000250000002500E5
:1035500000002500000025000000250001002400D7
:1035600000002400000024000000240000002400CB
:1035700001002300000023000000230000002300BE
:1035800000002300000023000000230001002200AF
:1035900000002200000022000000220000002200A3
:1035A0000000220001002100000021000000210095
:1035B0000000210000002100000021000000210087
:1035C000010020000000200000002000000020007A
:1035D000000020000000200000002000000020006B
:1035E00001001F0000001F0000001F0000001F005E
:1035F00000001F0000001F0000001F0001001E004F
:1036000000001E0000001E0000001E000000232C11
:103610000000B8220000561800003A0F0000B80859
:103620000000B1040000710200003E0100002043D0
:103630006F756E7420583A0042656400453100622F
:103640006564002C2073797374656D2073746F70DA
:1036500070656421204865617465725F49443A2051
:103660000048656174696E67204661696C65640035
:1036700048656174696E67206661696C6564004DB8
:103680003131322053687574646F776E001000C951
:103690000210012C014001220170011801B0010E3D
:1036A00001F00104015002FA00B002F0003003E61C
:1036B00000D003DC009004D2007005C800A006BE54
:1036C000000008B400B009AA00D00BA000600E965C
:1036D0000060118C000015820020197800C01D6E5A
:1036E00000A0226400B0275A00902C500000314600
:1036F00000E0343C0010383200903A2800603C1E54
:1037000000A03D1400803E0A00203F0000544845C0
:10371000524D414C2052554E415741590054686515
:10372000726D616C2052756E6177617900457272BD
:103730003A204D415854454D50004D415854454D47
:103740005020747269676765726564004572723AE9
:10375000204D494E54454D50004D494E54454D5015
:103760002074726967676572656400202F002042CB
:10377000403A0020403A0020573A0020573A00498A
:103780006E76616C69642065787472756465720A1E
:10379000007C3C3E5E2B3D3F2F5B5D3B2C2A225C38
:1037A0000043616E6E6F74206F70656E207375627A
:1037B0006469722000534420496E6974204661692F
:1037C0006C0053442063617264206F6B0A006F7059
:1037D000656E526F6F74206661696C65640A00766D
:1037E0006F6C756D652E696E6974206661696C65B4
:1037F000640A004E6F20534420636172640A0041E2
:10380000425300504C41000A4D3234004D323320B7
:103810002573002E0A006F70656E206661696C6505
:10382000642C2046696C653A200046696C652073FB
:10383000656C65637465640A002053697A653A2093
:103840000046696C65206F70656E65643A200045BE
:103850004E4420535542524F5554494E450A00227A
:1038600020706F73002220706172656E743A2200BE
:10387000535542524F5554494E452043414C4C20DC
:103880007461726765743A220053756263616C6C8F
:10389000204F766572666C6F770045786365656466
:1038A0006564206D617820535542524F5554494EFE
:1038B000452064657074683A002E0A0044656C65A2
:1038C00074696F6E206661696C65642C2046696C52
:1038D000653A200046696C652064656C65746564B2
:1038E0003A005344207072696E74696E6720627981
:1038F000746520004E6F74205344207072696E749A
:10390000696E670A002F6175746F25632E67005713
:10391000726974696E6720746F2066696C653A20FD
:1039200000667265736800646F696E67002066697F
:103930006C653A20004E6F77200002FD55555555B5
:10394000555FFFFFFFFFFFFFFFFFFFFE00000000CE
:10395000003FFFFFFFFFFFFFFFFFFFFD000007FF2E
:10396000FFFFFFFFFFFFFFFFFFFFFFFE07C0055543
:10397000555555555FFFFFFFFFFFFFFC0A2006006E
:10398000000000003FFFFFFFFFFFFFFE14100500D7
:103990000007FFFFFFFFFFFFFFFFFFFC28080607F0
:1039A000C00555555555555FFFFFFFFE5404040AE9
:1039B000200600000000003FFFFFFFFC600406142B
:1039C0001005000007FFFFFFFFFFFFFE5004042863
:1039D000080607C00555555555555FFC600406544B
:1039E00004040A200600000000003FFE54041C608E
:1039F000040614100500000000001FFC28082E50CB
:103A0000040428080607C00001F03FFE14105460AB
:103A100004065404040A200002081FFC0A2066540D
:103A2000041C60040614100005043FFE07C054285F
:103A3000082E5004042808000A021FFC00002E145F
:103A4000105460040654040015013FFE00001C0AD7
:103A5000206654041C60040018011FFC00000607C7
:103A6000C05428082E50040014013FFE000004003A
:103A7000002E14105460040018011FFCFFFFFE000C
:103A8000001C0A206654041C15013FFED555540045
:103A9000000607C05428082A0A021FFC84104600AA
:103AA000000400002E14105105043FFEC41044FF12
:103AB000FFFE00001C0A206102881FFC841046D50E
:103AC000555400000607C05101F03FFE84104484A5
:103AD000104600000400002A00001FFCC41046C469
:103AE0001044FFFFFE00001C00003FFE84104484D1
:103AF0001046D5555400000000001FFCD5555684D3
:103B0000104484104600000000003FFCFFFFFCC48E
:103B10001046C41044FFFFFFFFFF9FFE0000068415
:103B20001044841046D555555555BFFD555554D5AF
:103B3000555684104484104104109FFFFFFFFCFF82
:103B4000FFFCC41046C410410411BFFFFFFFFE007C
:103B5000000684104484104104109FFFFFFFFD55B0
:103B60005554D5555684104104109FFFFFFFFFFFA9
:103B7000FFFCFFFFFCC410410411BFFFFFFFFFFF6C
:103B8000FFFE00000684104104109FFFFFFFFFFFAF
:103B9000FFFD555554D555555555BFFFFFFFFFFF48
:103BA000FFFFFFFFFCFFFFFFFFFF9FFFFFFFFFFF88
:103BB000FFFFFFFFFE00000000003FFFFFFFFFFFD1
:103BC000FFFFFFFFFD55555555555FFFFFFFFFFFF9
:103BD000FFFFFFFFFFFFFFFFFFFFFFFFFFFFFFFFF5
:103BE000FFFFFFFFFFFFFFFFFFFFFFFFFFFFFFFFE5
:103BF000FFFFFFFFFFFFFFFFFFFFFFFFFFFFFFFFD5
:103C0000FFFFFFFFFFFFFFFFFFFFFFE02EFB7DFB3E
:103C1000FBCFC1DFBB3EC0E1FE3C1FFDEE7B39F9AF
:103C2000F3CF9EDFBB3EDFDEFCDDE7FDEE3BBBF905
:103C3000EBD7BF5FBB5EDFDEFDEDF7FDEEBBD3FA7A
:103C4000EBB73FDFBB4EDFDFFFCDF3FDEEDBC7FAA7
:103C5000EBBB7FC03B6EC0E3FF1DF3FDEECBEFFA85
:103C6000DBBB7FDFBB66DFF8FFCDF3FDEEEBEFFBE9
:103C70005B033F5FBB76DFFE7FEDF3FDEEF3EFFB13
:103C80005B79BEDFBB7ADFDE7DEDF7FDEEF3EFFBA8
:103C9000BAFD9EDFBB7CDFDEFDCDE7FDEEFBEFFB7B
:103CA000BAFDC1DFBB7EC0E0FE1C1F6D61726C6996
:103CB0006E66772E6F726700322E302E375F445754
:103CC000372E332E31001FFFFFFFFFFFFF60000084
:103CD000000001FF400000000000FF800000000025
:103CE000007F83CF00000C303F87FF80000C301F27
:103CF000867980000C000F8C30C7838C30E78C30C5
:103D0000CFC7CC31F38C30DCECEC33B98C30D86CD1
:103D10006C33198C30D06C0C33198C30D86C0C335C
:103D2000198C30DC6C0E3B198C30CF7C079F198CC2
:103D300030C77C038F1940000000000002600000C3
:103D4000000000061FFFFFFFFFFFF870012C01902D
:103D5000012701B0012201C0011D01F0011801106D
:103D600002130130020E016002090190020401C039
:103D700002FF000003FA004003F5008003F000D0CA
:103D800003EB002004E6007004E100E004DC0040E6
:103D900005D700C005D2004006CD00D006C800807F
:103DA00007C3003008BE00F008B900C009B400B075
:103DB0000AAF00B00BAA00D00CA500000EA0005066
:103DC0000F9B00C01096005012910000148C00C090
:103DD000158700B0178200B0197D00D01B78000055
:103DE0001E730040206E0090226900F024640040A1
:103DF000275F0090295A00E02B5500102E5000201C
:103E0000304B0010324600E033410090353C00104A
:103E100037370070383200A0392D00B03A2800A0A2
:103E20003B2300603C1E00103D1900903D14001023
:103E30003E0F00703E0A00C03E0500003F000040FB
:103E40003FFBFF803FF6FFC03FF1FF2020506C6139
:103E50006E6E657242756666657242797465733A14
:103E600020002046726565204D656D6F72793A209D
:103E700000436F6D70696C65643A20417072203246
:103E80003920323032310A00204C61737420557071
:103E900064617465643A20323032312D30342D3112
:103EA00038207C20417574686F723A2054696E79AD
:103EB0004D616368696E657333440A00322E302E9B
:103EC000375F4457372E332E310A004D61726C69CB
:103ED0006E0020536F66747761726520526573655A
:103EE000740A00205761746368646F6720526573B9
:103EF00065740A002042726F776E206F75742052CD
:103F0000657365740A002045787465726E616C2073
:103F100052657365740A00506F77657255700A00B8
:103F200073746172740A004739310A47315A350A8D
:103F30004739300A4D38340A4D31303453300A4D48
:103F40003134305330004D31303031006572726F92
:103F5000722077726974696E6720746F2066696C6D
:103F6000650A00446F6E6520736176696E6720662E
:103F7000696C652E0A004D323900456E6473746FAA
:103F80007073002553202563202563202563202599
:103F90006300205A3A0020593A0020583A00656ED2
:103FA0006473746F7073206869743A200000000AAB
:103FB0000B02090C0D0E08070304010000000000AD
:103FC00000000000000000000000000000000000F1
:103FD00000000000000000000012111000000000AE
:103FE00000000000000000000000000000000000D1
:103FF000000000004D6F76652025736D6D004D6FDC
:10400000766520302E316D6D004D6F766520316DF7
:104010006D004D6F76652031306D6D004D6F7665AA
:104020002041786973004578747275646572004D3B
:104030006F7665205A004D6F76652059004D6F767A
:10404000652058000338FF374368616E6765204676
:10405000696C616D656E7400556E6C6F61642046AD
:10406000696C616D656E74004C6F61642046696CAB
:10407000616D656E7400507265686561742043758A
:1040800073746F6D0050726568656174202400421E
:1040900061636B00FFFFFF486F6D6520257325731B
:1040A00025732046697273740073686F77006275B8
:1040B00074746F6E00626567696E00446973616253
:1040C0006C6552756E6F75740050757267654D6FD3
:1040D00072650050617573656400436F6E74696E3C
:1040E0007565004C6F61642046696C616D656E7426
:1040F000205400496E736572742066696C616D6549
:104100006E7420616E642073656E64204D313038AA
:104110000A00220A00556E6B6E6F776E20636F6D1A
:104120006D616E643A2022002042002050006F6BC7
:1041300000343030205375506552205265616479E7
:104140002E005072696E74696E672E2E2E005072AA
:10415000696E742050617573656400204500205AB3
:1041600000205900204D393220580020453A0020C7
:104170005A3A0020593A00583A0020746F6F206C68
:104180006F6E6720657874727573696F6E207072D8
:104190006576656E7465640A0020636F6C642065E3
:1041A0007874727573696F6E2070726576656E745F
:1041B00065640A00526573656E643A20006E6F7420
:1041C000696669636174696F6E20000000220025D2
:1041D0000028002B002E00310034000201000005F1
:1041E0000108010B0100002100240027002A002DF6
:1041F000003000330001010000040107010A01053D
:10420000050505070508080808020202020A0A084F
:104210000804040404010101010101010103030375
:104220000303030303040707070C0C0C0C0C0C0C12
:104230000C0202020206060606060606060B0B0B19
:104240000B0B0B0B0B010210202008081020401054
:10425000204080020102010804020101020408104A
:104260002040808040201008040201800402018068
:104270004020100804020108040201010204081091
:10428000204080010204081020408000B8015E0137
:1042900011241FBECFEFD1E2DEBFCDBF00E00CBFC7
:1042A00013E0A0E0B2E0ECE2F1EC02E00BBF02C0F0
:1042B00007900D92A037B107D9F729E1A0E7B3E045
:1042C00001C01D92AA39B207E1F711E2C7E4D1E2B9
:1042D00000E006C021970109802FFE010F94EC5CDD
:1042E000C634D10780E00807A9F70F949E4B0D94C0
:1042F00084600C940000FC0184910895FC0180818D
:1043000008951198000000009091020187FD90959A
:10431000917090930001119A0000000000000000CD
:104320001198000000009091020186FD9095917017
:1043300090930001119A0000000000000000119805
:10434000000000009091020185FD9095917090937E
:104350000001119A00000000000000001198000008
:1043600000009091020184FD90959170909300015E
:10437000119A0000000000000000119800000000E9
:104380009091020183FD9095917090930001119A94
:104390000000000000000000119800000000909153
:1043A000020182FD9095917090930001119A000096
:1043B0000000000000001198000000009091020130
:1043C00081FD9095917090930001119A000000007A
:1043D000000000001198000000008091020181702F
:1043E00080930001119A0000000000000000089571
:1043F00090E080E00895CF93DF93DB01F9019C9179
:104400009130C1F0943080F094509C938830D1F476
:1044100080819181009771F0019791838083480F8B
:10442000591FEA01188206C08C3539F49C5F9C93B1
:10443000943041F4DF91CF9108958B3339F781E0C7
:104440008C93F8CF20813181B9016F5F7F4F7183E9
:104450006083420F531FEA018883808191818F35E9
:1044600091056CF7E7CF0F931F9381E000918117BF
:1044700010918217209183173091841740917D17F6
:1044800050917E1760917F17709180170417150760
:104490002607370708F480E01F910F91089590E0F8
:1044A00080E00895282F90911209833021F495FD22
:1044B0000FC094FD0FC0892F90E0B0E0A0E004C0D1
:1044C000B695A795979587952A95D2F78170089507
:1044D00081E0089580E008951092F90880915102DA
:1044E00090915202A0915302B09154028093E00641
:1044F0009093E106A093E206B093E3060895129A22
:104500000895269A2E9A0895AF92BF92CF92DF9285
:10451000EF92FF920F931F93CF93DF936B01E9010B
:104520004A3009F4C1C0453109F073C0DB0112966D
:10453000ED91FC91F280C681D78180910201809536
:1045400082708093000188E28A950000E9F7BF2C11
:10455000B29420EFB22230E1A32EAF0C48E2E42E59
:1045600088EF0E9481218E2D8A950000E9F7BFE136
:10457000BF1508F485C08F2D807780680E94812147
:104580008B2D0E9481218E2D8A950000E9F780E80D
:104590000E94812180E00E9481218E2D8A95000059
:1045A000E9F78AEF0E9481218E2D8A950000E9F7B4
:1045B0008E01005F1F4F8881807F0E948121899139
:1045C0008295807F0E948121C017D107A1F78E2D8F
:1045D0008A950000E9F7F394E0E1BE0EFA10C0CF2F
:1045E00080910201827080930001D6011296CD91D4
:1045F000DC91CE010F94FE3E811147C2DF91CF9135
:104600001F910F91FF90EF90DF90CF90BF90AF90F0
:104610000895FB0102811381423309F4F1C108F4CA
:10462000F5C1463409F4E2C1473409F4E5C14B331E
:1046300029F589812B81D80112966C9112971396D6
:104640004C91213009F438C2233009F002C238EF0E
:10465000380F582F91E0431708F490E041E05317CA
:1046600008F040E031E0561708F430E0592F542BA1
:10467000352309F016C2942309F013C281E0BECF9E
:1046800080EE8F0D8068807F0E9481218F2D829522
:10469000807F0E9481218E2D8A950000E9F780E8B5
:1046A0000E94812180E877CF809101018260809310
:1046B00001018091020182708093000180910101CB
:1046C00081608093010180910201817080930001DB
:1046D000099A119A8091020180958270809300015D
:1046E00088E28A950000E9F788E790E0CEE9DFE00C
:1046F000FE013197F1F70197D9F788EF0E948121E8
:1047000018E2812F8A950000E9F780E20E9481215A
:1047100080E00E948121812F8A950000E9F780E0E6
:104720000E94812180E80E948121812F8A950000CA
:10473000E9F780E00E94812180E10E948121812FA0
:104740008A950000E9F7CE010197F1F7CE010197B4
:10475000F1F7CE010197F1F7CE010197F1F7CE0104
:104760000197F1F7CE010197F1F7CE010197F1F72B
:10477000CE010197F1F7CE010197F1F7CE01019734
:10478000F1F7CE010197F1F7CE010197F1F7CE01D4
:104790000197F1F7CE010197F1F72197F1F780E248
:1047A0000E94812180E40E948121812F8A9500004E
:1047B000E9F780E20E94812180E60E9481211A951A
:1047C0000000E9F710E0D0E0C8E28D2F8077806824
:1047D0000E948121812F0E9481218C2F8A950000C7
:1047E000E9F780E80E94812180E00E9481218C2FDE
:1047F0008A950000E9F78AEF0E9481218C2F8A9523
:104800000000E9F790E21198000000008091020199
:10481000817080930001119A0000000000000000E8
:1048200011980000000080910201817080930001C6
:10483000119A000000000000000011980000000024
:1048400080910201817080930001119A00000000A4
:1048500000000000119800000000809102018170AA
:1048600080930001119A00000000000000001198E0
:104870000000000080910201817080930001119A74
:10488000000000000000000011980000000080916E
:104890000201817080930001119A00000000000065
:1048A0000000119800000000809102018170809347
:1048B0000001119A000000000000000011980000A3
:1048C000000080910201817080930001119A000024
:1048D000000000000000119800000000809102011B
:1048E000817080930001119A000000000000000018
:1048F00011980000000080910201817080930001F6
:10490000119A000000000000000011980000000053
:1049100080910201817080930001119A00000000D3
:1049200000000000119800000000809102018170D9
:1049300080930001119A000000000000000011980F
:104940000000000080910201817080930001119AA3
:10495000000000000000000011980000000080919D
:104960000201817080930001119A00000000000094
:104970000000119800000000809102018170809376
:104980000001119A000000000000000011980000D2
:10499000000080910201817080930001119A000053
:1049A0000000000000008C2F8A950000E9F791506C
:1049B00009F029CF88EF0E9481218C2F8A95000071
:1049C000E9F7DF5F105FD03209F0FFCE80E00E9490
:1049D000812180EC0E948121CA950000E9F7809135
:1049E000020182708093000181E008CED801159603
:1049F0008C91888381E002CEF80181818883FACF8F
:104A0000B901C8010F941B3F81E0F8CD443171F02A
:104A1000473109F033CE1882F8018281898385817C
:104A200081508A8383818B8381E0E8CDD8011596FC
:104A30004C91159750E0440F551F70E060E01696BA
:104A40008D919C910F942560C8010F94143F81E0D3
:104A5000D5CD481708F412CE861708F40FCEFA8089
:104A6000E12CD12C243070F41DC0BE01C8010F947C
:104A70001B3F898198819D0D98838E0D8983FF0C42
:104A800009F4FCCDF7FEF6CFF0CF4D8150E0440F96
:104A9000551F70E060E08E819F810F94256081E05A
:104AA000ADCDFA8030E0F901E555FD4FD0802955B4
:104AB0003D4FF901E080E6CF58E0580F382FCACDBE
:104AC000EF92FF920F931F93CF93DF93EC018B0133
:104AD0007A018A859B858617970731F088819981AD
:104AE0000F94F4401B870A87B701888199810F943E
:104AF0009D322E813F81820F932F911D9F838E8344
:104B000090E080E0DF91CF911F910F91FF90EF90A7
:104B100008959F92AF92BF92CF92DF92EF92FF9251
:104B20000F931F93CF93DF93EC018B01942EA52E4F
:104B30008A859B858617970731F0888199810F9424
:104B4000F4401B870A8788859985019649F5BC80C2
:104B50000A818E81080FC880D980D6015596ED91C3
:104B6000FC91C6011995B80EE92CFA2C10E0F7015A
:104B700021917F01211127C08E819F81810F911D7D
:104B80009F838E8390E080E0DF91CF911F910F9102
:104B9000FF90EF90DF90CF90BF90AF909F900895DF
:104BA0000E811F81692D7A2D888199810F949D3204
:104BB000800F912F911D288539852817390738F6E0
:104BC00081E090E0E1CF4B2D602FC6010F944C4166
:104BD000080F180FCCCFDF92EF92FF920F931F9325
:104BE000CF93DF93EC01D62E1CAD0BAD7C0184E09E
:104BF000E80EF11CE98DFA8DC7011995412F480F78
:104C00002D2D602FC7010F944C419BAD890F8BAFA9
:104C100081E090E0DF91CF911F910F91FF90EF9095
:104C2000DF900895AB01BC01409381175093821728
:104C300060938317709384178AEE98E10C9496D151
:104C4000809323028032B8F590910F05891724F0E4
:104C500091E0980F90930F0540910B0550910C0532
:104C600060910D0570910E05082E04C0769567952C
:104C7000579547950A94D2F741704093FE1087FDEF
:104C80001DC0282F082E000C330B3F938F9386E80E
:104C900099E09F938F9386E999E09F938F931F925A
:104CA0000E9477B58DB79EB707960FB6F8949EBF52
:104CB0000FBE8DBF08951092FE10E1CF0D940446F3
:104CC0000F931F93CF93DF9300D01F92CDB7DEB722
:104CD0009C0100EE18E090E1E9E4F1E1D8010190D7
:104CE0000D929A95E1F7F90120813181428153813A
:104CF000F80160857185828593850F94F55CF801D4
:104D0000608771878287938780E090E0A0EAB0E4B3
:104D100089839A83AB83BC83CE0101960E9456FCA3
:104D20000F900F900F900F90DF91CF911F910F91E7
:104D300008952F923F924F925F926F927F928F923F
:104D40009F92AF92BF92CF92DF92EF92FF921F930A
:104D5000CF93DF93CDB7DEB72C970FB6F894DEBFB5
:104D60000FBECDBF7A011901DC012D913D914D910E
:104D70005C912D833E834F835887FB014080518097
:104D8000628073808090491190904A11A0904B11DD
:104D9000B0904C11A50194016D817E818F81988521
:104DA0000F94035681110EC011E0A301920160918E
:104DB0004D1170914E1180914F11909150110F949F
:104DC0000356811110E0D1012D913D914D915C91DF
:104DD00029873A874B875C87F701C080D180E280C2
:104DE000F3802091090230910A0240910B02509108
:104DF0000C02C701B6010F940356882309F44EC074
:104E0000C0920902D0920A02E0920B02F0920C02C8
:104E10008091551190915611A0915711B091581150
:104E200040914D1150914E1160914F117091501160
:104E30008092E0089092E108A092E208B092E30824
:104E40004093E4085093E5086093E6087093E70800
:104E5000C092E808D092E908E092EA08F092EB08E4
:104E60008093EC089093ED08A093EE08B093EF08C0
:104E700020E030E040E05FE360912C1170912D1153
:104E800080912E1190912F110F94695669837A8326
:104E90008B839C83CE0101960E9456FC2D813E811E
:104EA0004F8158852093E0083093E1084093E20851
:104EB0005093E3084092E4085092E5086092E608B7
:104EC0007092E708D1012D913D914D915C916091D7
:104ED000EC087091ED088091EE089091EF080F9426
:104EE000F55C6093EC087093ED088093EE08909366
:104EF000EF0811112FC020E030E0A90169857A8503
:104F00008B859C850F940356811133C060E070E05F
:104F100088EC92E469837A838B839C83CE0101962B
:104F20000E9456FC2C960FB6F894DEBF0FBECDBF84
:104F3000DF91CF911F91FF90EF90DF90CF90BF90C6
:104F4000AF909F908F907F906F905F904F903F9029
:104F50002F9008952AEF3EE74AE25FE36091301117
:104F60007091311180913211909133110F946956E3
:104F7000D1CF60E070E080EA91E4CCCF8091C604AC
:104F80009091C704009731F04AE050E070E060E093
:104F90000D941E5460E070E0CB01089580910B0ADF
:104FA00082FF0BC063E682E79AE00E9492B50F94FD
:104FB00008390E945DBC81E0089580E008958091E9
:104FC000C6049091C704009731F04AE050E070E0C9
:104FD00060E00D94F05260E070E0CB010895AF9274
:104FE000BF92CF92DF92EF92FF920F931F93CF93D6
:104FF000DF93EC015B018A01FB01199587FD16C067
:10500000C82ED12CF12CE12C2196F801C082D1823E
:10501000E282F382CE01DF91CF911F910F91FF9039
:10502000EF90DF90CF90BF90AF900895982F907E33
:10503000903CA9F48F7190E0B0E0A0E06C017D019C
:1050400056E0CC0CDD1CEE1CFF1C5A95D1F7CE01AE
:105050000196F50119958F73C82A2296D6CF982FFD
:10506000907F903E11F58F7090E0B0E0A0E06C0171
:105070007D0136E0CC0CDD1CEE1CFF1C3A95D1F70F
:10508000CE010196F50119958F73C82A46E0CC0C24
:10509000DD1CEE1CFF1C4A95D1F7CE010296F501EE
:1050A00019958F73C82A2396B0CF982F987F903F79
:1050B00079F5877090E0B0E0A0E06C017D0186E0BA
:1050C000CC0CDD1CEE1CFF1C8A95D1F7CE0101969D
:1050D000F50119958F73C82A96E0CC0CDD1CEE1CE7
:1050E000FF1C9A95D1F7CE010296F50119958F73A1
:1050F000C82A26E0CC0CDD1CEE1CFF1C2A95D1F73B
:10510000CE010396F50119958F73C82A24967DCF99
:10511000982F907C903841F4807C803869F42196F7
:10512000CE01F5011995F8CF8E7F8D3F28F021969D
:10513000CE01F5011995F8CFC12CD12C760165CFA0
:105140009CE0899F802D112491E0980F9093100589
:105150002CE0280F2093DA0830E02E5F3F4F40917B
:1051600033174217130619F014F080E008952091C8
:1051700035179217D0F7662341F08E5F0F940E40DB
:105180008091DA088E5F0F940E408091DA0890913A
:105190003317891750F3209135179091100529176F
:1051A00020F3109236178093371781E00895CF933C
:1051B00080910205811154C0109236171092371752
:1051C00010923817109204171092031710920617B6
:1051D000109205171092081781E08093071782E25A
:1051E0008093091710920E1710920D17E2E2F7E163
:1051F00020E337E18FEF81932E173F07E1F7C1E0FE
:10520000C0931F1722E431E0309315172093141731
:10521000C0931617109217171092181790E49093D6
:10522000191710921A172EEA30E030933117209395
:10523000301726E132E0309302172093011797E1EF
:105240009093261791E19093271790E1909324175C
:1052500080932317809322170F94353FC093020544
:1052600081E08093030587E497E190937216809321
:1052700071161092741610927316CF9108952091A2
:105280000105022E000C330B8217130641F08093A8
:10529000010567E477E18FEF96E10D94F4400895FE
:1052A000CF92DF92EF92FF920F931F93CF93DF93F2
:1052B000CDB7DEB72C970FB6F894DEBF0FBECDBFCB
:1052C0006F3F71058105910509F0D0F48BEF96E1F0
:1052D0000E94EB25E0910317F09104173196849119
:1052E00090E02C960FB6F894DEBF0FBECDBFDF91D5
:1052F000CF911F910F91FF90EF90DF90CF90089585
:10530000F0903617E09037172091030521110FC058
:1053100047E257E16E2D8F2D0F94B84190E080E069
:10532000F80EF0923617E09237179927DACFC0902F
:105330000317D09004172FEF36E13A8329832F2DDE
:1053400030E03C832B832E2D30E03E832D83188666
:105350001F822FEF3FEF3A8729871C861B8609E8BB
:1053600015E29E012F5F3F4FAB01BC01C6010F94B8
:10537000DA28B6018FEF96E10F94F4408F8198857B
:10538000CFCFCF93DF93FC0125AD211104C021E0E5
:1053900025AF0F94353FC0910117D0910217E091CE
:1053A0003017F091311782E01995E0913017F091A4
:1053B000311781E0199530E020E044E1BE018FEF24
:1053C00096E10F94313F22E337E147E1BE018FEFD1
:1053D00096E10F94313FE0913017F091311780E062
:1053E000DF91CF911994CF92DF92EF92FF920F93BA
:1053F0001F93CF93DF93CDB7DEB72C970FB6F894FA
:10540000DEBF0FBECDBFF0903617E090371720916A
:10541000030521111DC047E057E16E2D8F2D0F941C
:10542000B84190E080E0F80EF0923617E09237171E
:1054300099272C960FB6F894DEBF0FBECDBFDF9133
:10544000CF911F910F91FF90EF90DF90CF90089533
:10545000C0900317D09004172FEF36E13A832983C9
:105460002F2D30E03C832B832E2D30E03E832D8387
:1054700018861F827A8769871C861B8609E815E2D1
:105480009E012F5F3F4F4BE751E2BC01C6010F94D5
:105490009E29B6018FEF96E10F94F4408F81988595
:1054A000C2CF6FEF7FEF0C94F329CF92DF92EF9290
:1054B000FF920F931F93CF93DF93CDB7DEB72C9757
:1054C0000FB6F894DEBF0FBECDBFF0903617E09058
:1054D00037172091030521111DC047EE56E16E2DAF
:1054E0008F2D0F94B84190E080E0F80EF0923617BF
:1054F000E092371799272C960FB6F894DEBF0FBEAF
:10550000CDBFDF91CF911F910F91FF90EF90DF9072
:10551000CF900895C0900317D09004172FEF36E175
:105520003A8329832F2D30E03C832B832E2D30E0CE
:105530003E832D8318861F827A8769871C861B8687
:1055400009E815E29E012F5F3F4F4EE751E2BC0193
:10555000C6010F949E29B6018FEF96E10F94F44097
:105560008F819885C2CFBF92CF92DF92EF92FF9248
:105570000F931F93CF93DF938B01F42EE90141FB2F
:10558000662760F90E94A028882309F45AC0B12C2C
:105590000115110521F0C8010E942EBDB82EE12C85
:1055A000209721F0CE010E9419BFE82E80E8C82E76
:1055B000D12CF0FE1EC085E190E08B199109B7FC5B
:1055C00093958E199109E7FC939597FD0196959512
:1055D0008795F82E30E8C32ED12CFA94F7FC09C039
:1055E00060E270E080E090E00E945029C81AD90A79
:1055F000F4CFBB2099F0C60166E070E00F94C45C64
:10560000262F4091DC085091DD086091DB08C8012D
:105610000E946EBC96E0899F60011124EE2031F05B
:10562000B601CE010E94552AC81AD90A87E0C816C9
:10563000D10438F060E270E080E090E00E945029F0
:10564000F3CFDF91CF911F910F91FF90EF90DF90FB
:10565000CF90BF9008956FEF7FEF0C94552AAF92D3
:10566000BF92CF92DF92EF92FF920F931F93CF934F
:10567000DF935C016B010E942EBDE82EC6010E94E3
:1056800019BFF12C03E110E0081B1109C5E20E154A
:105690001F050CF4CFE18C2F90E09C012E5F3F4F53
:1056A000409133174217130609F0CCF50997209162
:1056B0003517281719069CF14091DC085091DD0838
:1056C0006091DB0810923617C093371725E1C501AA
:1056D0000E946EBCD1E0C114D104B1F06AE370E065
:1056E00080E090E00E9450290E151F05D4F4C45F9D
:1056F00080913317C81740F0209135174C2F49502F
:10570000550B241715067CF4DF91CF911F910F9153
:10571000FF90EF90DF90CF90BF90AF900895D0E0D2
:10572000DACFDD2389F3802F880F080F000F009355
:105730003617C093371760E270E080E090E00E9477
:105740005029C601DF91CF911F910F91FF90EF90EB
:10575000DF90CF90BF90AF900C942B2B8F929F92A5
:10576000AF92BF92CF92DF92EF92FF920F931F936F
:10577000CF93DF93CDB7DEB72C970FB6F894DEBF8B
:105780000FBECDBF982F862F5A017901D02E692FD9
:105790000E94A028882309F489C0C701002391F141
:1057A0000E942EBDC82E8090031790900417809100
:1057B0000305811145C01FEF23E12C194091DC083E
:1057C0005091DD086091DB08C5010E946EBCCC20C1
:1057D00009F46CC0B6E08B9F500111246AE370E0BD
:1057E00080E090E00E94502957E0A516B10408F42B
:1057F00044C060E270E080E090E00E945029A81A66
:10580000B90AF2CF0E9419BFC82E8090031790905A
:10581000041780910305882371F2FE0133968AE014
:10582000DF011D928A95E9F78FEF96E19A838983CC
:1058300000E615E29E012F5F3F4F4EE751E212C096
:10584000FE0133968AE0DF011D928A95E9F78FEF1A
:1058500096E19A83898300E615E29E012F5F3F4F10
:105860004BE751E2B701C4010F949E29B4018FEFB9
:1058700096E10F94F4401F819FCF4091DA08212FC9
:1058800030E0A6E0CA9EC00111242E5F3F4F2817CA
:1058900039070CF49C0180E8821B809336174093F3
:1058A0003717C701DD20A9F00E94512A2C960FB6A8
:1058B000F894DEBF0FBECDBFDF91CF911F910F9146
:1058C000FF90EF90DF90CF90BF90AF909F908F9020
:1058D00008950E942B2BEACFEBEFF6E183AF64AF84
:1058E000CA010C942B2B2F923F924F925F926F9292
:1058F0007F928F929F92AF92BF92CF92DF92EF9260
:10590000FF920F931F93CF93DF93D62FC72FFC01E6
:1059100080809180A280B380C501B40120E831E588
:1059200041E050E00F94475CC9016DE671E00F94CF
:10593000C45C6B017C01C501B40120E13EE040E0A4
:1059400050E00F94475CCA01B90128E130E040E023
:1059500050E00F94475C362E272E062F172F8CE32E
:10596000482E512C612C712CC501B401A301920168
:105970000F94475CB62EA72ECA01B901A30192016C
:105980000F94475CCB01C114D10479F1AF92BF925F
:105990007F936F932F923F92FF92EF92DF92CF927D
:1059A00085E495E19F938F93CF93DF930F949A555E
:1059B0008DB79EB70E960FB6F8949EBF0FBE8DBFE3
:1059C0008D2F9C2FDF91CF911F910F91FF90EF9022
:1059D000DF90CF90BF90AF909F908F907F906F900F
:1059E0005F904F903F902F900895E114F104C9F01B
:1059F000AF92BF927F936F932F923F92FF92EF925D
:105A000085E395E19F938F93CF93DF930F949A55FE
:105A1000EDB7FEB73C960FB6F894FEBF0FBEEDBFD4
:105A2000CFCF012BB9F0AF92BF927F936F932F929C
:105A30003F9289E295E19F938F93CF93DF930F94E9
:105A40009A558DB79EB70A960FB6F8949EBF0FBEB3
:105A50008DBFB6CF892BA9F0AF92BF927F936F9382
:105A600081E295E19F938F93CF93DF930F949A55A3
:105A7000EDB7FEB738960FB6F894FEBF0FBEEDBF78
:105A80009FCFAF92BF928DE195E19F938F93CF937C
:105A9000DF930F949A550F900F900F900F900F90E7
:105AA0000F908ECF8F929F92AF92BF92CF92DF9244
:105AB000EF92FF920F931F93CF93DF931092000505
:105AC0001092FF042FE32093FE041092FD04109225
:105AD000FC041092FB041092F7041092F804109248
:105AE000F9041092FA049C01F90190812F5F3F4F55
:105AF0009032D1F39E34C9F4818190ED980F9A30A1
:105B000020F08D3211F08B3281F432969F012F5F9D
:105B10003F4F808180538A3008F47BC09F012F5F04
:105B20003F4F8081803209F476C0F093FF08E09304
:105B3000FE088F010F5F1F4FC0816AE270E0C8014D
:105B40000F944A60009731F0FC01319780818032D8
:105B5000E1F31182CD3429F0C43519F0C73409F0CE
:105B60004BC0F80180810F5F1F4F8032D1F380530B
:105B70008A3008F041C0C093FE0430E020E04AE0E3
:105B8000DF011196429FC001439F900D11249C019B
:105B9000205331098081280F311D87FD3A9581817D
:105BA00090ED980F9A30C8F13093FD042093FC04D7
:105BB0008E3261F4329690E04AE0DF0131968C91AA
:105BC00050ED580F5A3058F19093FB04CD01DC0191
:105BD00001964C914032D9F3CD3489F52E313105FF
:105BE00039F018F52731310519F02C31310539F527
:105BF000B0930005A093FF04DF91CF911F910F9107
:105C0000FF90EF90DF90CF90BF90AF909F908F90DC
:105C10000895F9017BCFF90181CFFD01B1CF949FA8
:105C2000800D112490ED980FC8CF2537310538F03D
:105C300027373105E8F2203A83E03807C9F2D091DE
:105C4000FE0840E050E0BA0110E000E0C12CD12C89
:105C50007601C394FD0131968C91882309F47FC0AD
:105C60008132E1F4CD34D1F420323105B9F44093DE
:105C7000F7045093F8046093F9047093FA04F093D6
:105C80000005E093FF0463E270E0CF010F944A60E7
:105C9000009709F4B1CFFC011082AECF81548A3154
:105CA00008F058C0DF019D91903291F0A0EDA90F4E
:105CB000AA30E8F09E3271F4918190539A30B8F096
:105CC0000115110519F48F010150110990E013C05D
:105CD000FD01E8CF9D3211F09B3291F79181A0ED4B
:105CE000A90FAA3020F09E3259F79281E6CF9E2F5D
:105CF0009D1B309759F3A82FB0E04601570104C00F
:105D0000880C991CAA1CBB1C8A95D2F748295929D2
:105D10006A297B29A352BB4F9C9380818154DF0168
:105D20008A3108F497CFDF018191882309F492CF5B
:105D300090ED980F9A30B8F393ED980F923098F356
:105D40008B3289F3CD010196EC91E03209F082CFDC
:105D5000DC01F8CF0115110501F78D01DECF10939D
:105D600000050093FF044093F7045093F8046093F8
:105D7000F9047093FA0440CF9B01AC01485F5F4F78
:105D8000BC016C5F7F4F0C9499260F931F93CF93A8
:105D9000DF9300D000D01F921F92CDB7DEB7FC0179
:105DA0008B0183A5811112C081E083A78481958135
:105DB000A681B781B05889839A83AB83BC83BE0127
:105DC0006F5F7F4F80EE98E00E94BC2E1D821E8286
:105DD0001F82188620E030E040E05FE360915111BF
:105DE0007091521180915311909154110F94F55C60
:105DF00069837A838B839C839E012B5F3F4FAE0127
:105E00004F5F5F4F6DE471E189E491E10E94992653
:105E10001D821E821F82188620E030E040E05FE392
:105E2000F80160857185828593850F94F55C69839F
:105E30007A838B839C83B8016C5F7F4F9E012B5FBD
:105E40003F4FAE014F5F5F4FC8010E9499262896D1
:105E50000FB6F894DEBF0FBECDBFDF91CF911F917B
:105E60000F9108952F923F924F925F926F927F927F
:105E70008F929F92AF92BF92CF92DF92EF92FF925A
:105E80000F931F93CF93DF93CDB7DEB7A2970FB6D3
:105E9000F894DEBF0FBECDBF8C011B015E834D8326
:105EA0004090491150904A1160904B1170904C11E4
:105EB00080904D1190904E11A0904F11B0905011C4
:105EC000DB018D919D910D90BC91A02D8F87988BBA
:105ED000A98BBA8B9C01AD01C301B2010F94F45C94
:105EE0006B017C01D10114968D919D910D90BC9117
:105EF000A02D8B8B9C8BAD8BBE8B9C01AD01C50106
:105F0000B4010F94F45C6F8B788F898F9A8FAD8179
:105F1000BE818D919D910D90BC91A02D8F8398870E
:105F2000A987BA879C01AD01C301B2010F94F45C4B
:105F30006B8F7C8F8D8F9E8FAD81BE8114968D91DE
:105F40009D910D90BC91A02D8B879C87AD87BE87BE
:105F50009C01AD01C501B4010F94F45C6F8F78A36F
:105F600089A39AA3A7019601C701B6010F946956A8
:105F70006B017C012F89388D498D5A8DCA01B90179
:105F80000F9469569B01AC01C701B6010F94F55CF3
:105F90004B015C012F85388949895A896F81788541
:105FA00089859A850F94F45C2B013C012B893C89EF
:105FB0004D895E896B857C858D859E850F94F45C0B
:105FC0006B017C01A3019201C301B2010F946956D8
:105FD0002B013C01A7019601C701B6010F94695638
:105FE0009B01AC01C301B2010F94F55C0F94A35F58
:105FF0006B017C012B8D3C8D4D8D5E8DCA01B901ED
:106000000F9469562B013C012F8D38A149A15AA14B
:10601000CA01B9010F9469569B01AC01C301B201D9
:106020000F94F55C9B01AC01C501B4010F94555F61
:106030001816B4F520E030E0A901C701B6010F94AD
:10604000555F87FF2AC0C701B601905820E030E0B5
:1060500040EA50E40F94555F181614F5A1016D81C4
:106060007E81C8010E94322FA2960FB6F894DEBF3F
:106070000FBECDBFDF91CF911F910F91FF90EF9099
:10608000DF90CF90BF90AF909F908F907F906F9058
:106090005F904F903F902F900895C701B601D6CFE3
:1060A00020E030E040E050E4C501B4010F94555FBA
:1060B000181624F4B101C8010E94C52E19821A8253
:1060C0001B821C82BE016F5F7F4FC1010E94BC2EEC
:1060D0002DEC3CEC4CEC5CE3C701B6010F94695627
:1060E0009B01AC01F80160817181828193810F94E1
:1060F000695669837A838B839C83C8010F94CF315F
:10610000BE016F5F7F4F8D819E810E94BC2EACCF00
:106110004F925F926F927F929F92AF92BF92CF9277
:10612000DF92EF92FF920F931F93CF93DF93CDB740
:10613000DEB768970FB6F894DEBF0FBECDBFFB0188
:106140009080342F390D383008F026C1E180022FBD
:106150000E0D083008F020C1EE2DF0E0E654FB4FA4
:106160004080512C712C612C092C04C076946794CA
:10617000579447940A94D2F740FE0EC110E0F801FC
:10618000E654FB4F4080512C712C612CC32ED12C36
:1061900004C076946794579447943A95D2F740FE9A
:1061A000FBC0F22E642F5C01660F770B072E000CEC
:1061B000880B990B0F940A562B013C01892D94E012
:1061C0008902F0011124E65AF84EA3019201608180
:1061D0007181828193810F94F55C6D877E878F87B3
:1061E000988BF601EE0FFF1FEE0FFF1FE65AF84ED9
:1061F000A301920160817181828193810F94F45C8B
:1062000069837A838B839C836F2D660F770B072EB0
:10621000000C880B990B0F940A562B013C018E2D14
:1062200094E08902F0011124E65CF84EA30192018A
:1062300060817181828193810F94F55C698B7A8B87
:106240008B8B9C8B000F111F000F111FF801E65C58
:10625000F84EA301920160817181828193810F9434
:10626000F45C6D837E838F839887F50180859185AB
:10627000A285B38589879A87AB87BC878D8B9E8BD8
:10628000AF8BB88F4FE851E061E070E0CE014196EE
:106290000E9483D84FE851E061E070E0CE0105969E
:1062A0000E9483D849E951E061E070E0CE010D968B
:1062B0000E9483D849E951E061E070E0CE01019687
:1062C0000E9483D8C988DA88EB88FC8827E137EBFD
:1062D00041ED58EBC701B6010F94555F87FD5CC0D7
:1062E00023E030E048EC53E4C701B6010F940356B5
:1062F00018160CF451C0CD84DE84EF84F88827E1B1
:1063000037EB41ED58EBC701B6010F94555F87FDA0
:1063100043C023E030E04DEC53E4C701B6010F94D5
:1063200003561816CCF1CD80DE80EF80F88427E18B
:1063300037EB41ED58EBC701B6010F94555F87FD70
:106340002BC023E030E048EC53E4C701B6010F94C2
:10635000035618160CF1C980DA80EB80FC8027E127
:1063600037EB41ED58EBC701B6010F94555F87FD40
:1063700013C023E030E04DEC53E4C701B6010F94A5
:10638000035618164CF0AE014F5F5F4FBE01635FBE
:106390007F4FC5010E94322F68960FB6F894DEBF7A
:1063A0000FBECDBFDF91CF911F910F91FF90EF9066
:1063B000DF90CF90BF90AF909F907F906F905F9055
:1063C0004F9008958C38910514F08CE890E09093EC
:1063D0001E0980931D090C9482C90E94DF2797FD36
:1063E0000CC00E94DF276F3F71058105910509F000
:1063F00034F40E94DF27862F089580E008958FEF00
:1064000008958091C6049091C704892B41F00E94A1
:10641000ED3191E0811101C090E0892F089591E064
:10642000FCCF0E94DF27CB0108950F931F93CF93DA
:106430008091C6049091C7040097E9F0FC018F0198
:10644000C1912C2F2F7D81F0C53411F0C536B9F7DD
:10645000F801108270E060E00F949251F801C0835F
:10646000CF911F910F91089570E060E0CF911F913F
:106470000F910D94925160E070E0CB01F1CF2FEBC2
:10648000280F2A3108F047C0E22FF0E08091F7048E
:106490009091F804A091F904B091FA0404C0B69563
:1064A000A795979587952A95D2F780FD02C08170B0
:1064B0000895E352FB4FE081EE2341F18091FE0805
:1064C0009091FF08E80FF92FF11D808190ED980F52
:1064D0009A3030F08E3251F4818180538A3098F4B2
:1064E000F093C704E093C60481E008958D3211F063
:1064F0008B3249F4818190ED980F9A3088F38E3277
:1065000011F48281EACFF0E0E0E0EACF1092C70414
:106510001092C604E9CF80E008950E943F3288239C
:1065200041F081E02091C6043091C704232B09F487
:1065300080E00895CF93DF93EB010E948D32882392
:1065400019F00E94DF27EB01CE01DF91CF91089572
:10655000CF92DF92EF92FF926A017B010E948D320F
:10656000882331F0FF90EF90DF90CF900C9415329C
:10657000C701B601FF90EF90DF90CF9008954F9242
:106580005F926F927F928F929F92AF92BF92CF92C3
:10659000DF92EF92FF921F93CF93DF9300D01F9271
:1065A000CDB7DEB719821A821B821C82CE010196FA
:1065B0004C0189E4C82E81E1D82E90EEE92E98E0B6
:1065C000F92E2BEFA22E29E0B22E10E088E5810FE4
:1065D0000E948D32F40181934F01882341F00E9483
:1065E00015322B013C018091FE10882359F0F601F1
:1065F00080819181A281B381F70180839183A283FD
:10660000B38314C0812F0E945222882309F4D0C082
:10661000F6012081318142815381C301B2010F947F
:10662000F55CF70160837183828393831F5FF4E0DD
:10663000CF0ED11C84E0E80EF11C94E0A90EB11C31
:10664000133021F685E40E948D328C83882309F46F
:10665000B9C00E9415326B017C0183E00E94522276
:10666000882371F0209155113091561140915711A6
:1066700050915811C701B6010F94F55C6B017C0174
:10668000C092EC08D092ED08E092EE08F092EF088C
:106690008091D605882359F18091851782FF27C004
:1066A0008C81882321F18981811103C08A8188230B
:1066B000F1F02DEC3CEC4CE45DE3609152097091FB
:1066C000530980915409909155090F94F55C9B01F1
:1066D000AC016091511170915211809153119091C0
:1066E00054110F94555F181614F40F94CD4240E0E6
:1066F00050E0BA0186E40E94A83220E030E0A9010F
:106700000F94555F181684F40E94153220E030E093
:1067100040E752E40F94EF5D60937C0270937D023A
:1067200080937E0290937F028091FF1083FD2CC0A6
:106730008091FE10811128C080915A08882321F190
:106740002091551130915611409157115091581187
:106750006091EC087091ED088091EE089091EF083F
:106760000F94F45C209167083091680840916908A3
:1067700050916A080F94F55C6093670870936808FD
:106780008093690890936A080F900F900F900F9074
:10679000DF91CF911F91FF90EF90DF90CF90BF904E
:1067A000AF909F908F907F906F905F904F900895E3
:1067B000F5012081318142815381C301B2010F94DF
:1067C000F45C2FCF8091551190915611A0915711E3
:1067D000B09158118093EC089093ED08A093EE08C7
:1067E000B093EF0855CFCF93DF93EB010E948D322A
:1067F000882321F0DF91CF910C941132CE01DF91EB
:10680000CF910895CF93DF93C82FD62F0E948D325A
:10681000882321F0DF91CF910C9401328C2F0E94BC
:106820003F32811101C08D2FDF91CF910895E9E4AE
:10683000F9E082EBDF011D928A95E9F708958091D6
:10684000D605811104C00E9417340D94094580912A
:10685000851782FD0D94CD420895809149098823C2
:1068600061F09091FA09891308C08091851783FF20
:1068700004C087E899E00D94144580E00895FC0178
:10688000238121110C94F2D40895CF92DF92EF92DC
:10689000FF920F931F93CF9390912402913009F4AC
:1068A00061C0662351F01092A6041092A2041092C7
:1068B000A3041092A4041092A504C82F0F94CF38FB
:1068C000C090A204D090A304E090A404F090A5048A
:1068D0009B01AC012C193D094E095F0969017A0140
:1068E000F7FC40C02091A604C7FD15C04C2F0C2E0C
:1068F000000C550B4C5F5F4FE22F022E000CFF0B7C
:106900004E175F077CF144EFC42EDD24D394E12CB5
:10691000F12C2C1734F438EEC32E33E0D32EE12CB7
:10692000F12CC60ED71EE81EF91EC092A204D0920A
:10693000A304E092A404F092A504022F017010E0D9
:1069400084E2809FB001819F700D701B11246059FB
:106950007C4F82E390E00E944A808091A6048F5F82
:106960008093A604CF911F910F91FF90EF90DF903D
:10697000CF9008950F931F9301E010E020E030E0E6
:10698000082E04C0000F111F221F331F0A94D2F7D4
:1069900040910B0550910C0560910D0570910E050D
:1069A000402B512B622B732B40930B0550930C05FE
:1069B00060930D0570930E0590912302891303C017
:1069C00081E08093FE101F910F9108951092D706D9
:1069D0001092D8061092D9061092DA06E7EDF5E08B
:1069E00080E091E0DF019C011D9221503040E1F7F1
:1069F0000895909148119817B1F00E9456DF809148
:106A00004811882341F089E491E10E9479DF1092D6
:106A100048110C9466F581E08093481189E491E176
:106A20000E94ABDEF6CF08954F925F926F927F92F5
:106A30008F929F92AF92BF92CF92DF92EF92FF928E
:106A40001F93CF93DF93EC01162F20911309309100
:106A500014094091150950911609688179818A813C
:106A60009B810F940356882309F4AEC0B09048115F
:106A700080E00E94F934C880D980EA80FB8020E061
:106A800030E0A901C701B6010F94555F18161CF03C
:106A9000C12CD12C7601C0921309D0921409E09236
:106AA0001509F09216092DEB37E346E855EBC701BF
:106AB000B6010F94555F87FD0BC02DEB37E346E819
:106AC00055E3C701B6010F94035618160CF078C0B1
:106AD000A701960160E070E080E89FE30F94EF5D0E
:106AE0006093BA057093BB058093BC059093BD0578
:106AF00080EF9FEFA9E7B4EC8093BE059093BF05AC
:106B0000A093C005B093C105BB2009F45DC04090BF
:106B1000491150904A1160904B1170904C11809027
:106B20004D1190904E11A0904F11B0905011C09007
:106B30005111D0905211E0905311F090541181E016
:106B40000E94F934112309F43FC02091491130917A
:106B50004A1140914B1150914C11C301B2010F9455
:106B6000035681111CC020914D1130914E1140915E
:106B70004F1150915011C501B4010F94035681116A
:106B80000EC02091511130915211409153115091EA
:106B90005411C701B6010F9403568823A9F0DF9161
:106BA000CF911F91FF90EF90DF90CF90BF90AF906B
:106BB0009F908F907F906F905F904F900C940EFEFF
:106BC00060E070E0CB018CCFDF91CF911F91FF90FF
:106BD000EF90DF90CF90BF90AF909F908F907F907D
:106BE0006F905F904F900895EF92FF920F931F93D5
:106BF000CF93DF9307ED15E0C8E07801D8E0F70107
:106C000061917191819191917F0120E030E0A90122
:106C10000F94035681110EC0D15089F7C150005E08
:106C20001F4FC111EACFDF91CF911F910F91FF90BC
:106C3000EF90089581E0F7CFEFE6F0E08081826089
:106C4000808308958091F4089091F508892B79F458
:106C50008091F4089091F508892B49F42091F4086B
:106C60003091F50881E0232B19F480E0089581E04C
:106C70000895CF92DF92EF92FF926B017C0183E344
:106C8000C816D104E104F10470F082E3C81AD108F7
:106C9000E108F10862E370E080E090E00F949C3836
:106CA0000E9468F5ECCFC701B6010F949C38FF90A5
:106CB000EF90DF90CF900C9468F58091DA07811106
:106CC0000AC080911109813041F08091851782FBC3
:106CD000882780F9089580E0089581E008955F9AFB
:106CE00080916E088E7F80936E088A9A80916E08DC
:106CF0008D7F80936E0880910801809581708093CC
:106D0000060180916E088B7F80936E080C947F2221
:106D10009091851793FB882780F993FF06C081E047
:106D20009091ED18911101C080E008958091DA07EB
:106D3000811110C080911109823061F00E94883663
:106D4000882349F08091851782FB882780F991E09C
:106D50008927089581E008950E94963681110DC01B
:106D600010920B0510920C0510920D0510920E0555
:106D700010920F058FEF0E9420260D946501E9E324
:106D8000FAE010821182089581E008958F929F9217
:106D9000AF92BF92CF92DF92EF92FF920F93CF9379
:106DA000DF931F92CDB7DEB75C017B0149016B0118
:106DB000C40ED51EF501808191810F94215C8983D9
:106DC000002311F0F7018083BE016F5F7F4FC40184
:106DD0000F94C428F501808191810196918380836D
:106DE000FFEFEF1AFF0AEC14FD0421F780E00F908B
:106DF000DF91CF910F91FF90EF90DF90CF90BF90F8
:106E0000AF909F908F9008959091C00095FFFCCF18
:106E10008093C6000895CF93DF93EC018991882376
:106E200019F00E940437FACF8DE00E9404378AE0FF
:106E3000DF91CF910C940437CF92DF92EF92FF92C3
:106E4000CF936B017C01C42F4A3069F4F7FE0BC06D
:106E5000F094E094D094C094C11CD11CE11CF11CAE
:106E60008DE20E9404374C2FC701B601CF91FF90ED
:106E7000EF90DF90CF900D942F42CF93DF93EC01F2
:106E8000FE0184912196882319F00E940437F8CFDF
:106E9000DF91CF9108950F931F93CF938C01C62F4D
:106EA00085E892E10E943D37C8010E943D378AE3A0
:106EB0000E94043780E38C0F0E9404378AE0CF9150
:106EC0001F910F910C94043788E094E10E943D37A4
:106ED00060E088EF93E10E944B3760E083EE93E13E
:106EE0000E944B3761E08CED93E10E944B3761E0EB
:106EF00081ED93E10E944B3761E081EC93E10E94C8
:106F00004B3760E088EB93E10E944B3761E08EEAFB
:106F100093E10E944B3760E084EA93E10E944B3793
:106F200061E08DE993E10E944B3760E085E993E1F0
:106F30000E944B3761E087E893E10E944B3761E0A4
:106F400089E793E10E944B3760E08AE693E10E9473
:106F50004B3760E08CE593E10E944B3760E086E4BC
:106F600093E10E944B3761E085E393E10E944B3748
:106F700061E086E293E10E944B3761E08FE193E1AB
:106F80000E944B3760E088E193E10E944B3761E05B
:106F90008FE093E10E944B3761E08AEF92E10E941B
:106FA0004B3761E08CEE92E10E944B3761E089ED56
:106FB00092E10E944B3760E08CEC92E10E944B37EB
:106FC00061E087EC92E10E944B3761E08AEB92E14D
:106FD0000E944B3760E086EA92E10E944B3760E006
:106FE00083E992E10E944B3760E089E897E10E94D3
:106FF0004F22682F61708AE892E10C944B378091A0
:10700000F704827149F48091F9048C7829F4809115
:10701000FA04837009F475C082E40E943F32882329
:1070200051F00E94BE27609310117093111180934C
:1070300012119093131183E50E943F32882351F07F
:107040000E94153260934011709341118093421158
:107050009093431184E50E943F32882351F00E94AF
:1070600015326093441170934511809346119093AB
:10707000471188E50E943F32882351F00E94153263
:107080006093210A7093220A8093230A9093240A22
:1070900089E50E943F32882351F00E9415326093A7
:1070A000250A7093260A8093270A9093280A8AE576
:1070B0000E943F328823B1F00E9415326093290A62
:1070C00070932A0A80932B0A90932C0A2DEC3CECA7
:1070D0004CEC5DE30F940356181624F083E69EE013
:1070E0000E943D3785E40E943F32882351F00E9480
:1070F000153260932D0A70932E0A80932F0A909375
:10710000300A08950E94043785E29DE00C943D37D3
:107110000F931F93CF938C01C62F8CE999E00E94A7
:107120003D37C8010E943D37CC2331F08AE0CF9132
:107130001F910F910C940437CF911F910F910895D7
:107140000F931F93CF938C01C62F60E08CEA99E0D8
:107150000E948838C8010E943D37CC2331F08AE074
:10716000CF911F910F910C940437CF911F910F91E4
:10717000089561E084EB99E00C94A038EF92FF92BF
:107180000F931F93CF937C018B01C42F60E08CEA97
:1071900099E00E948838C7010E943D3780E20E9432
:1071A0000437C8010E943D37CC2319F08C2F0E9470
:1071B00004378AE0CF911F910F91FF90EF900C94CC
:1071C0000437DF92EF92FF920F931F93CF93DF93D9
:1071D000D82E7B018A01E9010E94B938D092F808C3
:1071E00040E0B70185EB90E40E94BE38011511051F
:1071F00031F040E0B8018EEA90E40E94BE3820975A
:1072000031F040E0BE018EEA90E40E94BE3861E0B9
:1072100089EA90E4DF91CF911F910F91FF90EF9059
:10722000DF900C94A03861E086EA99E00C948838ED
:10723000AF92BF92CF92DF92EF92FF920F931F9384
:10724000CF93DF9381E799E00E943D376091D706A5
:107250007091D8068091D9069091DA0645E00F9496
:10726000AB0A8EE599E00E943D37C0E0D9E0D150ED
:1072700021F080E20E940437FACF8C2F0F949642BF
:10728000CF5FC83099F78AE00E94043707ED15E018
:10729000C0E080E20E9404378C2F0F949642580180
:1072A000D8E080E20E940437F501C080D180E280FE
:1072B000F380A7019601C701B6010F94E75F811122
:1072C0002CC020E030E0A901C701B6010F94555F42
:1072D00087FD03C08BE20E94043745E0C701B60179
:1072E0000F94AB0AD15080E2A80EB11CD111D9CFB6
:1072F0008AE00E940437CF5F0C5F1F4FC83049F609
:107300008AE0DF91CF911F910F91FF90EF90DF9076
:10731000CF90BF90AF900C940437F12C80E20E9484
:107320000437F3948DE3F8E0FF12F9CFDBCF81113E
:1073300007C085E99EE00E943D378AE00C9404373F
:1073400089E99EE0F8CFCF93DF93EB010E943D37B0
:10735000CE01DF91CF910D949D42CF93C62F0E9415
:107360003D378C2FCF910D949642CF92DF92EF92C2
:10737000FF926A017B010E943D3742E0C701B601DE
:10738000FF90EF90DF90CF900D94AB0ACF92DF92F9
:10739000EF92FF926A017B010E943D374AE0C701EC
:1073A000B601FF90EF90DF90CF900C941C372F9296
:1073B0003F924F925F926F927F928F929F92AF9285
:1073C000BF92CF92DF92EF92FF920F931F93CF93D2
:1073D000DF93CDB7DEB7C654D1090FB6F894DEBF40
:1073E0000FBECDBF70E060E085E40E94F333182F3C
:1073F0008F3F09F483C08823E9F083EC96E1CA5BF0
:10740000DF4F0FB6F894DEBF0FBECDBFDF91CF9137
:107410001F910F91FF90EF90DF90CF90BF90AF90B2
:107420009F908F907F906F905F904F903F902F90A4
:107430000C943D3724EB30E03A83298383E50E94A6
:107440008D32882321F00E9411329A83898365E06E
:1074500070E083E40E94F3338AA760E085E50E9430
:10746000023425968FAF259760E086EB96E10E9467
:1074700092B5A981BA81BD01BB0F880B990B0F94FE
:107480000A566D837E838F8327969FAF27970F942D
:10749000CF38688B798B8A8B9B8B1F3F09F045C453
:1074A00020E030E04CE053E46D817E818F812796AF
:1074B0009FAD27970F94555F18160CF0AAC18BE863
:1074C00096E10E943D37CA5BDF4F0FB6F894DEBFEE
:1074D0000FBECDBFDF91CF911F910F91FF90EF9025
:1074E000DF90CF90BF90AF909F908F907F906F90E4
:1074F0005F904F903F902F900D94044646E450E0EB
:107500005A8349839BCF1FAEAFC12496EEADFFAD2A
:107510002497808383C2FBEE4F2E512C612C712C5B
:1075200004C384E190E0A0E0B0E08C8B9D8BAE8B37
:10753000BF8BE4E14E2E512C612C712C04C34C8A7C
:107540005D8A6E8A7F8AFFC22496EEADFFAD2497D6
:107550008083D4C389819A81AB81BC8129A93AA94E
:107560004BA95CA9821B930BA40BB50BB7FD59C0AB
:107570008FAD0F944F0B8AE00E94043789819A8166
:10758000AB81BC818053984FAF4FBF4F89AB9AAB53
:10759000ABABBCAB9DA9911177C02EA93FA948AD5B
:1075A00059ADB101802F26969FAD26970F94555F58
:1075B00018160CF053C020E030E040E050E4B10178
:1075C000802F26969FAD26970F94F55C6EAB7FAB10
:1075D00088AF99AF2CA53DA54EA55FA589819A815D
:1075E000AB81BC81280F391F4A1F5B1F2AAF3BAFFD
:1075F0004CAF5DAF20E030E040EC50E46D817E8127
:107600008F8127969FAD27970F94F45C9101402FAF
:1076100026965FAD26970F940356881F8827881FEC
:107620008DAB88899989AA89BB89C816D906EA06CB
:10763000FB0610F4D701C60129813A814B815C8198
:10764000281B390B4A0B5B0BDA01C90181389F44B7
:10765000A241B105A8F187ED95E10EC289819A8119
:10766000AB81BC812AAD3BAD4CAD5DAD821B930BB4
:10767000A40BB50B41E656E360E776E3B7FDD1CF47
:10768000812F0E94C5D8CDCF20E030E040EF51E4FB
:107690006D817E818F8127969FAD27970F94F45C33
:1076A0009B01AC01B101802F26969FAD26970F94C8
:1076B000035687FFB6CF4DE057E36DE177E3E0CFA8
:1076C0004AA55BA5888D998D481759070CF09EC077
:1076D00003970CF49BC08AE795E10E943D371F3F5A
:1076E00009F076C0AAE6B5E1BA83A98389E595E1F8
:1076F0000E943D3789819A810E943D37488559858E
:107700006A857B8586E795E10E94B5398AE00E940B
:10771000043789E595E10E943D3789819A810E946D
:107720003D3749A15AA16BA17CA182E795E10E9456
:10773000B5398AE00E94043789E595E10E943D371A
:1077400089819A810E943D37B501A4018EE695E1B9
:107750000E94B5398AE00E9404372596FFAD25972F
:10776000FF2391F12CEA35EC47E25EE369A17AA1AF
:107770008BA19CA10F9469566B017C012CEA35EC1E
:1077800047E25EE3C501B4010F94EF5D28853985BA
:107790004A855B851F3F09F5209320093093210915
:1077A0004093220950932309C0922409D0922509BD
:1077B000E0922609F092270960932809709329091D
:1077C00080932A0990932B0981E0809365027BCEF8
:1077D000E3EFFFE3FA83E98389CF209384163093A4
:1077E00085164093861650938716C0928816D092BD
:1077F0008916E0928A16F0928B1660938C1670931D
:107800008D1680938E1690938F16DECF0E949EB9B0
:1078100080C087E796E10E943D370E94B8D78FE786
:1078200080931F0924EB30E0A8EEB3E00F949B5C3B
:107830006CA77DA78EA79FA7288939894A895B896C
:10784000260F371F481F591F2AAF3BAF4CAF5DAF04
:107850001092650281E08093740232E0310F3EAFF6
:10786000323008F450CE1FAFC888D988EA88FB8828
:10787000C9AADAAAEBAAFCAA812C912C540189A2EC
:107880009AA2ABA2BCA288869986AA86BB868FE7FD
:1078900090E0A0E0B0E08C8B9D8BAE8BBF8B1C8604
:1078A00090E49A8FACE1AB8FB6E4BC8F1D8E1E8E38
:1078B0001F8E18A23FE7432E512C612C712C1DAA5C
:1078C0008EAA9FAAA8AEB9AE1EA21FA218A619A67C
:1078D000E1E0EDA3198E188E212C312C00E02696C4
:1078E0001FAE2697F5E11F02C00111249C01255807
:1078F000394E22963FAF2EAF2297285F3F4F2496F6
:107900003FAF2EAF24974AA5042E000C550B5BA762
:107910004AA780917402882309F4B0C00F94CF382D
:1079200069837A838B839C835091F40658AB5523EB
:1079300009F48BC00E946BD860911B0970911C09DF
:107940001F3F39F02296AEADBFAD229714966D91D0
:107950007C91072E000C880B990B0F940A561B0183
:10796000082F26969FAF26972D8D3E8D4F8D58A1BF
:1079700026969FAD26970F94555F18163CF42D8ED2
:107980003E8E0F8F2696BFAD2697B8A32C853A8DD5
:107990004B8D5C8DB101802F26969FAD26970F945D
:1079A000035687FF07C02C863A8E0B8F2696EFADC5
:1079B0002697EC8FFDA19101402F26965FAD26976B
:1079C0006D817E818F8127969FAD2797FF2309F4D4
:1079D0005AC00F94035687FF38C049815A816B8182
:1079E0007C814C195D096E097F09DB01CA01885849
:1079F0009341A109B109B7FD28C08C899D89AE8941
:107A0000BF8984199509A609B709B595A7959795D2
:107A100087951F3F09F079CD80931F094EA35FA37F
:107A200068A779A7FD81FD8F2E812E8F3F813F8F23
:107A300027964FAD279748A389819A81AB81BC8156
:107A4000888B998BAA8BBB8B1DA220E030E040EF86
:107A500051E46D817E818F8127969FAD27970F948A
:107A6000F55C9101402F26965FAD26970F94035643
:107A700087FF70CD85EF95E10E943D37109274022B
:107A80000E94B8D7A1CE0F94555F1816F4F68981DD
:107A90009A81AB81BC81288939894A895B89821B9B
:107AA000930BA40BB50BAC01BD01485853416109C0
:107AB000710977FDCACF488D598D452B09F40DC149
:107AC000CEA0DFA0E8A4F9A4C80ED91EEA1EFB1EB2
:107AD0002EA13FA148A559A5281B390B4A0B5B0BCA
:107AE000C301B2010F94375CA70196010F94695C42
:107AF0004C885D886E887F88420E531E641E751EFA
:107B000054E145165104610471040CF40ACD8CEE65
:107B100048165104610471040CF0FDCC90E849163C
:107B20005104610471040CF40ACD4C8A5D8A6E8A9A
:107B30007F8A2EEF30E040E050E0241935094609F5
:107B4000570929013A014C895D896E897F898FE641
:107B500096E10E94C639B301A2018AE696E10E942D
:107B6000C6394C855A8D6B8D7C8D83E696E10E94DB
:107B7000B5394D8D5E8D6F8D78A18CE596E10E94B3
:107B8000B539A88DB98D13970CF4A7C0C301B20104
:107B90000F940A5620E030E040E850E40F94695614
:107BA0004B015C012C853A8D4B8D5C8D6D8D7E8DEE
:107BB0008F8D98A10F94F45C2BED3FE049E450E4E5
:107BC0000F94695620E030E040E05FE30F9469567F
:107BD0009B01AC01C501B4010F94EF5D6C877D87FB
:107BE0008E879F87C701B6010F940A562FE632E1B0
:107BF00043E85AE30F9469566B017C011E3F59F02C
:107C00002AE939E949E15FE3812C912CA12C6EE34B
:107C1000B62E1F3F59F42DEC3CEC4CE45EE37BEABE
:107C2000872E7AEA972EA92C7EE3B72E6C857D8568
:107C30008E859F850F946956688779878A879B8789
:107C40009B01AC010F94F55CA70196010F94EF5DC9
:107C500069A37AA38BA39CA3288539854A855B8574
:107C6000C701B6010F946956A50194010F94695696
:107C70004B015C014C855D856E857F8586E596E1CF
:107C80000E94B539B701A60180E596E10E94B53999
:107C90008AE00E940437BEAD81E496E1B23010F074
:107CA00082E396E10E943D37488559856A857B8548
:107CB0008CE296E10E94B53949A15AA16BA17CA141
:107CC00086E296E10E94B539B501A40180E296E111
:107CD0000E94B5398AE00E9404378C899D89AE895B
:107CE000BF89840D951DA61DB71DB595A7959795C0
:107CF00087951F3F09F028CC80931F09288D398D67
:107D00002F5F3F4F398F288F3D813C874E814A8FAF
:107D10005F815B8F27968FAD27978C8FC980DA8024
:107D2000EB80FC8098A99DA390CEE12E012E000C43
:107D3000FF08F70183E0EE0FFF1F8A95E1F7E45992
:107D4000FD4F668177816F507109072E000C880BFB
:107D5000990B0F940A569B01AC016D817E818F8136
:107D600027969FAD27970F94555F18160CF4A7CB55
:107D700087E796E10E943D370E94B8D785E18E9D46
:107D8000F0018F9DF00D1124E558F94E8FE78087A3
:107D900022E330E049CDCF93DF93EB010E943D37E2
:107DA000CE01DF91CF910D947B2A2F923F924F927B
:107DB0005F926F927F928F929F92AF92BF92CF927B
:107DC000DF92EF92FF920F931F93CF93DF93CDB784
:107DD000DEB7C058D1090FB6F894DEBF0FBECDBFD5
:107DE00080EB9CE00E943D370F94264681118FC0A6
:107DF00084E50E948D32882329F00E94113281117E
:107E00000E946ED780E090E0A0E8BFE389839A8368
:107E1000AB83BC838D839E83AF83B8878DEC9CEC52
:107E2000ACE4BEE389879A87AB87BC8780E090E0AB
:107E3000A0E2B1E48D879E87AF87B88B8CE390E09A
:107E40009A8B898B8DEC90E09C8B8B8B8DEC9CECD2
:107E5000ACECBEE38D8B9E8BAF8BB88F80E090E057
:107E6000A0EEBFE3898F9A8FAB8FBC8F1BA61CA699
:107E70004AE959E969E97EE38FE40E94A8326D8FEF
:107E80007E8F8F8F98A360E083E40E94023489A3E1
:107E900060E08BE40E9402348AA389E40E948D3260
:107EA00010E0F12CE12C8823C1F00E94ED3190E02C
:107EB0001816190614F481E090E011E0180F212F34
:107EC0002150330BC90126E0289FF001299FF00DB6
:107ED0001124EC54F74FE280F38082E40E948D324B
:107EE000882319F00E9411327C01E114F10459F148
:107EF000C70188978536910520F16CE870E082E82B
:107F00009CE00E94CB3E8DE79CE00E943D37C0582C
:107F1000DF4F0FB6F894DEBF0FBECDBFDF91CF911C
:107F20001F910F91FF90EF90DF90CF90BF90AF9097
:107F30009F908F907F906F905F904F903F902F9089
:107F40000895FA8AE98A8CE40E948D328823E1F050
:107F50000E9415326B017C01C986DA86EB86FC86AD
:107F600020E030E0A9010F94555F87FD0AC020E0B2
:107F700030E040E050E4C701B6010F9403561816F4
:107F80001CF485E59CE0C1CF81E50E943F32882347
:107F900031F18091C6049091C704892BE9F00E94C9
:107FA00015326B017C01CD82DE82EF82F8862DECEA
:107FB0003CEC4CE45DE30F94555F87FD0AC020E084
:107FC00030E040E751E4C701B6010F94035618169C
:107FD00034F484E29CE099CF89EF9BE096CF83E56F
:107FE0000E948D328823E9F00E9415326B017C01DA
:107FF000CD8ADE8AEF8AF88E2DEC3CEC4CEC5DE30A
:108000000F94555F87FD0AC020E030E040E050E467
:10801000C701B6010F94035618161CF482ED9BE0BD
:1080200074CF80E50E943F32882341F08091C604DE
:108030009091C704892B29F58FEF8BA786E40E94C6
:108040008D32882309F43DC00E9415326B017C01FA
:10805000C98EDA8EEB8EFC8E20E030E040E85FE3E4
:108060000F94555F87FD0AC020E030E040E850E4FF
:10807000C701B6010F94035618161CF581E89BE062
:1080800044CF8BA58F5F8BA70E9415326B017C01BB
:10809000CD86DE86EF86F88A20E030E0A9010F94D5
:1080A000555F87FD0BC020E030E048EC51E4C7018C
:1080B000B6010F94035618160CF0C0CF8AEA9BE065
:1080C00024CFC98CDA8CEB8CFC8C8D889E88AF8891
:1080D000B88CA7019601C701B6010F9469569B01A0
:1080E000AC0160E070E084E490E40F94EF5D2981DE
:1080F0003A814B815C810F9469562B013C01A501AB
:108100009401C501B4010F946956A70196010F941B
:1081100069562CEE31E548EB5DE30F94EF5D9B0172
:10812000AC01C301B2010F94695669837A838B83D2
:108130009C83112309F1412F4150550B26E0249FC8
:10814000F001259FF00D1124EC54F74F00811181AF
:1081500088E40E948D32882319F00E9411328C012C
:108160000115110571F0C801855A910988389105EA
:1081700030F083E59BE0C9CE10E000E0E9CF1C8B36
:108180000B8B85E50E943F328823C9F00F94CF38CE
:10819000611571058105910511F00F948951809148
:1081A000C6049091C704892BC9F00E9415326093D0
:1081B000C2047093C3048093C4049093C50461E423
:1081C00070E082E50E94F333E5969FAF8EAFE597AE
:1081D0001816190644F08FE19BE097CE60E070E03E
:1081E00088E492E4E4CF89E50E948D32882309F483
:1081F0000AC10E9415322091FF093091000A409176
:10820000010A5091020A0F94F45C4B015C0188E56D
:108210000E948D32882309F4FFC00E9415322091FC
:10822000FB093091FC094091FD095091FE090F9422
:10823000F45C6B017C01CBA2DCA2EDA2FEA28FA2BA
:1082400098A6A9A6BAA627E137EB41ED58EBC501E0
:10825000B4010F94555F87FDE8C023E030E048EC9F
:1082600053E4C501B4010F94035618160CF4DDC095
:1082700027E137EB41ED58EBC701B6010F94555F8D
:1082800087FDD3C023E030E04DEC53E4C701B601D5
:108290000F94035618160CF4C8C084E40E943F32B1
:1082A00011E081270E94F93480E090E0A0EAB0E478
:1082B0008DA79EA7AFA7B8ABCE018D960F94743152
:1082C00050913009EC965FAFEC97109230090E9404
:1082D00005C782EA9AE00E943D3789899A894A97C0
:1082E0000CF0A6C063E68FE79AE00E9492B50F9467
:1082F00008398B899C890E94D8DE41E061E080E0EA
:108300000F94470D882309F4A6C00F9404460F94D8
:10831000083910925511109256111092571110925F
:10832000581185E591E10E945EF11BA5112309F426
:10833000F5C020E030E040E751E4609130117091E9
:10834000311180913211909133110F94EF5D21968C
:108350006CAF7DAF8EAF9FAF21971F3F09F0F9C47F
:1083600081E08093080563E687ED9AE00E9492B56C
:1083700068E873E182E090E00E944A8080E1E9E4ED
:10838000F1E1A0EEB8E001900D928A95E1F7CE01FF
:1083900001960F94CF31C12CD12C760180910B0A1C
:1083A00082FDB1C068E873E182E090E00E944A80FB
:1083B00020E030E040E85EE36091EC087091ED0869
:1083C0008091EE089091EF080F94F55C6093EC08B3
:1083D0007093ED088093EE089093EF0820E030E072
:1083E00040E85EE3C701B6010F94F55C6B017C01C8
:1083F00020E030E84BE354E40F94555F87FD73C0F1
:108400001092080528C080904D1190904E11A090B8
:108410004F11B0905011FBCEC0904911D0904A112D
:10842000E0904B11F0904C1106CF85EF9AE06DCDA6
:1084300063E682E99AE00E9492B50F94083910939E
:10844000080589899A890E94E23161E081E00F94F0
:10845000C20B811147CF6FEF89EE9AE00E9492B56F
:108460008CA5811112C081E08CA78D819E81AF8186
:10847000B885B0588DA79EA7AFA7B8ABBE01635D06
:108480007F4F80EE98E00E94BC2E80E090E0A0EA52
:10849000B0E48093E8089093E908A093EA08B093C9
:1084A000EB081DA61EA61FA618AABE01635D7F4F7E
:1084B00080EE98E00E94BC2EEC965FADEC97509356
:1084C00030090E9405C7109208058AA181111FCDAD
:1084D00010921E0910921D090E9482C990E080E04E
:1084E0000E94D8DE14CDCE01CD960E9456FC80E1CC
:1084F000E9E4F1E1A0EEB8E001900D928A95E1F790
:108500000E9456DF4BCF0E945DBC63E68AEC9AE086
:108510000E9492B50F94083910920805EAEBF4E036
:1085200088E0DF011D928A95E9F780E1E9E4F1E155
:10853000A0EEB8E001900D928A95E1F789859A85C1
:10854000AB85BC858093E8089093E908A093EA087E
:10855000B093EB081DA61EA61FA618AABE01635D58
:108560007F4F80EE98E00E94BC2EBE01635E7F4F7D
:1085700080EE98E00E94BC2E81E08093080589A1DE
:10858000882309F43CC42091491130914A1140914B
:108590004B1150914C11AC962CAF3DAF4EAF5FAF2D
:1085A000AC9780914D1190914E11A0914F11B091C7
:1085B0005011E0968CAF9DAFAEAFBFAFE097AAE58C
:1085C000B7E1A196BFAFAEAFA197312C212CBFEF81
:1085D0006C96BFAF6C97EFEFA496EFAFA497FFEF49
:1085E000E396FFAFE3972FE4EA962FAFEA9733ECD9
:1085F000EB963FAFEB9707E481E090E0A0E0B0E0BE
:10860000022C04C0880F991FAA1FBB1F0A94D2F71F
:10861000C458DF4F88839983AA83BB83CC57D0404B
:10862000AAEBB4E0E296BFAFAEAFE297EAE3F7E1C0
:10863000A396FFAFEEAFA39710E0C058DF4F28829C
:10864000C058D040E296AEADBFADE2978D91E296B4
:10865000BFAFAEAFE29790E0B0E0A0E0C458DF4F0C
:10866000288139814A815B81CC57D0408223932372
:10867000A423B523892B8A2B8B2B09F0E5C0A19667
:10868000AEADBFADA197CD90DD90ED90FC90A396DF
:10869000AEADBFADA3972D913D914D915C91A89644
:1086A0002CAF3DAF4EAF5FAFA897A7019601AC9638
:1086B0006CAD7DAD8EAD9FADAC970F94F45C2B018E
:1086C0003C01A8962CAD3DAD4EAD5FADA897E096B0
:1086D0006CAD7DAD8EAD9FADE0970F94F45C4B011A
:1086E0005C01A3019201C301B2010F9469562B01F1
:1086F0003C01A5019401C501B4010F9469569B0189
:10870000AC01C301B2010F94F55C0F94A35F4B0160
:108710005C01A70196016BA17CA18DA19EA10F9484
:10872000F45C6B017C01A8962CAD3DAD4EAD5FAD08
:10873000A8976FA178A589A59AA50F94F45C2B0141
:108740003C01A7019601C701B6010F9469566B0160
:108750007C01A3019201C301B2010F9469569B01F0
:10876000AC01C701B6010F94F55C0F94A35F20E044
:1087700030E040E751E40F94EF5DA50194010F94C0
:10878000F55C6B017C018090C2049090C304A090C2
:10879000C404B090C50420E030E040E85FE3C501C8
:1087A000B4010F94555F1816F4F4C501B4010F9489
:1087B000615E4B015C0160E070E0CB0118141904AC
:1087C0001A041B0434F40F943A51A50194010F9438
:1087D000695C0F940A569B01AC01B601C7010F9466
:1087E000F55C6B017C01E3962FADE397EA963FAD14
:1087F000EA97EB964FADEB97502FB601C7010F9458
:10880000035687FF21C06C961FAF6C97C058DF4F8F
:10881000B881C058D040A496BFAFA497E696CFAE1B
:10882000E697E796DFAEE797E896EFAEE897E9962A
:10883000FFAEE997E396CFAEE397EA96DFAEEA970D
:10884000EB96EFAEEB970F2D1F5FA396EEADFFAD4E
:10885000A3973496A396FFAFEEAFA397183009F015
:10886000F1CEFFEF2F1A3F0AA1962EAD3FADA19793
:108870002C5F3F4FA1963FAF2EAFA19738E0231654
:10888000310409F0B9CE6C964FAD6C97E42FF0E04F
:10889000E654FB4F208181E090E0A0E0B0E0A49698
:1088A0000FACA49704C0880F991FAA1FBB1F0A947E
:1088B000D2F7822B8083A4965FADA49762965FAFB8
:1088C000629763964FAF6397E6968FADE697E7960C
:1088D0009FADE797E896AFADE897E996BFADE9970A
:1088E00067968CAF9DAFAEAFBFAF67975F3F09F4A0
:1088F00014C24F3F09F411C284E04802F001112470
:10890000E65CF84E108101813280238027E137EB4D
:1089100041ED58EB612F702F832D922D0F94555FF1
:1089200087FDFFC123E030E048EC53E4612F702F56
:10893000832D922D0F94035618160CF4F2C1A496B1
:108940009FADA497A4E09A02F0011124E65AF84ED4
:10895000C080D180E280F38027E137EB41ED58EB16
:10896000B601C7010F94555F87FDDBC123E030E0FE
:108970004DEC53E4B601C7010F94035618160CF4DE
:10898000D0C120E030E040EA50E4B601C7010F94C6
:10899000F55CA0966FAFA097A2967FAFA297A59621
:1089A0008FAFA597A9969FAFA997CB01A596AFAD1D
:1089B000A597A996BFADA99721968CAF9DAFAEAFF5
:1089C000BFAF2197812F902FA32DB22D25968CAF6D
:1089D0009DAFAEAFBFAF2597A496BFADA497B11121
:1089E00050C26C96EFAD6C97E11118C220E030E0F8
:1089F00040EA50E4612F702F832D922D0F94F55C87
:108A0000A4966FAFA497AD967FAFAD97E1968FAF69
:108A1000E197E3969FAFE3976C96FFAD6C97FF23CA
:108A200009F4F1C26C963FAD6C97A096CFAEA097BB
:108A3000A296DFAEA297A596EFAEA597A996FFAE38
:108A4000A99737300CF014C222ED822E23E5922E26
:108A50002BE7A22E21E4B22E21964CAC5DAC6EAC7D
:108A60007FAC219725962CAD3DAD4EAD5FAD2597E2
:108A70006F962CAF3DAF4EAF5FAF6F97A3019201E2
:108A8000B601C7010F94F45C2D966CAF7DAF8EAF2D
:108A90009FAF2D976F962CAD3DAD4EAD5FAD6F97EF
:108AA000612F702F832D922D0F94F45C61966CAF23
:108AB0007DAF8EAF9FAF6197A30192016091491185
:108AC00070914A1180914B1190914C110F94F45C6C
:108AD0002B013C016F962CAD3DAD4EAD5FAD6F9758
:108AE00060914D1170914E1180914F1190915011E4
:108AF0000F94F45C6F966CAF7DAF8EAF9FAF6F97A6
:108B0000A0968FADA097A2969FADA297A596AFAD68
:108B1000A597A996BFADA9978DA79EA7AFA7B8ABFC
:108B2000A4968FADA497AD969FADAD97E196AFADEE
:108B3000E197E396BFADE39789AB9AABABABBCAB28
:108B4000C984DA84EB84FC84CDAADEAAEFAAF8AE4D
:108B50002DEC3CEC4CEC5CE3C501B4010F94695680
:108B600029813A814B815C810F946956209155117E
:108B70003091561140915711509158110F94F55C56
:108B800069AF7AAF8BAF9CAFA3019201C301B20171
:108B90000F9469562B013C016F962CAD3DAD4EAD47
:108BA0005FAD6F97CA01B9010F9469569B01AC0183
:108BB000C301B2010F94F55C20E030E040E050E4E6
:108BC0000F94555F1816ACF420E030E040E05FE30E
:108BD000C701B6010F94F55C29966CAF7DAF8EAFDF
:108BE0009FAF2997BE01635C7F4FCE0101960E9423
:108BF000C52E89859A85AB85BC8529968CAF9DAF9E
:108C0000AEAFBFAF29976B961CAE1DAE1EAE1FAEAA
:108C10006B97BE01695A7F4FCE01CD960E94BC2E44
:108C2000CE0101960F94CF31A0902811B090291158
:108C3000C0902A11D0902B11E0902411F0902511B2
:108C400000912611109127119701A801B501C601C5
:108C50000F94555F181614F07501860180907C0200
:108C600090907D02A0907E02B0907F022DEC3CECB3
:108C70004CEC5DE3B701C8010F94695660937C0228
:108C800070937D0280937E0290937F0240E0BE014C
:108C9000675B7F4FCE018D960F94C93980E1E9E47F
:108CA000F1E1A0EEB8E001900D928A95E1F7809293
:108CB0007C0290927D02A0927E02B0927F020E947E
:108CC000CE278111C8CB20E04FEFBE016F5A7F4FF6
:108CD000CE0101960E94883020E041E0BE016F5A2B
:108CE0007F4FCE0101960E9488302FEF40E0BE01F9
:108CF0006F5A7F4FCE0101960E94883021E040E0FC
:108D0000BE016F5A7F4FCE0101960E9488300E94AB
:108D100056DF0E94CE2781119ECB809159118093FE
:108D20005A11E5964EAD5FADE59741505109E59674
:108D30005FAF4EAFE597452B09F48DCB62968FADB3
:108D4000629787FD88CB63968FAD639787FF17CCBB
:108D500082CB63E687EB9AE00E9492B50F940839C4
:108D600080E1E9E4F1E1A0EEB8E001900D928A958E
:108D7000E1F72D853E854F8558896091EC0870910B
:108D8000ED088091EE089091EF080F94F55C6093E8
:108D9000EC087093ED088093EE089093EF08CE01F5
:108DA000CD960E9456FC2D853E854F855889609151
:108DB000EC087091ED088091EE089091EF080F9407
:108DC000F45C6093EC087093ED088093EE08909348
:108DD000EF088CA58111A2CB81E08CA78D819E81AB
:108DE000AF81B885B0588DA79EA7AFA7B8ABBE011D
:108DF000635D7F4F80EE98E00E94BC2E8FCB2BA14D
:108E00003CA14DA15EA1AC962CAF3DAF4EAF5FAF84
:108E1000AC978FA198A5A9A5BAA5CBCBC601D701C0
:108E200021968CAF9DAFAEAFBFAF219720E030E071
:108E300040EA50E4612F702F832D922D0F94F45C43
:108E400025966CAF7DAF8EAF9FAF25976C962FADFB
:108E50006C9727300CF4CACDA4961FAFA497AD969B
:108E60000FAFAD97E1963FAEE197E3962FAEE39754
:108E700092ED892E93E5992E9BEFA92E90E4B92EC1
:108E8000EBCDA4964FADA49747300CF46EC06C9612
:108E90005FAD6C975730BCF120E030E040EA50E421
:108EA000B601C7010F94F45C21966CAF7DAF8EAF15
:108EB0009FAF219720E030E040EA50E4612F702F0F
:108EC000832D922D0F94F45CA4966FAFA497AD966A
:108ED0007FAFAD97E1968FAFE197E3969FAFE397B2
:108EE0006C969FAD6C97A096CFAEA097A296DFAE82
:108EF000A297A596EFAEA597A996FFAEA997973032
:108F00000CF0B6CFA1CDC601D70121968CAF9DAF95
:108F1000AEAFBFAF219720E030E040EA50E4612FD0
:108F2000702F832D922D0F94F55C25966CAF7DAF3D
:108F30008EAF9FAF25976C968FAD6C978111BACF8E
:108F400020E030E040EA50E4B601C7010F94F45C41
:108F5000A0966FAFA097A2967FAFA297A5968FAF6E
:108F6000A597A9969FAFA99777CF6C96AFAD6C9751
:108F7000A1112BC020E030E040E251E4A0966FAD9B
:108F8000A097A2967FADA297A5968FADA597A9961B
:108F90009FADA9970F94F45CA0966FAFA097A2968F
:108FA0007FAFA297A5968FAFA597A9969FAFA997D8
:108FB000A4961FAFA497AD960FAFAD97E1963FAEC5
:108FC000E197E3962FAEE3973FCD6C96BFAD6C97DC
:108FD000B73034F120E030E040E251E4A0966FADCC
:108FE000A097A2967FADA297A5968FADA597A996BB
:108FF0009FADA9970F94F45C21966CAF7DAF8EAFB7
:109000009FAF2197D5CFA096CFAEA097A296DFAE07
:10901000A297A596EFAEA597A996FFAEA99728CFE0
:10902000A4961FAFA497AD960FAFAD97E1963FAE54
:10903000E197E3962FAEE39782ED882E83E5982E95
:109040008BEFA82E81E4B82E07CD87E599E00C942C
:109050003D37CF92DF92EF92FF920F931F93CF9302
:10906000DF9388E50E943F32D82E89E40E943F3288
:10907000C82E8823D1F10E941132D82F89E50E9491
:109080003F32182F8AE40E943F32082F882309F4C8
:1090900055C00E941132C82F8AE50E943F32E82E47
:1090A000F12C811104C081E50E943F32F82EC110DD
:1090B00001C000E0802F90E0D11001C010E0810FCE
:1090C000911D019721F4E11062C0F11060C00E946F
:1090D000254883E49EE0DF91CF911F910F91FF908F
:1090E000EF90DF90CF900C943D37D11002C0DFEFAE
:1090F000C5CF0E9415322091FB093091FC094091A7
:10910000FD095091FE090F94F45C20E030E040EA44
:1091100051E40F94F45C2BED36EB4DEC51E40F94DD
:10912000F55C25EF39E44FE95CE30F9469560F9441
:10913000615ED62F683008F4A1CFD9CF111102C0DB
:10914000CFEFAACF0E9415322091FF093091000A7B
:109150004091010A5091020A0F94F45C20E030E043
:1091600040EA51E40F94F45C2BED36EB4DEC51E406
:109170000F94F55C25EF39E44FE95CE30F946956F1
:109180000F94615EC62F683008F486CFD9CFD7FD23
:1091900002C0C7FF05C00E9425488AE29EE09BCF1F
:1091A0000E9415329B01AC01AC2FCC0FBB0B88E0A9
:1091B000D802E001112460E070E0CB01FF2069F0EB
:1091C000FE01EA0FFB1FEE0FFF1FEE0FFF1FE9521C
:1091D000FA4F6081718182819381CA0FDB1FCC0FAE
:1091E000DD1FCC0FDD1FC952DA4F0F94F55C688389
:1091F00079838A839B83DF91CF911F910F91FF9099
:10920000EF90DF90CF90089581E599E00C943D3781
:10921000CF9384E50E948D32C0E08823D9F00E946C
:10922000ED31C82F1816B4F40E9404498DE40E9451
:1092300004378091FC049091FD040F949D426C2FA3
:10924000CC0F770B8DE59FE00E94CB3E8AE00E9419
:109250000437CFEF8C2FCF9108954F925F926F928A
:109260007F928F929F92AF92BF92CF92DF92EF92B6
:10927000FF92CF93DF93CDB7DEB72C970FB6F8945C
:10928000DEBF0FBECDBF4090FB095090FC0960903F
:10929000FD097090FE092091390230913A02409107
:1092A0003B0250913C02C301B2010F94F55C69830B
:1092B0007A838B839C838090FF099090000AA09012
:1092C000010AB090020A20913D0230913E02409185
:1092D0003F0250914002C501B4010F94F55C6D83CB
:1092E0007E838F839887C090030AD090040AE09011
:1092F000050AF090060A2091410230914202409105
:10930000430250914402C701B6010F94F55C69878E
:109310007A878B879C872091450230914602409145
:10932000470250914802C301B2010F94F55C2B0132
:109330003C012091490230914A0240914B025091E8
:109340004C02C501B4010F94F55C4B015C01209106
:109350004D0230914E0240914F0250915002C70190
:10936000B6010F94F55C6B017C010E9404498EEA02
:109370009EE00E943D3783E50E943F32882321F022
:109380000E9401328093370280913702811151C0CF
:1093900085E99EE00E943D3786EA9EE00E943D37C7
:1093A00049815A816B817C8183E39CE20E94B539BB
:1093B0004D815E816F81788581E691E40E94B539A7
:1093C00049855A856B857C858EE591E40E94B53987
:1093D00084EA9EE00E943D378CE99EE00E943D3782
:1093E000B301A20183E39CE20E94B539B501A40157
:1093F00081E691E40E94B539B701A6018EE591E4BA
:109400000E94B5398AE02C960FB6F894DEBF0FBEE5
:10941000CDBFDF91CF91FF90EF90DF90CF90BF90C5
:10942000AF909F908F907F906F905F904F900C9433
:10943000043789E99EE0AECF2F923F924F925F9220
:109440006F927F928F929F92AF92BF92CF92DF9254
:10945000EF92FF920F931F93CF93DF93CDB7DEB7B9
:109460006A970FB6F894DEBF0FBECDBF83E50E94AA
:109470003F32182F30904811882319F00E94013292
:10948000382E4090491150904A1160904B117090C5
:109490004C1180914D1190914E11A0914F11B091AE
:1094A00050118B8B9C8BAD8BBE8B80915111909109
:1094B0005211A0915311B09154118F8B988FA98F95
:1094C000BA8F112329F0311003C080E00E94F934D3
:1094D00086E50E943F32888B0E94F435882309F488
:1094E000BFC083E40E943F32882309F498C00E94E1
:1094F00015326B017C01A7EDB5E0BF83AE83B98760
:10950000A887F8E0FD831D861E8628EC2F8702ECD5
:109510001A86212C88EC8B8792E49C87A885B985D4
:10952000BA8BA98B18E0E989FA8981909190A19072
:10953000B190FA8BE98B2A85322D4B855C85C5016C
:10954000B4010F94035687FF04C08A86292CAB868A
:10955000BC862D853E854F85502FC501B4010F94E3
:10956000555F181624F48D869E86AF860B2D1150FC
:10957000D1F6FD81F150FD83888599858096998784
:109580008887F111CBCF2D853E854F85502F6A8579
:10959000722D8B859C850F94F55C20E030E040E0D7
:1095A0005FE30F946956A70196010F94F55C6B0178
:1095B0007C012DEB37E346E855EB0F94555F87FDB3
:1095C0000AC02DEB37E346E855E3C701B6010F9417
:1095D0000356181624F580E00E94F93418E0AE8096
:1095E000BF8008E0D5016D917D918D919D915D01C8
:1095F0004D01B4E08B1A9108A70196010F94F45C19
:10960000F4016083718382839383015059F7115071
:109610008E819F8180969F838E831111E0CFA889D0
:10962000AA2351F00E94F435882331F080E09DE0B8
:109630000E943D370E9418398AE50E943F328823F4
:1096400059F00E94153269837A838B839C8360E092
:10965000CE0101960E941435832D0E94F9340BC06F
:10966000311003C09889992339F30E94044986E197
:109670009DE00E943D37332051F0809148118111C7
:1096800006C00E94254881EE9CE00E943D370E9462
:10969000044983ED9CE00E943D37809148110E946F
:1096A00097390E94044986EC9CE00E943D37C090A7
:1096B0001309D0901409E0901509F090160920E0E4
:1096C00030E0A901C701B6010F94555F18160CF0E0
:1096D00053C042E0C701B6010F94AB0A8DE00E946F
:1096E00004378AE00E940437A30192016091491176
:1096F00070914A1180914B1190914C110F94035627
:1097000081111FC02B893C894D895E8960914D1163
:1097100070914E1180914F11909150110F940356FA
:1097200081110FC02F89388D498D5A8D609151114B
:109730007091521180915311909154110F940356CE
:1097400081110E940EFE6A960FB6F894DEBF0FBE1E
:10975000CDBFDF91CF911F910F91FF90EF90DF90E0
:10976000CF90BF90AF909F908F907F906F905F90C1
:109770004F903F902F90089581EC9CE00E943D37E0
:10978000B3CFCF93C82F82E0C11184E040E060E006
:109790000E949F870E94044989EC99E0CC2311F034
:1097A0008EED99E0CF910C943D37FF920F931F936C
:1097B000CF93DF93EC018B01F42E0E94B8D70E9467
:1097C000254881E399E00E943D370115110511F408
:1097D00003EF1FE3209711F4C8E2D9E00E944EBCCA
:1097E0001F930F93DF93CF9388E199E09F938F931B
:1097F00081E08F930E9477B50E94B686C0910017D2
:10980000C695C6958BEF96E10E94C129DC2FDD0F2E
:109810001D2F1C0FEDB7FEB737960FB6F894FEBF9D
:109820000FBEEDBF83E00E943F2940E154E16C2F61
:1098300080E00E946C2C10923617D093371789E085
:1098400099E00E94512A10923617109337178CEF27
:1098500098E00E94512A8FEF96E10F94C240811147
:10986000E1CF61E08FE199E00E94883889EE93E0D2
:1098700030E6019729F0232F2A950000E9F7F9CF68
:10988000F89489EE93E038EE019729F0232F2A957A
:109890000000E9F7F9CF0E94B8D7FF2041F00E94FD
:1098A0006F360E948122909905C0A895FCCF0E9436
:1098B0007F22F7CF909B02C0A895FCCFF0E0E0E0BC
:1098C000DF91CF911F910F91FF9019945F926F924A
:1098D0007F928F929F92AF92BF92CF92DF92EF9240
:1098E000FF920F931F93CF93DF931F92CDB7DEB7F5
:1098F0007C0139018B015B01A40EB51ED12CC12C5A
:10990000A016B10609F450C0F70180809180F801DB
:1099100051908F015982C4010F94215C5816B9F1FE
:10992000652DC4010F94295CFFEFCF1ADF0AC60131
:109930008F779927892B21F162E070E080E090E039
:109940000F949C38C4010F94215C99818917F9F018
:109950000E9404498BE596E00E943D3781E00F901C
:10996000DF91CF911F910F91FF90EF90DF90CF90FB
:10997000BF90AF909F908F907F906F905F90089571
:1099800062E070E080E090E00E943936DBCFBE01FB
:109990006F5F7F4FC3010F94C428F70180819181CD
:1099A000019691838083ACCF80E0D9CF809159110B
:1099B00090915A112FEF3FEF981751F0E92FF0E0F7
:1099C000E75AFE4E228130E09F5F9F7790935A11B5
:1099D000C90108951F920F920FB60F9211240F9094
:1099E0000FBE0F901F9018951F920F920FB60F92F7
:1099F00011240BB60F920F931F932F933F934F9306
:109A00005F936F937F938F939F93AF93BF93CF9306
:109A1000DF93EF93FF93C091C60000915A11D0914C
:109A2000591111E01D0F1F7790918104913108F0B9
:109A30009FC0E92FF0E08827EF5DF24B8F4F0D9428
:109A4000EC5C324D614D704D7F4D864DB84D8A4D69
:109A5000B84D8E4D924DB84D964D9A4D9E4DA54D9B
:109A6000B84DB04DC03229F028F5CA3011F0CD30D4
:109A700031F5011731F0ED2FF0E0E75AFE4EC283C9
:109A8000D12FD0935911FF91EF91DF91CF91BF91D9
:109A9000AF919F918F917F916F915F914F913F9186
:109AA0002F911F910F910F900BBE0F900FBE0F9033
:109AB0001F901895CD3481F081E0CE3471F080E1B3
:109AC0000CC0CA3338F4C033A0F6C03291F2CD32A4
:109AD000B1F7CFCFCD3499F782E080938104C9CF1D
:109AE000C13359F018F4C03221F2E9CF88E0C43311
:109AF000A1F38BE0C83389F3E2CF83E0EECF84E0BB
:109B0000C03359F386E0C13341F3D9CF85E0C83380
:109B1000B1F6E3CF87E0C23391F6DFCF89E0C133FE
:109B200071F6DBCF8AE0C03351F6D7CF8CE0C73374
:109B300031F6D3CF8DE0C63311F6CFCFC03209F462
:109B400098CF8EE0C33549F2BACF80ED8C0F8A30C2
:109B500008F08FCF9FE0909381048093800489CF99
:109B6000CA3019F0CD3009F084CF1092810481CF32
:109B7000CA3019F0CD3009F07CCF80913917882395
:109B8000A1F3973041F138F4953079F710927402CF
:109B90001092FB08EACF9A3011F19F3031F7909183
:109BA00080048091F8081092F808823089F384309C
:109BB000E9F08130D1F69923B1F09130B1F682E02D
:109BC0008093FA088091F908882379F2109255025F
:109BD0000E946C22CACF81E08093E906C6CF81E063
:109BE0008093E806C2CF8093FA08BFCF83E39EE15B
:109BF0009093710880937008B8CF8EBD0DB407FEA6
:109C0000FDCF08958FEF8EBD0DB407FEFDCF8EB54D
:109C10000895909164009B7F90936400982F906AC0
:109C200096959CBD80FD03C091E0863009F490E0DC
:109C30009DBD0895CF93DF93EB010E943D37CE0188
:109C4000DF91CF910C948AD1AF92BF92CF92DF92E5
:109C5000EF92FF920F931F93CF93DF93CDB7DEB7B1
:109C6000E6970FB6F894DEBF0FBECDBF0091FF049C
:109C700010910005F80101900020E9F731976F017C
:109C8000C01AD10AF801CF01801B910B8C159D05DC
:109C90003CF481918F32B9F7DF0111971C92F3CF19
:109CA0008BE1E6EAF7E1DE015C9601900D928A9580
:109CB000E1F7F12CE12CEC14FD040CF05DC0F8018F
:109CC000EE0DFF1D8081811103C08FEFE81AF80AA5
:109CD0005801AE0CBF1CF5018081882309F44CC0EB
:109CE000FFEFEF1AFF0AF801EE0DFF1D7F01E01AEA
:109CF000F10A81918111FACFCE014C960E949BD539
:109D00008BE1FE017C96DE01119601900D928A9501
:109D1000E1F7B501CE0101960E94FCCDCE0101967E
:109D20000E943F348FE20E9404378091CD1381114D
:109D30003BC08FE593E00E948AD18091851784FF14
:109D40001BC019821C8221E0A501BE01645E7F4F09
:109D5000CE0101960F94CC08811129C08AE00E949F
:109D600004370E940449B50189E095E10E941A4E2A
:109D7000CE0101960E943F348AE00E940437CE0152
:109D80004C960E943F34E6960FB6F894DEBF0FBEA5
:109D9000CDBFDF91CF911F910F91FF90EF90DF909A
:109DA000CF90BF90AF9008958DEC93E1C4CFCE01DA
:109DB0004C960E94F2D48BE1FE013196DE015C9656
:109DC00001900D928A95E1F7CE0101960E943F34F1
:109DD00072CF2F923F924F925F926F927F928F92AB
:109DE0009F92AF92BF92CF92DF92EF92FF920F932A
:109DF0001F93CF93DF9300D000D000D01F921F920B
:109E0000CDB7DEB7B82E80914612843008F0D1C1AC
:109E10000F94CF386B017C0180914612811108C0EC
:109E20008091591190915A11891B8F7709F4D9C6E5
:109E300081E6A82E13C08A3019F08D3009F0F6C0E3
:109E4000109241128091DF119091E011FC01E552D6
:109E5000FE4E1682892BF1F40E9468F5809146121D
:109E6000843008F0ECC08091591190915A11891BEF
:109E70008F7709F4E4C00E94D64C97FFDCCF0E9494
:109E8000254881EA97E00E943D37809159118093DF
:109E90005A11E4CF1092E0111092DF1101EE11E19E
:109EA000F8018191803209F446C08E3409F0A9C0CE
:109EB0006CE977E0C8010F9480554C01892B41F083
:109EC0006EE470E0C80104960F944A60009709F4AC
:109ED000C8014AE050E070E060E001960F94F05253
:109EE0002B013C018091DB119091DC11A091DD11DF
:109EF000B091DE110196A11DB11D481659066A06E2
:109F00007B0629F060E089E697E0892851F16AE252
:109F100070E0C8010F9479609C01009729F1982F97
:109F2000901B912C992349F09150F801E90FF11DF4
:109F300080819826F7CF8F01B3CF4AE050E070E0E0
:109F400060E0C90101960F94F052292D30E050E0F5
:109F500040E0621773078407950751F060E08AE4D8
:109F600097E00F94912D7ACF60E080E297E0F9CFEF
:109F70004092DB115092DC116092DD117092DE1183
:109F80008091B3088130E1F067E470E0C8010F947C
:109F90004A600097A9F04AE050E070E060E0019666
:109FA0000F94F052643071058105910548F48FE7F4
:109FB00096E00E943D3760E085E796E00E9492B50A
:109FC000C0920009D0920109E0920209F0920309BF
:109FD0008091E1118B3309F441CF80914612843096
:109FE00008F03CCF809148128A9DC001112461EE97
:109FF00071E1875B9D4E0F94556080E00F944B2D6F
:10A000002DCF8091851780FFBBCF66E77FE3C80126
:10A010000F948055009731F0FC01838180538A3082
:10A0200008F0AECF60E086EF96E09BCF2FED31E1F8
:10A0300041EE51E161E472E10E94FB210FCF80917A
:10A04000851782FFB6C01A82198271E6F72EE0E109
:10A05000EE2EF9E6DF2E80914612843008F0A9C07A
:10A060000E9433228111A5C041E050E0BE016B5F28
:10A070007F4F8AEE98E10E942AD20D8110E001976D
:10A0800011F00FEF1FEF8091F2189091F318A0914B
:10A09000F418B091F5188093811790938217A093CC
:10A0A0008317B09384170E9433220F3F100749F49F
:10A0B000811107C00E9425488FEB97E00E943D3731
:10A0C000CACF40914812242F30E00A3061F00D30A1
:10A0D00051F0882309F45FC089819A81009719F0B3
:10A0E00001969A8389831092820489819A81F29ED3
:10A0F000F001F39EF00D1124EA5BFD4EE80FF91F0D
:10A100001382892B69F50E9468F50E943322882307
:10A1100009F4A1CF0E9456DF8AEE98E10E94F2D4A2
:10A1200080917C17882391F1815080937C178D9DBD
:10A13000C001112462E08152984F0F94C446E0910F
:10A140007C1724E0E29FF0011124E552F84F608172
:10A150007181828193810E9412260F943B447BCFB0
:10A160001A82198281E00F944B2D80918117909172
:10A170008217A0918317B091841780934212909315
:10A180004312A0934412B0934512BFCF0F942A44B8
:10A19000E092B30860CF4F9DA0011124475B5D4E54
:10A1A0009E012F5F3F4F62E874E0802F0E94FB21E9
:10A1B00052CF0F94CF386B017C01B11004C0809155
:10A1C000DA07882351F0C092F008D092F108E092AB
:10A1D000F208F092F308BB24B3948091D8049091D4
:10A1E000D904A091DA04B091DB040097A105B10570
:10A1F00051F14091F0085091F1086091F20870918E
:10A20000F308840F951FA61FB71FA7019601281BEF
:10A21000390B4A0B5B0BDA01C901B7FD14C00E9470
:10A2200025486091FE087091FF088AE198E00E943D
:10A230001A4E8AE00E94043740E070E060E090E04F
:10A2400080E00E94D54B8091100290911102A09164
:10A250001202B0911302892B8A2B8B2B79F09091EB
:10A26000C3168091C416981709F4ACC1C092F008C7
:10A27000D092F108E092F208F092F30880919304F2
:10A28000909194049099E0C10196909394048093E6
:10A29000930480919304909194048E3E92406CF0CC
:10A2A0000E94254887EF97E00E943D3740E070E02C
:10A2B00060E090E080E00E94D54B0F94CF384B01D6
:10A2C0005C018091FB08811108C02091C316909118
:10A2D000C41681E0291301C080E020917F163091DF
:10A2E000801691E089272A3A31050CF480E091E04C
:10A2F00040918704509188046091890470918A0488
:10A30000452B462B472B09F490E0981789F08823BA
:10A3100009F4A0C1D501C40180569444A24FBF4F97
:10A320008093870490938804A0938904B0938A044F
:10A3300040905511509056116090571170905811DF
:10A3400020918304309184044091850450918604C7
:10A35000C301B2010F940356882319F18091870439
:10A3600090918804A0918904B0918A04409283045A
:10A37000509284046092850470928604892B8A2B03
:10A380008B2B09F449C0D501C40180569444A24FD7
:10A39000BF4F8093870490938804A0938904B0935F
:10A3A0008A048091870490918804A0918904B091D7
:10A3B0008A040097A105B10579F1881A990AAA0AB9
:10A3C000BB0AB7FC29C0109287041092880410922F
:10A3D000890410928A0482EE97E00E943D3760E083
:10A3E0008EEC97E00E9492B5809181169091821632
:10A3F0001816190624F490E080E00E94D8DE8091BF
:10A400001D0990911E091816190634F410921E09A0
:10A4100010921D090E9482C980918F04909190042E
:10A42000A0919104B091920446015701881A990AAB
:10A43000AA0ABB0AD501C401B7FD9CC12091C3166D
:10A440009091C4164091640280916302291306C161
:10A450009091390A899FC0011124880F892F881F84
:10A46000990B91958D8380913A0A489FC0011124E0
:10A47000880F892F881F990B91958E830F94CF3861
:10A4800069837A838B839C8340E0BE016F5F7F4F3B
:10A49000CE0105960E94AADF6D8170E089E00F94DD
:10A4A000C63741E0BE016F5F7F4FCE0105960E9427
:10A4B000AADF6E8170E087E00F94C6378091F506C1
:10A4C000882309F44AC10091330210913402C80173
:10A4D00002972091811630918216281739070CF4C3
:10A4E0003CC18090C4168F82188619861A861B86F6
:10A4F0008091C3169F80891509F4CAC0892D90E008
:10A500003BE6A32EA89EF001A99EF00D1124E25B6C
:10A51000F54F458956896789708D452B462B472B0A
:10A5200081F4418D528D638D748D452B462B472BC5
:10A5300041F4458D568D678D70A1452B462B472BD9
:10A54000E1F12BE6B22EB89E9001B99E300D112498
:10A55000A901425B554F1A01FA0161817281838121
:10A5600094810F94A35F4B015C01F10161A172A181
:10A5700083A194A10F9408562B013C01F10165A120
:10A5800076A187A190A50F9408569B01AC01C30149
:10A59000B2010F94EF5DA50194010F9469564B0130
:10A5A0005C01288539854A855B850F94555F1816AF
:10A5B00024F488869986AA86BB868F818F5F8F70E8
:10A5C0008F8396CFBB2019F01092950457CE0F942D
:10A5D000CF380091F0081091F1082091F2083091E5
:10A5E000F3088090100290901102A0901202B09097
:10A5F0001302080D191D2A1D3B1D601B710B820BD8
:10A60000930B97FDE1CF80919504811137CE81E0C6
:10A61000809395045F9A80916E088E7F80936E0878
:10A620008A9A80916E088D7F80936E0880910801D0
:10A63000809581708093060180916E088B7F809356
:10A640006E080E947F221ACE181619060CF021CE31
:10A6500001971BCE80E090E0DC0162CE2091C41611
:10A660005BE6259F90011124225B354FF901EF59DC
:10A67000FF4F9081899FC0011124880F892F881F67
:10A68000990B91958D832E593F4FF9018081EDCE25
:10A6900020912D0230912E0240912F0250913002D4
:10A6A000688579858A859B850F9469564B015C0185
:10A6B000B801012E000C880B990B0F940A569B01D0
:10A6C000AC01C501B4010F94F55C69837A838B8377
:10A6D0009C834091310250913202B801CE01019623
:10A6E0000E9483D889809A80AB80BC8040908B0484
:10A6F00050908C0460908D0470908E04A3019201A0
:10A70000C501B4010F94035687FF16C028E431EE4B
:10A710004AE75FE3C301B2010F94695620E037EDC9
:10A7200043EA5CE30F94F55CA50194010F9469562C
:10A7300069837A838B839C8369817A818B819C81F5
:10A7400060938B0470938C0480938D0490938E049B
:10A750000F94615ECB010E94D8DEF4E6CF0ED11CCF
:10A76000E11CF11CC0928F04D0929004E0929104FD
:10A77000F09292040E9468F58091B308882309F44E
:10A78000F0C180915502882309F471C08091F908C5
:10A7900081116DC00E945D36811105C08091DA077C
:10A7A000882309F464C0F894649B10C0809151021E
:10A7B00090915202A0915302B09154028093E0060E
:10A7C0009093E106A093E206B093E3066091E00661
:10A7D0007091E1068091E2069091E306789420E082
:10A7E00030E0A9010F94035687FF41C001E00093B8
:10A7F000F9088091DA07811138C00E94B9380093B6
:10A80000F80840E366E878E085EB90E40E94BE3803
:10A8100061E089EA90E40E94A0381091DC0460E0D5
:10A82000102784E59AE069F484E798E00E9488386C
:10A8300080E30E9404378AE00E94043760E087E5E5
:10A8400098E00E94883882E698E00E943D3780E3D5
:10A850000E9404378AE00E940437112331F08DE50D
:10A8600098E090937108809370080E9456DF909151
:10A870000901892F8095817010910802181709F439
:10A880005AC0209185172062209385178093080273
:10A8900090FD10C064EF71E080E090E00E943936D6
:10A8A0000E94FBD48091851783FDBEC1112309F45A
:10A8B00042C002C00E94BACD123008F46BC100E061
:10A8C0000E94D72883E0809380020F94CF386C5980
:10A8D0007F4F8F4F9F4F60930405709305058093C2
:10A8E000060590930705002331F1123021F5809180
:10A8F000851783FF20C00F948743882379F081E078
:10A900000F94A34242EB50E069E479E08BE897E1D1
:10A910000E942AD28BE897E10E94F2D40E942D3443
:10A92000811144C10E9417340F94094581E080933E
:10A930007B170F944B450F94CF386B017C0110911E
:10A940000F021123F1F08091FC088823D1F040918F
:10A95000960450919704609198047091990446016F
:10A960005701841A950AA60AB70AB501A40177FD12
:10A970001AC0833009F430C10CF01FC181300CF0D3
:10A9800024C1212F30E0A8EEB3E00F949B5CC60EEB
:10A99000D71EE81EF91EC0929604D0929704E0924A
:10A9A0009804F092990480911109813009F073C0E4
:10A9B0000F94CF386B017C0180919E0490919F048D
:10A9C000A091A004B091A104A7019601281B390B06
:10A9D0004A0B5B0BDA01C901B7FD3AC0D701C601CA
:10A9E000805F984DAF4FBF4F80939E0490939F041C
:10A9F000A093A004B093A1048090CA059090CB05C9
:10AA0000A090CC05B090CD050F94A300AB01BC0184
:10AA10004093CA055093CB056093CC057093CD0548
:10AA200080915F0890916008A0916108B0916208E0
:10AA300088199909AA09BB09840F951FA61FB71F7A
:10AA400080935F0890936008A0936108B0936208B8
:10AA500080919A0490919B04A0919C04B0919D04D4
:10AA600046015701881A990AAA0ABB0AD501C401EE
:10AA7000B7FD11C020E8C20E2EEED21E26E3E21E64
:10AA8000F11CC0929A04D0929B04E0929C04F09234
:10AA90009D040E945ADE0F9434050E949EB9809155
:10AAA000D704882379F10F94CF386B017C01809112
:10AAB000D3049091D404A091D504B091D60446015A
:10AAC0005701881A990AAA0ABB0AD501C401B7FD21
:10AAD00019C02091D70430E0A8EEB3E00F949B5C3E
:10AAE000C60ED71EE81EF91EC092D304D092D4041D
:10AAF000E092D504F092D60480E00F944F0B8AE0E8
:10AB00000E9404378091D204882359F10F94CF38E2
:10AB10006B017C018091CE049091CF04A091D00470
:10AB2000B091D104A7019601281B390B4A0B5B0B8E
:10AB3000DA01C901B7FD15C02091D20430E0A8EEBA
:10AB4000B3E00F949B5CC60ED71EE81EF91EC092A0
:10AB5000CE04D092CF04E092D004F092D1040F94AE
:10AB6000AA432B960FB6F894DEBF0FBECDBFDF9180
:10AB7000CF911F910F91FF90EF90DF90CF90BF90FA
:10AB8000AF909F908F907F906F905F904F903F908D
:10AB90002F90089560E087E998E00E9492B5809137
:10ABA000120581118CCE0E94B68689CE84EB98E086
:10ABB0009093710880937008BECE843009F0E1CE86
:10ABC0000E9404498BEB98E004C00E9404498AEE7D
:10ABD00098E00E943D37D5CE0E94044983ED98E06D
:10ABE000F8CF8091000990910109A0910209B091DC
:10ABF0000309A7019601281B390B4A0B5B0BDA01ED
:10AC0000C901885E9340A109B109B7FD11C989EB5B
:10AC100097E00E943D37C0920009D0920109E0926E
:10AC20000209F092030904C9123028F460E085EAB1
:10AC300098E00E9492B501E043CECF93DF93C82FF6
:10AC4000D62F8091FF1083FD14C080914B0A811193
:10AC500010C08091850290918602AC01415051094B
:10AC600020918116309182162417350714F40E9422
:10AC7000D8DE40E06D2F8BE00E949F87CC2339F017
:10AC800040E061E080E0DF91CF910D94470D80912D
:10AC90004B0A91E089278093740280917402882383
:10ACA00089F080917F1690918016209181163091C5
:10ACB0008216821B930B97FF03C091958195910992
:10ACC000029744F4109274028091FF1083FF06C033
:10ACD000C1E01AC080E00E94E94EDFCFC0914B0A6C
:10ACE000C11112C080918502909186020197209136
:10ACF0008116309182162817390754F70E940449AB
:10AD000088EB99E00E943D378C2FDF91CF91089519
:10AD1000AF92BF92CF92DF92EF92FF920F931F9369
:10AD2000CF93DF93CDB7DEB764970FB6F894DEBF4D
:10AD30000FBECDBF0E940849D82E87FDB5C08AE559
:10AD40000E948D32882309F4C0C040E050E0BA016F
:10AD50008AE50E94A8327B018C014D2D63E085E0DD
:10AD60000E949F87209151113091521140915311AF
:10AD70005091541160E070E088EC93E40F94F45C1F
:10AD80005B016C019701A8010F94555F181614F030
:10AD90007501860120E030E0A901B701C8010F94D8
:10ADA000555F181624F4E12CF12C00E010E0B701F7
:10ADB000C8010F94615E072E000C880B990B0F944D
:10ADC0000A566D837E838F83988720E030E0A90147
:10ADD0000F940356882321F0CE0105960E94602629
:10ADE00080E090E0A0EAB1E489879A87AB87BC87CE
:10ADF0001D861E861F86188A8CE40E943F32882397
:10AE000009F468C00E9415326B017C0120E030E03B
:10AE1000A901C701B6010F94555F87FF04C0F7FA77
:10AE2000F094F7F8F094C98ADA8AEB8AFC8A2091C8
:10AE30008116309182162430310574F080917F168E
:10AE400090918016821B930B97FF03C0919581957B
:10AE5000910901E004970CF400E063E080E00E94B7
:10AE60001D56811140C083E0809324021092110589
:10AE70000E94B6866D817E818F8198858B019C01B1
:10AE8000305809831A832B833C8320E030E0A901EA
:10AE90000F940356882321F0CE0101960E9460266C
:10AEA000109211050E94B68664960FB6F894DEBF24
:10AEB0000FBECDBFDF91CF911F910F91FF90EF900B
:10AEC000DF90CF90BF90AF900895E12CF12C00E27D
:10AED00011E443CFC090D205D090D305E090D405C3
:10AEE000F090D50593CF83E0E82E22E0AE01475FD6
:10AEF0005F4FBE016F5E7F4FCE010D960F94952F71
:10AF0000B9CF6F927F928F929F92AF92BF92CF9262
:10AF1000DF92EF92FF920F931F93CF93DF9300D0B6
:10AF200000D01F921F92CDB7DEB75C014B013A01F2
:10AF3000F22E68010091EE061092EA061092EB06DE
:10AF40001092EC061092ED061092EE060F94DB388C
:10AF500080918116909182168C159D051CF4C60176
:10AF60000E94D8DE60E080E00E941D5681112FC152
:10AF7000109211050E94B6861C141D0444F4C601EB
:10AF80000E94D8DE40E060E080E00F94470D40E092
:10AF900060E088E00E949F8760E081E00E941D568B
:10AFA00080E090E0A0E7B2E489839A83AB83BC831E
:10AFB00080E090E0A0E8B0EC8D839E83AF83B887FB
:10AFC000BE016F5F7F4FCE0105960E9436F587E088
:10AFD0000E9476F3811158C08091511190915211C5
:10AFE000A0915311B09154114091AE045091AF040F
:10AFF0006091B0047091B104C090AA04D090AB04E9
:10B00000E090AC04F090AD04C092E008D092E1086A
:10B01000E092E208F092E3084093E4085093E508D8
:10B020006093E6087093E7088093E8089093E90836
:10B03000A093EA08B093EB0880E090E0A8E4B2E4C3
:10B0400089839A83AB83BC83CE0101960E9456FC10
:10B050008091B2049091B304A091B404B091B5046E
:10B060008093E8089093E908A093EA08B093EB086E
:10B0700080E090E0A0EAB0E489839A83AB83BC834C
:10B08000CE0101960E9456FCC12CD12C80E7E82EFF
:10B0900082E4F82EC982DA82EB82FC8280E090E0C2
:10B0A000A0E8B0E48D839E83AF83B887BE016F5F55
:10B0B0007F4FCE0105960E9436F520E030E0A901D1
:10B0C0006091B6047091B7048091B8049091B9046E
:10B0D0000F94035687FF0BC0C982DA82EB82FC8291
:10B0E000BE016F5F7F4F86EB94E00E9436F5809142
:10B0F000B6049091B704A091B804B091B9048093BC
:10B10000551190935611A0935711B09358118093F5
:10B11000EC089093ED08A093EE08B093EF088CEE46
:10B1200098E00E945EF18091D60581110F94CD4286
:10B13000109211050E94B68661E081E69AE00E94B5
:10B1400088388091DA0781508093DA0744EF5DE117
:10B1500069E67AE085E00F949F308091DA078823D2
:10B1600039F00F943B448091DA0781508093DA07DD
:10B170008091A904882351F01092A9048091A7041A
:10B180008093390A8091A80480933A0A0E946C2225
:10B1900080911109823011F40F9465010F940446D7
:10B1A0000E94B68628960FB6F894DEBF0FBECDBFBC
:10B1B000DF91CF911F910F91FF90EF90DF90CF9093
:10B1C000BF90AF909F908F907F906F900895E12CEB
:10B1D0002F2DA301B401C5010F94952FCDCE4F9211
:10B1E0005F926F927F92AF92BF92CF92DF92EF9277
:10B1F000FF921F93CF93DF9300D000D01F921F9236
:10B20000CDB7DEB75C01E62EF42E642F80E00E94FD
:10B210001D56182F81111BC0EE2021F01092110530
:10B220000E94B686812F28960FB6F894DEBF0FBE17
:10B23000CDBFDF91CF911F91FF90EF90DF90CF9026
:10B24000BF90AF907F906F905F904F900895EE20E9
:10B2500029F040E06F2D83E00E949F8780E090E01E
:10B26000A0E7B2E48D839E83AF83B88780E090E04F
:10B27000A0E8B0EC89839A83AB83BC83BE016B5F8B
:10B280007F4FCE0101960E9436F568E873E180E0B9
:10B2900090E00E943936C12CD12C88ECE82E81E454
:10B2A000F82ECD82DE82EF82F88680E090E0A0E882
:10B2B000B0E489839A83AB83BC83BE016B5F7F4F0D
:10B2C000CE0101960E9436F5409038115090391108
:10B2D00060903A1170903B11C0923811D0923911A0
:10B2E000E0923A11F0923B1180E090E0A0E2B2E4EB
:10B2F0008D839E83AF83B887F50180819181A28180
:10B30000B38189839A83AB83BC83BE016B5F7F4F1C
:10B31000CE0101960E9436F54092381150923911B3
:10B3200060923A1170923B11129A64E670E080E0EC
:10B3300090E00E94393676CFBF92CF92DF92EF92A3
:10B34000FF920F931F93CF93DF9300D01F92CDB73F
:10B35000DEB77C016B018A01B22E61E084E59AE0E0
:10B360000E94883844EF5DE16BE57AE085E00F9458
:10B370009F309091DA0781E0890F8093DA078091FE
:10B38000851782FF06C08B7F809385179E5F909301
:10B39000DA070F949D0180E1E9E4F1E1AAEAB4E063
:10B3A00001900D928A95E1F70E9456DF8091A904E1
:10B3B00081110FC081E08093A9048091390A8093A4
:10B3C000A7041092390A80913A0A8093A804109237
:10B3D0003A0A20E030E0A901F701608171818281A1
:10B3E00093810F9403568823F1F080914B0A8111C9
:10B3F0000CC08091850290918602019720917F1662
:10B40000309180162817390774F080E090E0A0E7AB
:10B41000B2E489839A83AB83BC83BE016F5F7F4FA5
:10B42000C7010E9436F587E00E9476F3811103C0C0
:10B43000B6010F94790420E030E0A901F8016081A1
:10B440007181828193810F940356882329F042E011
:10B450006B2DC8010E94EF58129A64E670E080E0FC
:10B4600090E00E94393681E00F900F900F900F907E
:10B47000DF91CF911F910F91FF90EF90DF90CF90D0
:10B48000BF900895CF92DF92EF92FF92CF93DF9318
:10B490006B017C01D42FC091FC0883E08093FC08F1
:10B4A00081E08093FB08C114D104E104F10431F080
:10B4B0000F94CF38C60ED71EE81EF91E8091FB08E8
:10B4C000882389F0C114D104E104F10421F48D2F03
:10B4D0000E94E94EF3CF0F94CF386C197D098E0985
:10B4E0009F0997FDF4CF1092FB08C093FC08DF91F1
:10B4F000CF91FF90EF90DF90CF9008951F93CF935F
:10B50000DF93D82FC62F0E94C14B61E08C2F0E9481
:10B5100045340F94CF38685370458F4F9F4F6093D9
:10B52000EA067093EB068093EC069093ED0610927A
:10B53000EE061091FC0883E08093FC0830E020E0E8
:10B540004AED50E466E47AE082E00E94E13881E06E
:10B550008093FB088091FB08882309F463C060E0B6
:10B560008C2F0E9445348091EE06882309F456C042
:10B5700040E060E08AE00E949F870E9404498CE2DC
:10B580009AE00E943D3730E020E046E15AE06DE16C
:10B590007AE082E00E94E13841E060E070E0CB01B7
:10B5A0000E94425A30E020E050E040E069E07AE05A
:10B5B00085E00E94E1381092EA061092EB061092A4
:10B5C000EC061092ED061092EE060F94DB3860E068
:10B5D00080E00E941D568D2F0E94C14B0F94CF38E2
:10B5E000685370458F4F9F4F6093EA067093EB0648
:10B5F0008093EC069093ED061092EE0630E020E08A
:10B600004AED50E46DEF79E082E00E94E13881E09C
:10B610008093FB0861E08C2F0E94453481E00E94FA
:10B62000E94E98CF1093FC08DF91CF911F910895B8
:10B63000CF92DF92EF92FF920F931F93CF93DF93FE
:10B64000CDB7DEB7A0970FB6F894DEBF0FBECDBF63
:10B650000E94084987FDD1C0482F61E081E00E9427
:10B660009F8785E40E943F32882309F4D5C00E9459
:10B6700015326B017C0120E030E0A9010F94555F89
:10B6800087FF04C0F7FAF094F7F8F094F7FAF09413
:10B69000F7F8F094C98ADA8AEB8AFC8A8CE0EBE846
:10B6A000F2E0DE01119601900D928A95E1F78AE5AC
:10B6B0000E948D32882351F040E050E0BA018AE5C3
:10B6C0000E94A83269877A878B879C8788E50E94C9
:10B6D0008D32882351F040E050E0BA0188E50E94A5
:10B6E000A83269837A838B839C8389E50E948D329B
:10B6F000882351F040E050E0BA0189E50E94A83269
:10B700006D837E838F83988785E50E943F328823EF
:10B7100009F489C00E9415326B017C0120E030E001
:10B72000A901C701B6010F94555F87FF04C0F7FA5E
:10B73000F094F7F8F094F7FAF094F7F8F094CD8AD3
:10B74000DE8AEF8AF88E198E1A8E1B8E1C8E8CE480
:10B750000E943F32882309F46FC00E9415326B01AA
:10B760007C0120E030E0A901C701B6010F94555FCC
:10B7700087FF04C0F7FAF094F7F8F094CD8EDE8ED0
:10B78000EF8EF8A262E070E082E40E94F333F82EBC
:10B790008091DA07811131C021E0AE014B5E5F4F2D
:10B7A000BE016F5F7F4FCE0141960E949C59882356
:10B7B00021F16F2D81E00E947E5A82E50E948D3238
:10B7C000882309F442C00E94113240E050E060EA50
:10B7D00071E44D875E876F87788B2091DA0722238B
:10B7E00061F08C012F2DAE01435F5F4FBE01635EA0
:10B7F0007F4FCE0149960E948157A0960FB6F894CC
:10B80000DEBF0FBECDBFDF91CF911F910F91FF9093
:10B81000EF90DF90CF900895C12CD12C80E8E82ED6
:10B8200080E4F82E33CFC090CE05D090CF05E090C5
:10B83000D005F090D10572CFC090D205D090D3053D
:10B84000E090D405F090D5058CCF90E080E0BDCF9E
:10B85000CF92DF92EF92FF920F931F93CF93DF93DC
:10B86000CDB7DEB76C970FB6F894DEBF0FBECDBF75
:10B870008CE40E943F32882309F4C3C00E94153231
:10B880006B017C0120E030E0A9010F94555F87FF38
:10B8900004C0F7FAF094F7F8F094F7FAF094F7F898
:10B8A000F094C98EDA8EEB8EFC8E8CE0EBE8F2E041
:10B8B000DE01119601900D928A95E1F788E50E94CC
:10B8C0008D328823A1F040E050E0BA0188E50E9463
:10B8D000A8322091FB093091FC094091FD0950915B
:10B8E000FE090F94F45C69837A838B839C8389E5DA
:10B8F0000E948D328823A1F040E050E0BA0189E532
:10B900000E94A8322091FB093091FC094091FD0969
:10B910005091FE090F94F45C6D837E838F8398872A
:10B920008AE50E948D32882351F040E050E0BA0150
:10B930008AE50E94A83269877A878B879C87F09076
:10B940008517F2FAFF24F0F840E061E080E00E9401
:10B950009F8760E080E50E940234E82E1D861E86E7
:10B960001F86188A8091DA0781113CC02E2DAE0106
:10B97000435F5F4FBE016F5F7F4FCE0149960E94CC
:10B980009C59882379F18091D60581110F94CD427D
:10B99000FF2011F0EE2031F160E080E00E947E5A3D
:10B9A000898D9A8DAB8DBC8DB0588D8B9E8BAF8B56
:10B9B000B88F198A1A8A1B8A1C8A1D861E861F86C2
:10B9C000188A8091DA07882369F010E000E020E00F
:10B9D000AE014B5E5F4FBE016F5E7F4FCE010D9695
:10B9E0000E9481576C960FB6F894DEBF0FBECDBF94
:10B9F000DF91CF911F910F91FF90EF90DF90CF904B
:10BA00000895C12CD12C80E8E82E80E4F82E45CF93
:10BA10002F923F924F925F926F927F928F929F925E
:10BA2000AF92BF92CF92DF92EF92FF920F931F934C
:10BA3000CF93DF93CDB7DEB7E1970FB6F894DEBFB3
:10BA40000FBECDBF89AB2091FC0828AB21E020932D
:10BA5000FC088091FE048D3409F461C4843511F42E
:10BA60000C94A671873409F044C18091FC04909134
:10BA7000FD048A31910509F4D5C108F03DC1843037
:10BA8000910508F030C12091B3088230910508F487
:10BA900051C1213009F054C111E0029709F010E0C2
:10BAA0000E94BF3219821A821B821C821D821E8252
:10BAB0001F82188682E50E948D32882309F451C1C5
:10BAC0000E9415326B017C0120E030E0A9010F9447
:10BAD0000356882309F4EAC04090491150904A1156
:10BAE00060904B1170904C1180914D1190914E11BE
:10BAF000A0914F11B091501188A799A7AAA7BBA7F1
:10BB00008090E0089090E108A090E208B090E308EF
:10BB10008091E4089091E508A091E608B091E708CB
:10BB20008CA79DA7AEA7BFA7A5019401C301B20131
:10BB30000F94035681110DC02CA53DA54EA55FA500
:10BB400068A579A58AA59BA50F940356882309F4B7
:10BB5000ADC0A3019201C501B4010F94F45C20E0D3
:10BB600030E040E05FE30F9469566CA37DA38EA3A1
:10BB70009FA328A539A54AA55BA56CA57DA58EA583
:10BB80009FA50F94F45C20E030E040E05FE30F9469
:10BB900069562B013C0120E030E0A901C701B60144
:10BBA0000F940356881F8827881F181709F4D0C0E0
:10BBB00080E090E0A0E8BFEB88A799A7AAA7BBA761
:10BBC0002CA13DA14EA15FA1CA01B9010F946956F4
:10BBD0004B015C01A3019201C301B2010F946956AC
:10BBE0009B01AC01C501B4010F94F55C0F94A35FF8
:10BBF0004B015C01AC019B01C701B6010F94F45CE1
:10BC00006CA77DA78EA79FA7A5019401C701B601C8
:10BC10000F94F55C9B01AC016CA57DA58EA59FA53D
:10BC20000F9469566B017C0120E030E0A9010F946C
:10BC3000555F87FD92C0C701B6010F94A35F6B01EA
:10BC40007C01C301B2019058A50194010F94EF5DEE
:10BC500028A539A54AA55BA50F946956A7019601A9
:10BC60000F9469562CA13DA14EA15FA10F94F55CE4
:10BC700069837A838B839C83A50194016CA17DA148
:10BC80008EA19FA10F94EF5D28A539A54AA55BA5BC
:10BC90000F946956A70196010F946956A30192016A
:10BCA0000F94F55C6D837E838F83988720E030E06E
:10BCB000A90169817A818B819C810F94035681113E
:10BCC00064C020E030E0A9016D817E818F8198857C
:10BCD0000F940356811159C00E94254880E79FE0C8
:10BCE0000E943D372DC08430910509F461C045970D
:10BCF00039F10F94872F24C08A32910509F4EAC1E3
:10BD000058F48C31910509F4A8C008F48EC04D9701
:10BD100081F70E94BA7414C08B35910509F457C29B
:10BD20008C35910509F457C28A35910511F71092A7
:10BD3000120906C0213021F40E94BF320E94A3F9EB
:10BD400039A931110C948F690F9430390C948F6993
:10BD500080E090E0A0E8BFE32FCFC12CD12C76018A
:10BD600070CF89E40E948D32882331F00E94153211
:10BD700069837A838B839C838AE40E948D32882333
:10BD800009F494CF0E9415328DCF412FBE016F5F11
:10BD90007F4F80EE98E00F94C9390F94CF386093AD
:10BDA000F0087093F1088093F2089093F308C8CFDD
:10BDB00080E50E948D32C12CD12C7601882321F0A0
:10BDC0000E94BE276B017C0183E50E948D3288238F
:10BDD00061F00E94153220E030E04AE754E40F940D
:10BDE00069560F94685E6B017C010E9456DF80915A
:10BDF0001014811105C060E086E89FE00E9492B5B2
:10BE00000F94CF38C60ED71EE81EF91E0F94CF38F8
:10BE10006C197D098E099F0997FF92CF80E00E94DF
:10BE2000E94EF4CF0E94D53E8BCF0F942646811168
:10BE300087CF8CE0E7E9F2E0DE01119601900D92E8
:10BE40008A95E1F770E060E080E50E949A32BE01D9
:10BE50006F5F7F4F0F94790473CF87E00E9476F372
:10BE6000811106C060E08FE40E940234811168CF26
:10BE70000E9456DF10923802609148118CE40E94B3
:10BE80000234982E80E00E94F9340F94CF386093EA
:10BE9000F0087093F1088093F2089093F308809172
:10BEA0007C0290917D02A0917E02B0917F028093EE
:10BEB000CA049093CB04A093CC04B093CD0480919A
:10BEC0007602909177029093C9048093C80484E627
:10BED00090E0909377028093760281E080936C08E3
:10BEE0000E9417FF8AE50E943F32A82E88E50E9433
:10BEF0003F32182F89E50E943F32B82E181308C030
:10BF0000B12EA11205C011E0BB24B394AA24A394BE
:10BF100082E50E948D32882309F4D2C00E94153236
:10BF20006C8F7D8F8E8F9F8F20E030E0A9010F9462
:10BF30000356882349F0111103C0BB2009F494C0B3
:10BF4000CE014C960F947431112309F488C0BB20A4
:10BF500009F482C01092491110924A1110924B11AB
:10BF600010924C1110924D1110924E1110924F11CF
:10BF7000109250110E9466F5E8EFF7E2C590D59057
:10BF8000E590F490ECEFF7E2459055906590749051
:10BF9000A7019601C301B2010F94035687FF95C014
:10BFA000A7019601C301B2010F94EF5D9B01AC01A3
:10BFB0000F94695620E030E040E85FE30F94F55CB1
:10BFC0000F94A35F20E030E048E452E40F946956F8
:10BFD00069837A838B839C83809151119091521154
:10BFE000A0915311B09154118CA39DA3AEA3BFA3F4
:10BFF00020E030E040EC5FE3C301B2010F946956EA
:10C000002B013C0177FA709477F8709420E030E0CF
:10C0100040EC5FE3C701B6010F9469569058DE010A
:10C0200011966D01ECA0FDA00EA11FA1A30192012C
:10C030000E945FF40F9495001092491110924A11DA
:10C0400010924B1110924C1110924D1110924E11F2
:10C0500010924F111092501180E00E94BDFCBB2045
:10C0600019F081E00E94BDFCAA2019F082E00E9434
:10C07000BDFC0E9466F580916B0880936C08892D49
:10C080000E94F9348091CA049091CB04A091CC0411
:10C09000B091CD0480937C0290937D02A0937E02A8
:10C0A000B0937F028091C8049091C9049093770265
:10C0B0008093760283E0809380020E940EFE40CE41
:10C0C00060E070E080E890E42BCFA3019201C7010B
:10C0D000B6016ACF8091B308813009F031CE89E48E
:10C0E0000E948D32082F10E0882319F00E9411322F
:10C0F000182F8AE40E948D32F82E882339F00E948E
:10C100001132011106C0883068F005C080E00023BC
:10C1100049F0183028F08FE89FE00E943D3710CE9C
:10C12000F110F1CF90E1E9E4F1E1A0EEB8E0019087
:10C130000D929A95E1F7002391F0B4E01B02F00113
:10C140001124E65AF84E40815181628173814093F7
:10C15000E0085093E1086093E2087093E308FF2041
:10C1600091F024E08202F0011124E65CF84E808117
:10C170009181A281B3818093E4089093E508A09314
:10C18000E608B093E70840E050E0BA0186E40E9478
:10C19000A8326B017C0120E030E0A9010F94555FCB
:10C1A00018168CF420E030E040E752E4C701B601F5
:10C1B0000F94EF5D69837A838B839C83CE01019614
:10C1C0000E9456FCBDCD60E070E0CB01F3CF8FE064
:10C1D00080931209B5CD8091FB04882381F18930C9
:10C1E00009F0AECD63EAA62E62E0B62E79E4C72E42
:10C1F00071E1D72EE12C00E010E0D5018D915D01B9
:10C200000E948D32F82E882361F0133011F4082F2C
:10C21000FE2C0E941532F601608371838283938322
:10C22000EF2C1F5FF4E0CF0ED11C143031F7EE205D
:10C2300009F457C00E9466F50E940EFE81CD53EAB4
:10C24000C52E52E0D52EF12CE12C00E010E0D601F5
:10C250008D916D010E948D32382E8823D9F10E9474
:10C2600015324B015C01133059F0F701E550F64FE0
:10C2700020813181428153810F94F45C4B015C0138
:10C28000F701E75BFE4E2081318142815381C50178
:10C29000B4010F94F45C2B013C012DEB37E346E82D
:10C2A00055EB0F94555F87FD0AC02DEB37E346E849
:10C2B00055E3C301B2010F94035618165CF4133012
:10C2C000C1F48092551190925611A0925711B092DC
:10C2D0005811032D1F5FB4E0EB0EF11C143009F070
:10C2E000B6CF002309F4A8CF85E591E10E945EF165
:10C2F000A3CFF701EF5CF64F5F01A30192016081CC
:10C300007181828193810F94F55CD5016D937D934A
:10C310008D939C931397812F0E9456F3DBCF8091CE
:10C32000FC049091FD048837910511F40C94A06BE6
:10C3300008F077C28D34910509F421C708F0D3C005
:10C340008A31910509F443C608F094C084319105FF
:10C3500009F489C508F071C08131910509F44AC515
:10C3600008F044C0029708F0C4CC80E50E948D32EA
:10C37000C12CD12C7601882321F00E94BE276B01AD
:10C380007C0183E50E948D32882361F00E94153282
:10C3900020E030E04AE754E40F9469560F94685E59
:10C3A0006B017C010E9456DF8091FF049091000593
:10C3B000009709F419C50F94D2458091FC0490911F
:10C3C000FD0460EB7FE0892B11F468EA7FE030E048
:10C3D00020E04AED50E482E00E94E13840E0C701ED
:10C3E000B6010E94425A0F940446AACC429709F023
:10C3F00080CC83E50E948D32882311F40C94D76A97
:10C400000F94CF386093F0087093F1088093F2088E
:10C410009093F3080E94153220E030E04AE754E49C
:10C420000F9469560F94685E609310027093110226
:10C43000809312029093130283CC8731910509F403
:10C4400047C570F48531910509F43EC5469709F05A
:10C4500050CC8091851782FD73CC0E94BACD70CCF0
:10C460008831910509F449C5499709F042CC0E94E9
:10C47000285C66CC8F31910509F44EC6D0F48C311E
:10C48000910509F411C608F4B5C58D31910509F47B
:10C4900013C64E9709F02DCC8091851783FF50CCA1
:10C4A0000F946D2F8091FF04909100050F94A1448B
:10C4B00047CC8934910509F44EC650F48032910579
:10C4C00009F401C6819709F014CC0E94244E38CC9F
:10C4D0008B34910509F44FC68C34910509F009CCD1
:10C4E0000F949D012DCC8B36910509F434C708F0CB
:10C4F0000FC18435910509F47CCF40F58135910554
:10C5000011F40C94B76A90F48E34910509F0F1CBD4
:10C5100070E060E083E50E94F3338E34910509F00A
:10C5200033C60E947CDE0F9404460ACC8235910506
:10C5300011F40C94CF6A8335910509F0DACB809120
:10C5400012098F7E806280931209FACB883691059A
:10C5500009F49EC608F09CC08535910511F40C9431
:10C560001A6B8C35910509F0C4CB0E94084987FDF0
:10C57000E7CB8091F70484FD0AC08091F90487FD20
:10C5800006C08091FA04837011F40C94486B23EA7E
:10C59000C22E22E0D22E30E0E32E31E1F32E10E065
:10C5A000D6018D916D010E948D32882309F466C0F9
:10C5B000133011F00C943F6B0E9415324B015C015B
:10C5C00020E030E040EA51E40F94035687FF4EC06C
:10C5D000A501940160912011709121118091221187
:10C5E000909123110F94EF5D2B013C01AC019B0155
:10C5F00060912D0A70912E0A80912F0A9091300A35
:10C600000F94695660932D0A70932E0A80932F0A17
:10C610009093300AA3019201609130117091311111
:10C6200080913211909133110F94695660933011BB
:10C630007093311180933211909333116091190AE4
:10C6400070911A0A80911B0A90911C0A0F94085647
:10C65000A30192010F9469560F94685E6093190AC2
:10C6600070931A0A80931B0A90931C0A80922011DF
:10C6700090922111A0922211B09223111F5FF4E039
:10C68000EF0EF11C143009F08BCF0E9432DF58CB33
:10C690008936910509F434C68A36910509F029CB0B
:10C6A00080E50F94A830F82E91E0981708F448CB55
:10C6B00081E40E943F326091390A062F10E0811117
:10C6C00002C00FEF10E089E40E948D32882311F43C
:10C6D0000C94D8710E94ED3190E01816190614F4EC
:10C6E00081E090E026E0289FF001299FF00D1124C1
:10C6F000EC54F74F04811581EF2DF0E0E75CF54F26
:10C700000F3F110519F010F00FEF10E0008318CB68
:10C710008137910509F481C608F068C08E3691050D
:10C7200009F427C608F059C08C36910509F408CBE6
:10C730008D36910509F0DDCA8091FF1083FD00CB95
:10C740000E940849F82E87FDFBCA89E40E948D32B9
:10C75000882311F40C94C6710E94ED3190E01816F4
:10C76000190614F481E090E026E0289FF001299F4B
:10C77000F00D1124EC54F74F8081918110E00E945C
:10C78000D8DE61E081E00F94134A20918116309148
:10C79000821680917F1690918016821793070CF075
:10C7A000A6C581EA90E19F938F938CEA90E19F93D5
:10C7B0008F931F920E9477B50F900F900F900F905C
:10C7C0000F9001E00F94DC49002309F4B9CA40E05E
:10C7D000612F8F2D0F94470DB3CA8F36910509F441
:10C7E000DBC58037910509F4ABCA83CA853791054B
:10C7F00009F45BC758F48237910509F44EC78337B3
:10C80000910509F076CA0E9464379ACA8637910565
:10C8100009F45DC78737910509F06BCA0E94F4FEE1
:10C820008FCA8A39E1E09E0709F48ACA08F03DC13F
:10C830008D3C910511F40C94A96C08F09FC08B39C4
:10C84000910509F46DC638F58D37910509F40FCEC1
:10C8500058F48937910509F04CCA10926C0810926F
:10C860006B080E9417FF6CCA8C38910509F4F4C557
:10C870008139910509F03DCA70E060E083E50E94CE
:10C88000F333823008F464C70E94254880E091E1C8
:10C890000E943D3755CA893C910509F4C5C7A8F5E2
:10C8A0008E3B910509F4FEC5883C910509F021CA2B
:10C8B0000E940849182F87FD43CA0091300984E47B
:10C8C0000E948D32F82E8823B9F00E9415324B0158
:10C8D0005C0120E030E0A9010F940356882309F49D
:10C8E000A1C724E01202F0011124E45DF64F80821A
:10C8F0009182A282B3820F2D602F83E50E940234C1
:10C90000809330090E9405C71BCA8B3C910509F42E
:10C91000B5C78C3C910509F0ECC98091F80487FDFE
:10C92000D0C78091F9048E7009F0CBC740913411C3
:10C9300050913511609136117091371185E291E176
:10C940000E94B539409138115091391160913A11D6
:10C9500070913B1182E291E10E94B53940913C1106
:10C9600050913D1160913E1170913F1182EC9CE21B
:10C970000E94B5398AE00E940437E2C98C3221E076
:10C98000920711F40C94CB6D08F04CC08C3D9105CE
:10C9900011F40C94FD6C58F48E3C910509F4DDC73C
:10C9A000833D910509F0A5C90E942D49C9C98D3D56
:10C9B000910511F40C94406D8232914009F099C9AF
:10C9C0008AE50E948D32882311F40C94976D0E94A1
:10C9D000153220E030E040E050EC0F94035687FF22
:10C9E00002C00C94B86D0E94153220E030E040E0A7
:10C9F00050E40F94555F181614F40C94BE6D0E9409
:10CA0000153220911C1130911D1140911E11509131
:10CA10001F110F9469560F94615ECB010F948339F7
:10CA20000C949D6D8F32B1E09B0711F40C94F86E5D
:10CA300078F58D32F1E09F0711F40C94E16D8E32A0
:10CA4000914009F056C983E50E943F32182F882390
:10CA500069F00E9411329C019093860280938502B6
:10CA600091E0232B09F090E090934B0A80E50E941F
:10CA70003F32882311F40C94D66E209185023091B8
:10CA80008602232B11F00E94013280934B0A58C971
:10CA9000803331E0930711F40C94626E8039914039
:10CAA00009F027C90E9456DF4BC9883FB1E09B07B8
:10CAB00011F40C945B7008F06DC08C3AF1E09F07A4
:10CAC00011F40C94306F08F03EC08D3931E09307BB
:10CAD00011F40C94897150F58C39914009F009C911
:10CAE0008091F704887811F00C94FC6E8091F90421
:10CAF000867011F00C94FC6E0E9404498EEC91E15A
:10CB00000E943D37809155020E9497394091510211
:10CB10005091520260915302709154028EEA91E159
:10CB20000E94B5398AE00E9404370AC9843AE1E0DC
:10CB30009E0711F40C942C6F853A914009F0D9C8E6
:10CB40000E942948FDC8853F21E0920711F40C940A
:10CB5000537068F4863EA1E09A0711F40C94E16FDB
:10CB6000843F914009F0C5C80E942FDBE9C8863F89
:10CB7000E1E09E0711F40C945770873F914009F053
:10CB8000B8C861E083E50E94023491E089270F94E0
:10CB9000D50ED6C88C3623E0920709F4D1C808F028
:10CBA000D3C08B35A2E09A0711F40C947E7068F420
:10CBB0008C30E2E09E0711F40C946D708835924041
:10CBC00009F097C80E94185BBBC88D3B22E0920712
:10CBD00011F40C94FE708E3B924009F08AC80E94BA
:10CBE0000849182F87FDACC88AE50E948D32812C38
:10CBF000912C90E2A92E91E4B92E882341F040E0D7
:10CC000050E0BA018AE50E94A8324B015C01412F35
:10CC100064E083E00E949F8720E030E0A901C50125
:10CC2000B4010F94555F18167CF580E090E0A0EAFF
:10CC3000B0E489839A83AB83BC83209151113091F6
:10CC400052114091531150915411C501B4010F94E8
:10CC5000F55C6B017C0120E030E048EC53E40F947C
:10CC6000035687FD06C0C12CD12C88ECE82E83E446
:10CC7000F82ECC8EDD8EEE8EFF8EBE016F5F7F4F65
:10CC8000CE014C960E9417F585E50E943F3288231D
:10CC900011F40C9402710E9415326B017C0120E0AA
:10CCA00030E0A901C701B6010F94555F87FF04C0AA
:10CCB000F7FAF094F7F8F094F7FAF094F7F8F094A4
:10CCC000C982DA82EB82FC8244E061E0CE01019607
:10CCD0000E94EF5820E030E0A901C501B4010F9493
:10CCE000555F18165CF580E090E0A0EAB0E4898317
:10CCF0009A83AB83BC83A50194016091511170911B
:10CD0000521180915311909154110F94F45C6B0166
:10CD10007C0120E030E0A9010F94555F18161CF04B
:10CD2000C12CD12C7601CC8EDD8EEE8EFF8EBE0115
:10CD30006F5F7F4FCE014C960E9417F51092110540
:10CD40000E94B6860C94A05E873EA3E09A0711F479
:10CD50000C947971C8F48438E3E09E0711F40C94C4
:10CD60000E71803A934011F00C94795E2091FF048B
:10CD70003091000590918517926090938517C901B5
:10CD80000F947B460C94A05E883E23E0920711F43A
:10CD90000C94A271893E934011F00C94795E0F942B
:10CDA0004B4581110C94A05E0E9417340F940945E5
:10CDB0000F94A3006D3371058105910520F081E882
:10CDC00092E10E942C728DE792E10E942C7284EE17
:10CDD0008093090589E692E10E943D3785E692E15C
:10CDE0000E942C720C94A05E60E088EB9FE00E9491
:10CDF00092B5E3CA8091F70484FD17C08091F904CD
:10CE000087FD13C08091FA04837079F460E08BECA5
:10CE10009FE00E9492B55F988A9880910801817086
:10CE20008093060112980C94A05E88E50E943F3220
:10CE300081115F9889E50E943F3281118A988AE5C5
:10CE40000E943F32882329F08091080181708093ED
:10CE5000060185E40E943F32882311F40C94A05E01
:10CE600012980C94A05E8091851783FF25C083EEF5
:10CE70009FE00E943D378091851783FF17C086EAA7
:10CE800097E10E949BD58BE1E6EAF7E1DE0111967E
:10CE900001900D928A95E1F770E060E0CE01019675
:10CEA0000F94C409CE0101960E943F3484ED9FE0A7
:10CEB0000E943D370C94A05E0E94044984EF9FE0DD
:10CEC0000E943D370C94A05E0E94FBD40C94A05E9F
:10CED0008091FF0490910005FC012191222331F003
:10CEE0002032D9F7DF0111971C92F7CF60E00F9441
:10CEF000C446109209050C94A05E83E50E948D3211
:10CF0000882321F00E94DF270E94122684E50E94D8
:10CF10008D328823A9F00E94DF276B017C010F94DA
:10CF20004A01C092C605D092C705E092C805F092AA
:10CF3000C905CD28CE28CF2819F081E080931109AA
:10CF40008091DA078823F9F080E090E0A0EAB1E46C
:10CF500089839A83AB83BC831C8E1D8E1E8E1F8E8D
:10CF600018A219A21AA21BA210E000E020E0AE0154
:10CF70004F5F5F4FBE01645E7F4FCE0180960E947F
:10CF800081570C94A05E0E948836882381F00F940C
:10CF90003B440E94AC3687E899E00F94E34310923B
:10CFA000421210924312109244121092451261E004
:10CFB0008CE29EE10E94883844EF5DE16EEF7FE0F5
:10CFC00085E00F949F300F9404460C94A05E8091EE
:10CFD000851783FD02C00C94A05E83E50E948D320C
:10CFE000882311F40C94A05E0E94DF270E94122671
:10CFF0000C94A05E83E40E943F32882361F184E1B7
:10D0000090E10E943D378091ED188823F9F0BE0130
:10D010006F5F7F4F8AEE98E10E9461D5CE01019645
:10D020000E948AD1CE0101960F94A4458091CD1320
:10D03000882339F080E20E9404378DEC93E10E944E
:10D040008AD18AE00E9404370C94A05E8AE090E1C5
:10D050000E943D37F6CF83E50E948D32882301F18F
:10D060000E94ED31182F8C3308F08CE38093D204AA
:10D070000F94CF386B017C01212F30E0A8EEB3E094
:10D080000F949B5CC60ED71EE81EF91EC092CE04FC
:10D09000D092CF04E092D004F092D1040C94A05E20
:10D0A0000F94AA430C94A05E8091FF049091000518
:10D0B0000F947B460C94A05E809185178E7F8093A1
:10D0C00085170C94A05E8091851782FD0E9456DF23
:10D0D0008091851783FD02C00C94A05E60E080E51E
:10D0E0000E940234182F682F8091FF049091000550
:10D0F0000F94C44683E50E948D32882321F00E945C
:10D10000DF270E9412260F943B4411110C94A05E5D
:10D110000E94AC360C94A05E0F94A3006C8F7D8FA0
:10D120008E8F9F8FBE016F5F7F4FCE014C960E9406
:10D13000732CCE0101960F94D2450E940449BE0182
:10D140006F5F7F4F83E290E10E941A4E8AE00E9457
:10D1500004370C94A05E80E50E943F32882311F4CE
:10D160000C94A05E0E94ED31853608F084E6809331
:10D1700009050C94A05E0E94AC360C94A05E81E080
:10D180000F94D5000C94A05E8EE890E10E943D378C
:10D1900060915B0870915C0885E890E10E94A3397A
:10D1A00060915D0870915E0888E790E10E94A33964
:10D1B00060915B0870915C0880915D0890915E08B9
:10D1C000681B790B80911109815021E030E0823099
:10D1D00010F030E020E0621B730B8DE690E10E94BE
:10D1E000A3398AE00E94043785E690E10E943D372A
:10D1F00080915F0890916008A0916108B0916208E9
:10D200008C8F9D8FAE8FBF8FBE016F5F7F4FCE0122
:10D210004C960E94732CBE016F5F7F4F88E590E1B2
:10D220000E941A4E8091630890916408A09165084D
:10D23000B09166088C8F9D8FAE8FBF8FBE016F5FE0
:10D240007F4FCE014C960E94732CBE016F5F7F4FC3
:10D2500088E490E10E941A4E20E030E04AE754E46E
:10D2600060916708709168088091690890916A08D8
:10D270000F94EF5DAB01BC0180E390E10E94B539F2
:10D280008DE60E9404378AE00E9404370C94A05E69
:10D290008091FF1083FF02C00C94A05E0E94084999
:10D2A00087FF02C00C94A05E89E40E948D3288231F
:10D2B00011F40C94BB710E94ED3190E01816190620
:10D2C00014F481E090E026E0289FF001299FF00D02
:10D2D0001124EC54F74F808191810E94D8DE61E0E7
:10D2E00080E00F94134A0F94DC490C94A05E86E909
:10D2F00090E1112309F457CA012F64CA182F62CA9A
:10D300000E940849182F87FD0AC081EB90E10E9416
:10D310003D37812F0F944F0B8AE00E94043788A974
:10D320008093FC08E1960FB6F894DEBF0FBECDBF28
:10D33000DF91CF911F910F91FF90EF90DF90CF90F1
:10D34000BF90AF909F908F907F906F905F904F9025
:10D350003F902F90089580E50F94A830823010F010
:10D360000C94A05EE82FF0E0E75CF54F10820C947F
:10D37000A05E8EE40E948D32882311F40C94A05E8E
:10D380000E94DF276093DB117093DC118093DD1125
:10D390009093DE110C94A05E83E50E943F328823B7
:10D3A00029F083E50F94A8308093FF100E94044970
:10D3B00082EC90E10E943D378091FF10882351F16B
:10D3C00010E000E020E08091FF1090E0B0E0A0E0ED
:10D3D000002E04C0B695A795979587950A94D2F725
:10D3E00080FF12C0FF24F394F20E222319F08CE286
:10D3F0000E940437F801EE0FFF1FE854FF4E85919D
:10D4000094910E943D372F2D0F5F1F4F053011055E
:10D41000D1F617CE84EB90E11BCE83E50E948D32CE
:10D42000882369F00E94ED318D3320F480930F0240
:10D430000C94A05E8CE380930F020C94A05E0E947B
:10D44000044960910F0289EC90E10E94AD398AE0B5
:10D450000E9404370C94A05E8091FF1083FF02C0ED
:10D460000C94A05E89E40E948D32882309F4ACC735
:10D470000E94ED3190E01816190614F481E090E056
:10D4800026E0289FF001299FF00D1124EC54F74F5E
:10D49000828193810E94E23161E080E00F94134A1F
:10D4A0000C94A05E8091FF1083FF02C00C94A05EDC
:10D4B00089E40E948D32882309F490C70E94ED31DF
:10D4C00090E01816190614F481E090E026E0289FF9
:10D4D000F001299FF00D1124EC54F74F82819381C4
:10D4E00010E00E94E23160E081E00F94134A209145
:10D4F0001D0930911E0980911B0990911C0982170A
:10D5000093071CF48FED90E102C080ED90E160E0A4
:10D510000E9492B560E0812F0F94C20B0C94A05E24
:10D5200083E50E948D32882311F40C94A05E0E9442
:10D53000ED31182F8C3308F08CE38093D7040F94CF
:10D54000CF386B017C01212F30E0A8EEB3E00F94BF
:10D550009B5CC60ED71EE81EF91EC092D304D09263
:10D56000D404E092D504F092D6040C94A05E0E94FC
:10D57000B8D70E9467DF81E00F94D5000E94BF36C4
:10D5800068EE73E080E090E00E9439360E948122CC
:10D5900060E08EEE90E10E9492B50C94A05E8091C6
:10D5A00012098F7D8061809312090C94A05E809196
:10D5B000F70484FD0CC08091F90487FD08C08091B8
:10D5C000FA04837021F40E9467DF0C94A05E0E942D
:10D5D00056DF88E50E943F32882331F05F9A8091C0
:10D5E0006E088E7F80936E0889E50E943F32882303
:10D5F00031F08A9A80916E088D7F80936E088AE55B
:10D600000E943F32882359F08091080180958170F3
:10D610008093060180916E088B7F80936E0885E46D
:10D620000E943F32882311F40C94A05E0E947F2256
:10D630000C94A05E83E50E943F32882311F40C9481
:10D64000A05E0F94CF386093F0087093F108809338
:10D65000F2089093F3080E94153220E030E04AE788
:10D6600054E40F9469560F94685E6093D8047093E5
:10D67000D9048093DA049093DB040C94A05E0E949A
:10D680001532F701648B758B868B978B0C943E63F8
:10D6900081E00F94322F0C94A05E0F94CD2E85ED77
:10D6A00096E10E9485DA0C94A05E8091FF0490912F
:10D6B0000005009741F0DC012C91222321F00F940A
:10D6C000D2450C94A05E0F9404460C94A05E009189
:10D6D000FF041091000594E0F12C40E09150F9F026
:10D6E000F8018081282F2B7F213499F42181213367
:10D6F000B1F4813411F1853409F441E098012E5FD1
:10D700003F4F89012F5F3F4FF80180818032C9F37D
:10D71000E5CF803521F4818180538A3078F341113F
:10D720000E940449FF2021F08DEF90E10E943D37D7
:10D73000C8010E940B370C94A05EFF24F394DECF47
:10D7400020936C0820936B080E9417FF0C94A05E36
:10D750008C01112788E40E948D328823C1F00E9439
:10D7600011328A3A91050CF44BC00E9411328D326D
:10D7700091400CF048C00E94113226E0209FF00139
:10D78000219FF00D1124EC54F74F9183808382E4A4
:10D790000E948D328823A9F00E9411320597B4F1BE
:10D7A0000E9411328D389105A4F50E94113226E0B5
:10D7B000209FF001219FF00D1124EC54F74F93832B
:10D7C000828386E40E948D32882311F40C94A05E3B
:10D7D0000E94113297FD20C00E9411328F3F9105A7
:10D7E00009F0ECF40E94113226E0209FF001219F05
:10D7F000F00D1124EC54F74F958384830C94A05EB4
:10D800008AEA90E0BACF8CE291E0B7CF85E090E071
:10D81000CECF8CE890E0CBCF90E080E0E5CF8FEFEB
:10D8200090E0E2CF80E06CC80E94084987FF02C008
:10D830000C94A05E03EA12E080E0E82E81E1F82E6D
:10D8400097EAC92E92E0D92ED8018D918D010E94C0
:10D850003F32882359F00E9415320F94685EF70119
:10D8600060837183828393830E94E4DEF4E0EF0E91
:10D87000F11CC016D10641F70C94A05E0E94084925
:10D8800087FF02C00C94A05EB3EAEB2EB2E0FB2E41
:10D8900010E000E0D7018D917D010E943F32882386
:10D8A00049F00E941532F801E050FF4E64A375A3C1
:10D8B00086A397A30C5F1F4F0031110559F70C94F5
:10D8C000A05E83E50E948D32882391F00E9415327C
:10D8D0006093341170933511809336119093371102
:10D8E00060933C1170933D1180933E1190933F11D2
:10D8F00080E50E948D32882351F00E94153260939A
:10D90000341170933511809336119093371182E55D
:10D910000E948D32882351F00E9415326093381195
:10D920007093391180933A1190933B1184E50E94D2
:10D930008D32882311F40C94A05E0E9415326093FE
:10D940003C1170933D1180933E1190933F110C94C4
:10D95000A05E0E94FF370C94A05EADE3EA2EA9E022
:10D96000FA2E10E088E5810F0E943F32882351F0A3
:10D970000E941532F7016083718382839383812F24
:10D980000E9456F31F5FF4E0EF0EF11C133051F7C5
:10D990008091F90487FF02C00C941C618091FA0405
:10D9A000837011F00C941C6140913D0950913E0927
:10D9B00060913F097091400985E391E10E94B5397A
:10D9C0004091410950914209609143097091440985
:10D9D00081E691E40E94B53940914509509146098C
:10D9E00060914709709148098EE591E40E94B5392C
:10D9F0008AE00E9404370C94A05E82E40E943F32C9
:10DA0000882341F0809176029091770290931502DD
:10DA10008093140282E50E943F32882341F0809176
:10DA2000140290911502909377028093760283E519
:10DA30000E948D32882331F00E9411329093770238
:10DA4000809376028091F7049091F804A091F904F4
:10DA5000B091FA04892B8A2B8B2B11F00C94A05EC9
:10DA600060917602709177028CE391E10E94CB3E47
:10DA700085E20E9404378AE00E9404370C94A05E7D
:10DA80000E940849082F87FF02C00C94A05E83E51E
:10DA90000E948D32002E000C110B7801EE0CFF1C41
:10DAA000882359F10E941132F701EB5CFD4F9183FD
:10DAB0008083000F111F000F111F98012F573D4F3A
:10DAC0007901BC01990F880B990B0F940A562AE033
:10DAD00037ED43E25CE30F9469560E531A4FD801B9
:10DAE0002D913D914D915C910F946956F7016083A2
:10DAF0007183828393830C94A05E0E94044985E421
:10DB00000E94043780E3800F0E940437F701EB5C2A
:10DB1000FD4F6081718180E491E10E94CB3E85E2FE
:10DB20000E9404378AE00E9404370C94A05E83E5CB
:10DB30000E948D3281110C94E7648091F90487FD75
:10DB400023C08091FA048370F9F40E940449409143
:10DB5000D7065091D8066091D9067091DA0688E40C
:10DB600091E10E94B5398AE00E9404370C94A05ECE
:10DB700060E070E080E090EC0C94016560E070E0A3
:10DB800080E090E40C94016582E50E943F328111AF
:10DB9000DCCF0C94A05E64E071E083E50E949A32D1
:10DBA0008C0168EE73E080E50E949A328938F3E1D7
:10DBB0009F0710F088E893E1B8010E944A800C9416
:10DBC000A05E85E40F94A830811174C080E50E94A6
:10DBD0003F32882351F00E9415326093841670936F
:10DBE0008516809386169093871689E40E943F32AB
:10DBF000882381F00E9415322CEA35EC47E25EE37F
:10DC00000F946956609388167093891680938A16CC
:10DC100090938B1684E40E943F32882381F00E9407
:10DC200015322CEA35EC47E25EE30F94EF5D60932A
:10DC30008C1670938D1680938E1690938F160E947B
:10DC40000449409184165091851660918616709112
:10DC500087168DE591E10E94B5392CEA35EC47E253
:10DC60005EE3609188167091891680918A16909172
:10DC70008B160F94EF5DAB01BC0189E591E10E9429
:10DC8000B5392CEA35EC47E25EE360918C16709171
:10DC90008D1680918E1690918F160F946956AB0158
:10DCA000BC0185E591E10E94B5398AE00E94043704
:10DCB0000C94A05E0E94254881E691E10E943D37C8
:10DCC0000C94A05E80E50E943F32882351F00E94B0
:10DCD0001532609320097093210980932209909353
:10DCE000230989E40E943F32882381F00E94153283
:10DCF0002CEA35EC47E25EE30F9469566093240901
:10DD000070932509809326099093270984E40E9443
:10DD10003F32882381F00E9415322CEA35EC47E22D
:10DD20005EE30F94EF5D6093280970932909809357
:10DD30002A0990932B090E9404494091200950918F
:10DD4000210960912209709123098BE791E10E94DA
:10DD5000B5392CEA35EC47E25EE360912409709115
:10DD6000250980912609909127090F94EF5DAB0159
:10DD7000BC0187E791E10E94B5392CEA35EC47E216
:10DD80005EE3609128097091290980912A09909198
:10DD90002B090F946956AB01BC0183E791E10E9406
:10DDA000B5398AE00E9404370C94A05E11110C94DE
:10DDB000A05E0E9404498BE991E10E943D37809169
:10DDC0004B0A882391F083E891E10E943D376091EE
:10DDD0008502709186028AE891E10E94CB3E86E836
:10DDE00091E10E943D370C94A05E8FE791E1EDCF69
:10DDF0000E94D7390C94A05E88E40E943F328823A9
:10DE000021F00E9401328093DC0482E50E943F32BF
:10DE1000082F83E50E943F32182F011102C088238A
:10DE200041F00E946C22112321F00E940132809364
:10DE3000550284E40E943F32882311F40C94A05EC2
:10DE40000E941532609351027093520280935302E4
:10DE5000909354020C94A05E0E941C4A0C94A05E05
:10DE60000F94264681110C94A05E77ECC72E77E2C2
:10DE7000D72E29E431E13DA32CA3CE0101961C014C
:10DE80007C0110E000E0F601659175918591949117
:10DE9000ACA1BDA18D909D90AD90BD90BDA3ACA354
:10DEA000A50194010F94F45C2B013C01F701408221
:10DEB00051826282738220E030E040EA51EC0F949C
:10DEC000555F87FD0AC020E030E040EA51E4C3011D
:10DED000B2010F940356181684F4F801EC56FF4B68
:10DEE000E4911E1654F4B7FAB094B7F8B094D70181
:10DEF0008D929D92AD92BC921397F7018190919073
:10DF0000A190B1907F0120E030E040EA51ECC501E2
:10DF1000B4010F94555F87FD3FC020E030E040EA38
:10DF200051E4C501B4010F9403561816ACF10F5F0C
:10DF30001F4FF4E0CF0ED11C0330110509F0A3CF21
:10DF40006DE3E62E69E0F62E10E0F10181919191EA
:10DF5000A191B1911F01F70181939193A193B19385
:10DF60007F01812F0E9456F31F5F133071F70E94CB
:10DF70000EFE60E08FED91E10E9492B563E972E0E0
:10DF800084E690E00E944A806AEB72E084E690E0CA
:10DF90000E944A800C94A05E0E9425488DEF91E17A
:10DFA0000E943D3761E08FEE91E10E9492B50E94A0
:10DFB000B68668E270E088EC90E00E944A800C949B
:10DFC000A05E84E50E943F328823A1F010920B05E9
:10DFD00010920C0510920D0510920E0510920F056F
:10DFE0008FEF0E94202661E070E084E50E94F33309
:10DFF00080930F0583E50E943F32882321F00E9421
:10E0000011320E94202683E40E943F32882331F09F
:10E0100080912302803210F40E94BA3480E50E947D
:10E020003F32882331F00E941132803210F40E9476
:10E03000BA3485E50E943F32882311F40C94A05E27
:10E040000E941132803210F00C94A05E41E050E04A
:10E0500060E070E0082E04C0440F551F661F771F54
:10E060000A94D2F7409550956095709500910B05F4
:10E0700010910C0520910D0530910E054023512380
:10E080006223732340930B0550930C0560930D0599
:10E0900070930E059091230289130C94A05E109248
:10E0A000FE100C94A05E0F9419160C94A05E0E94B2
:10E0B00022FF0C94A05E2093DB060F940D161092A5
:10E0C000DB06882311F40C94A05E0E9404498BE1C6
:10E0D00092E10E943D370C94A05E8091851782FFEB
:10E0E00005C08064809385170C94A05E83FD02C0F8
:10E0F0000C94A05E0F946D2F0C94A05E0E940849B2
:10E10000082F87FF02C00C94A05E85E50E943F3275
:10E11000882359F10E9415324B015C01E02E002E3C
:10E12000000CFF0820E030E0A9010F94555F87FF45
:10E1300004C0B7FAB094B7F8B09420E030E84BE3ED
:10E1400054E4C501B4010F94555F970153E0220FC9
:10E15000331F5A95E1F722533A4F1816D4F1D901DB
:10E160008D929D92AD92BC9213978CE40E943F32A7
:10E17000882311F40C94A05E0E9415326B017C017F
:10E18000002E000C110B20E030E0A9010F94555F28
:10E1900087FF04C0F7FAF094F7F8F09420E030E835
:10E1A0004BE354E4C701B6010F94555F980143E077
:10E1B000220F331F4A95E1F722533A4F18169CF06D
:10E1C000D9011496CD92DD92ED92FC9217970C94A2
:10E1D000A05E80E090E8ABE3B4E4F9018083918332
:10E1E000A283B383C2CF80E090E8ABE3B4E4F9014B
:10E1F00084839583A683B7830C94A05E0E9488567F
:10E200000C94A05E28E01202F0011124E253FA4FB0
:10E21000C080D180E280F3800C944F66A090310AD8
:10E22000B090320AC090330AD090340A8BE40E9436
:10E230008D32882339F10E9415327B018C0120E058
:10E2400030E0A9010F94555F87FD0AC020E030E05F
:10E2500040E251E4B701C8010F9403561816A4F424
:10E260008FE30E9404378BE40E94043781E392E13C
:10E270000E943D3789E292E10E943D3786E292E1B9
:10E280000E943D37750186019701A801B501C601BD
:10E290000F940356882361F00E9456DFC701D8010E
:10E2A0008093310A9093320AA093330AB093340AD0
:10E2B0008091F7049091F804A091F904B091FA04C8
:10E2C000892B8A2B8B2B11F00C94A05E0E940449A1
:10E2D0004091310A5091320A6091330A7091340AA8
:10E2E00085E492E10E94B5398AE00E9404370C94DB
:10E2F000A05E81E08093B3081092651460E083E52E
:10E300000E94023481110C94A05E0F94742D0C9421
:10E31000A05E83E50E943F32882341F00E940132D3
:10E320008093D6050E941F340C94A05E0E9404497D
:10E3300080E592E10E943D378091D6050E94973991
:10E340000C94A05E0E949E720C94A05E1091FC043E
:10E350000F94CF386093F0087093F1088093F2081F
:10E360009093F308112311F40C94A05E812F0E9466
:10E370006ED70C94A05E83E50E948D32882311F441
:10E380000C9473690E9411320C946D6983E50E94AC
:10E390008D32182F811108C082E50E948D32082F1E
:10E3A000882311F40C947E690E9411320C94BF638F
:10E3B00083E50E948D32882311F40C947C630E94C3
:10E3C000DF278B010C947C6383E50E948D328823C8
:10E3D00011F40C94A05E0E9411325CC883E50E9487
:10E3E0008D32182F811107C082E50E948D3288235B
:10E3F00011F40C94A05E0E94113273C8DF92EF9268
:10E40000FF920F931F93CF93DF93EC01E090FE08F0
:10E41000F090FF088AE0D82E6AE070E0CE010F94F9
:10E420004A608C01009711F0FC011082CE010E941D
:10E43000522D81E00E94085D0115110519F0E801D7
:10E44000D992EACFC701DF91CF911F910F91FF9031
:10E45000EF90DF900C94522D4F925F926F927F92CB
:10E460008F929F92AF92BF92CF92DF92EF92FF92E4
:10E470000F931F93CF93DF93CDB7DEB77C014DB6DB
:10E480005EB66090FE087090FF088DB69EB66AE09A
:10E4900070E0C7010F943E556C018C010E191F09E5
:10E4A000892B21F4C7010F9450558C01C8010196A6
:10E4B0002DB73EB7281B390B0FB6F8943EBF0FBEE1
:10E4C0002DBF8DB79EB701965C01A801B7010F94CF
:10E4D0007155F501E00FF11F1082C5010E94522D08
:10E4E00081E00E94085DC114D10451F076019FEFD4
:10E4F000E91AF90A0FB6F8949EBE0FBE8DBEC5CFBD
:10E500000FB6F8949EBE0FBE8DBEC3010E94522D61
:10E510000FB6F8945EBE0FBE4DBEDF91CF911F9136
:10E520000F91FF90EF90DF90CF90BF90AF909F90B2
:10E530008F907F906F905F904F9008954F925F9271
:10E540006F927F928F929F92AF92BF92CF92DF9203
:10E55000EF92FF920F931F93CF93DF93CDB7DEB768
:10E56000C059D1090FB6F894DEBF0FBECDBF0E94CF
:10E570002D34882369F083E50E943F32882301F11E
:10E5800020E040E070E060E080EE96E80E9450837A
:10E59000C057DF4F0FB6F894DEBF0FBECDBFDF917F
:10E5A000CF911F910F91FF90EF90DF90CF90BF9090
:10E5B000AF909F908F907F906F905F904F90089555
:10E5C00083E40E943F32882319F00E94D586E0CF71
:10E5D0008090F0099090F109A090F209B090F309B1
:10E5E0008091F90980FF05C09091FF109860909389
:10E5F000FF108695817080934B0A82E59FE00E9410
:10E600002C7280917F09909180099E012F5F3F4F6E
:10E610007901009799F09F938F9389E49FE09F93EE
:10E620008F933F932F930F949A55C7010E94FE71C9
:10E630000F900F900F900F900F900F9080917D0989
:10E6400090917E09009799F09F938F9380E49FE0CB
:10E650009F938F93FF92EF920F949A55C7010E9458
:10E66000FE710F900F900F900F900F900F906E0112
:10E6700031E8C30ED11C60915C0970915D098091F5
:10E680005E0990915F09860123E041E00F94D0502C
:10E690009F938F938EE29FE09F938F93FF92EF92D1
:10E6A0000F949A55C7010E94FE7186E29FE00E9476
:10E6B0002C7287E080936E088093B9050F900F90BD
:10E6C0000F900F900F900F90809178098823F9F0A8
:10E6D0006091790970917A0980917B0990917C0908
:10E6E00023E041E00F94D0509F938F938DE19FE002
:10E6F0009F938F93FF92EF920F949A55C7010E94B8
:10E70000FE710F900F900F900F900F900F908091CF
:10E7100081098823A1F01F928F931F921F9280E19D
:10E720009FE09F938F93FF92EF920F949A55C701AA
:10E730000E94FE710FB6F894DEBF0FBECDBF809170
:10E7400082098823A9F01F928F931F9281E08F93F3
:10E7500080E19FE09F938F93FF92EF920F949A55E1
:10E76000C7010E94FE710FB6F894DEBF0FBECDBF89
:10E7700040908309509084096090850970908609C3
:10E7800020E030E0A901C301B2010F9403568111CA
:10E7900004C08091F90982FF20C0860121E041E098
:10E7A000C301B2010F94D0509F938F938091F909C8
:10E7B00082FB882780F91F928F9383E09FE09F93CD
:10E7C0008F93FF92EF920F949A55C7010E94FE71AA
:10E7D0000FB6F894DEBF0FBECDBF60914E097091A9
:10E7E0004F0980915009909151098E010F581F4F88
:10E7F00023E041E00F94D050782E692E60914A09B1
:10E8000070914B0980914C0990914D09860123E04C
:10E8100041E00F94D0506F927F929F938F9382EF3D
:10E820009EE09F938F93FF92EF920F949A55C701AA
:10E830000E94FE71609152097091530980915409B0
:10E840009091550923E041E00F94D05087EE9EE06F
:10E850000E942C72DF92CF928DED9EE09F938F935A
:10E86000FF92EF920F949A55C7010E94FE7180911A
:10E870005B098F9380915A098F9386ED9EE09F9359
:10E880008F93FF92EF920F949A55C7010E94FE71E9
:10E8900060915609709157098091580990915909D2
:10E8A00023E041E00F94D0509F938F938CEC9EE037
:10E8B0009F938F93FF92EF920F949A55C7010E94F6
:10E8C000FE718CE0E0E6F9E0ADE3B9E001900D9275
:10E8D0008A95E1F78CE0ECE6F9E0A1E3B9E001907C
:10E8E0000D928A95E1F780E00E9456F381E00E9444
:10E8F00056F382E00E9456F38091F8098093120942
:10E9000081E08093D6050E941F3487E899E09F93A9
:10E910008F938CE098E39F938F93FF92EF920F94E5
:10E920009A550FB6F894DEBF0FBECDBFC7010E9447
:10E93000FE718091F7098F938091F6098F938091F2
:10E94000F5098F938091F4098F93BF92AF929F92B4
:10E950008F928EEB9EE09F938F93FF92EF920F9496
:10E960009A55C7010E94FE710FB6F894DEBF0FBE24
:10E97000CDBF0ECE4F925F926F927F928F929F92F9
:10E98000AF92BF92CF92DF92EF92FF920F931F93BD
:10E99000CF93DF9300D000D01F921F92CDB7DEB788
:10E9A00083E50F94A830863028F083E19EE00E9432
:10E9B0003D373FC0833009F478C1B0F4813021F194
:10E9C000823009F450C080E09EE00E943D370E94F2
:10E9D000F4358823A1F0809148110E9497390E9454
:10E9E00018390E940EFE25C0843009F4A4C1853078
:10E9F00051F780E00E94F9340E94E634F2CF82EFB2
:10EA00009DE00E943D37EDCF0E94E63410920E0249
:10EA100010920D0280910A05811125C08EE40E949A
:10EA20003F3281111DC080EE9DE09093710880936C
:10EA3000700828960FB6F894DEBF0FBECDBFDF91E9
:10EA4000CF911F910F91FF90EF90DF90CF90BF90EB
:10EA5000AF909F908F907F906F905F904F900895B0
:10EA600086EE9DE0E2CF80910D0290910E0297FF1D
:10EA700003C087EB9DE09BCF009709F0B3C01D82D8
:10EA80001E821F8218868DEC9CECACE4BEE3898369
:10EA90009A83AB83BC83BE016B5F7F4FCE0101962F
:10EAA0000E9417F520910D0230910E02203431059D
:10EAB0000CF0C7C081E080933802C90101969093A1
:10EAC0000E0280930D02822F877887FF03C081504A
:10EAD000886F8F5FA82FE22F27FF02C0E7E0E20FC9
:10EAE000E595E595E595E0FF02C0A7E0A81B84E069
:10EAF000A802D0011124A65AB84E8D909D90AD90D9
:10EB0000BC9094E0E902F0011124E65CF84E4080EC
:10EB10005180628073808DEC9CECACE4BEE38D830D
:10EB20009E83AF83B88719821A821B821C82CE0112
:10EB300001966C01E12CF12C00EA10E4A301920192
:10EB4000C501B4010E945FF419821A821B821C82E3
:10EB5000B601CE0105960E9417F580924911909258
:10EB60004A11A0924B11B0924C1140924D1150920B
:10EB70004E1160924F117092501110920A0500913F
:10EB80000D0210910E0280E4E82EF12C00341105E4
:10EB90000CF47801B70180E59DE00E94CB3E60E473
:10EBA00070E08BE49DE00E94CB3E8AE00E94043737
:10EBB000101611060CF015CF1F9280E48F93FF9270
:10EBC000EF9284E39DE09F938F9382E49DE09F9377
:10EBD0008F931F920E9477B50FB6F894DEBF0FBED9
:10EBE000CDBFFFCE8150982F977897FF03C09150EB
:10EBF000986F9F5FE92F87FD895F8595859585953E
:10EC000080FF02C0E7E0E91B28E0E202F0011124E6
:10EC1000E80FF11D87FDFA95EE0FFF1FEE0FFF1FA6
:10EC2000E952FA4F8091511190915211A0915311D4
:10EC3000B091541180839183A283B38310923802E0
:10EC400031CF80E090E0A0EAB0E48093511190933E
:10EC50005211A0935311B09354118CE792E00E948B
:10EC600044F40E9456DF8FEF9FEF90930E02809343
:10EC70000D0283EA9DE00E943D3781E99DE00F94FB
:10EC8000D24563E972E084E690E00E944A806AEB34
:10EC900072E084E690E00E944A808BE89DE00E944A
:10ECA0002C7281E00E94F93468CF89E40E948D3291
:10ECB000882371F00E941132182F883068F067E0C5
:10ECC00070E088E79DE00E94CB3E85E79DE06FCE37
:10ECD0008AE40E948238ADCE8AE40E948D32882375
:10ECE000B9F30E941132082F883048F067E070E0D5
:10ECF00082E69DE00E94CB3E8FE59DE058CE8AE5FE
:10ED00000E948D328823A9F00E94153228E0120259
:10ED1000F0011124E00FF11D07FDFA95EE0FFF1F22
:10ED2000EE0FFF1FE952FA4F608371838283938352
:10ED300058CE8AE5CECF8AE50E948D328823C9F36A
:10ED40000E9415326093D7067093D8068093D90637
:10ED50009093DA0646CECF93DF93C0914712C093CB
:10ED60000C0A81E6C89FE0011124C75BDD4E80914B
:10ED7000FF1080FF05C00E940449CE010E940B379E
:10ED8000CE010E94522D80E0DF91CF910C94085D5E
:10ED90008F929F92AF92BF92CF92DF92EF92FF92AB
:10EDA000CF936B017C0120E030E0A9010F94035662
:10EDB00087FFA3C06DEB77E386E095EBA701960193
:10EDC0000F94F55C6B017C0120E030E040E251E4FF
:10EDD0000F94695620E030E048EC52E40F946956F5
:10EDE0004B015C0120E030E040E251ECC701B6018C
:10EDF0000F940356181654F420E030E048EC52E427
:10EE0000C701B6010F94555F87FD8BC020E030E04D
:10EE1000A901C701B6010F94035687FF73C060E0D4
:10EE200070E080EA90ECA50194010F94F55C20E07D
:10EE300030E040E251E40F94EF5D0F94615E6B01AE
:10EE40007C01F7FC64C020E137E240E050E00F9421
:10EE5000695CCA01B9012AE030E040E050E00F945B
:10EE6000695C605D6093B205C701B60128EE33E0CE
:10EE700040E050E00F94695C9AE0892E912CA12C1F
:10EE8000B12CCA01B901A50194010F94695C605DC0
:10EE90006093B305C701B60124E630E040E050E0DE
:10EEA0000F94695CCA01B901A50194010F94695CD2
:10EEB000605D6093B4058EE28093B505C701B6012D
:10EEC000A50194010F94695CC62FCA01B901A5017F
:10EED00094010F94695C605D6093B605C05DC0935A
:10EEE000B70582EB95E0CF91FF90EF90DF90CF9048
:10EEF000BF90AF909F908F9008956DEB77E386E081
:10EF000095E35CCF60E070E080EA90E48CCFF09411
:10EF1000E094D094C094C11CD11CE11CF11C6DE2A2
:10EF2000A1CF20E030E0A901C701B6010F9403563C
:10EF300087FF6AC060E070E080EA90ECA501940170
:10EF40000F94F55C20E030E040E251E40F94EF5D77
:10EF50000F94615E4B015C0120E030E0A901C70124
:10EF6000B6010F94555F87FD0BC020E030E040E212
:10EF700051E4C701B6010F94035660E287FD13C048
:10EF8000B7FC47C0C501B40128EE33E040E050E0D3
:10EF90000F94695CCA01B9012AE030E040E050E01A
:10EFA0000F94695C605D6093B305C501B40124E60C
:10EFB00030E040E050E00F94695C8AE0C82ED12C2C
:10EFC000E12CF12CCA01B901A70196010F94695CEB
:10EFD000605D6093B4058EE28093B505C501B40110
:10EFE000A70196010F94695CC62FCA01B901A70158
:10EFF00096010F94695C605D6093B605C05DC09337
:10F00000B70583EB95E06FCF60E070E080EA90E4B5
:10F0100095CFB094A09490948094811C911CA11CD5
:10F02000B11C6DE2C0CF6091350270913602072E9F
:10F03000000C880B990B0F940A562AE037ED43E237
:10F040005CE30F9469562091C2053091C30540914D
:10F05000C4055091C5050F94695660938102709361
:10F06000820280938302909384020895E091DB08EA
:10F07000E23030F4F0E0E75CF54F8091D108808316
:10F08000089580917A178823C1F0815080937A1770
:10F09000E6EAF7E1882351F08150990B2BE1289F94
:10F0A000F001299FF00D1124E452F84E8BE1A1EC00
:10F0B000B7E101900D928A95E1F720917A1721111D
:10F0C00005C08091851780628093851781E090E06C
:10F0D000A0E0B0E0211103C080E090E0DC0180936B
:10F0E000C9089093CA08A093CB08B093CC0810929B
:10F0F000CE0881E08093C80883E080938002089561
:10F10000CF93DF93EC01CB01BA010F940A5629EC9F
:10F1100038EC48EC5EE30F94EF5D20E030E040E037
:10F120005FE30F94F55C0F94685E6883DF91CF9185
:10F130000895E091DB0886E0E802F0011124EC5428
:10F14000F74F8091D10890E0958384830895CF9301
:10F15000DF93EC01CB01BA010F940A5620E030E0B6
:10F16000A9010F94F55C0F94685E6883DF91CF91DD
:10F1700008958F929F92AF92BF92CF92DF92EF92BB
:10F18000FF92CF936B017C0120E030E0A9010F9446
:10F19000035687FD9FC06DEB77E386E095E3A701FB
:10F1A00096010F94F55C6B017C0120E030E040E2B9
:10F1B00051E40F94695620E030E048EC52E40F949B
:10F1C00069564B015C0120E030E0A901C701B6019E
:10F1D0000F94035620E030E040EA50E487FF04C07B
:10F1E00020E030E040EA50ECC501B4010F94F55C3A
:10F1F00020E030E040E251E40F94EF5D0F94615E57
:10F200006B017C018BE2F7FE09C0F094E094D0948E
:10F21000C094C11CD11CE11CF11C8DE28093B1058E
:10F22000C701B60120E137E240E050E00F94695C8D
:10F230008AE0882E912CA12CB12CCA01B901A5011C
:10F2400094010F94695C605D6093B205C701B601DB
:10F2500028EE33E040E050E00F94695CCA01B90148
:10F26000A50194010F94695C605D6093B305C701CB
:10F27000B60124E630E040E050E00F94695CCA013A
:10F28000B901A50194010F94695C605D6093B405B8
:10F290008EE28093B505C701B601A50194010F94D4
:10F2A000695CC62FCA01B901A50194010F94695C7C
:10F2B000605D6093B605C05DC093B70581EB95E0D6
:10F2C000CF91FF90EF90DF90CF90BF90AF909F9045
:10F2D0008F9008956DEB77E386E095EB60CF8F928A
:10F2E0009F92AF92BF92CF92DF92EF92FF92CF9315
:10F2F0006B017C0120E030E0A9010F94035687FDEB
:10F30000AAC06DEB77E386E095E3A70196010F9421
:10F31000F55C6B017C0120E030E0A9010F940356FD
:10F3200087FF9EC0C701B601905820E030E040E260
:10F3300051E40F94695620E030E040E251E40F942C
:10F34000695620E030E040EA50E40F94F55C20E09C
:10F3500030E040E251E40F94EF5D0F94615E6B0189
:10F360007C0180E28093B10560E280E1C81687E20B
:10F37000D806E104F1048CF0C701B60120E137E2C0
:10F3800040E050E00F94695CCA01B9012AE030E026
:10F3900040E050E00F94695C605D6093B20560E20C
:10F3A00088EEC81683E0D806E104F1048CF0C701AA
:10F3B000B60128EE33E040E050E00F94695CCA01EA
:10F3C000B9012AE030E040E050E00F94695C605DF4
:10F3D0006093B30560E284E6C816D104E104F10449
:10F3E0008CF0C701B60124E630E040E050E00F9415
:10F3F000695CCA01B9012AE030E040E050E00F94B6
:10F40000695C605D6093B4058AE0882E912CA12C24
:10F41000B12CC701B601A50194010F94695CC62FF8
:10F42000CA01B901A50194010F94695C605D609304
:10F43000B5058EE28093B605C05DC093B70581EB3C
:10F4400095E0CF91FF90EF90DF90CF90BF90AF907D
:10F450009F908F9008956DEB77E386E095EB55CF05
:10F4600020E030E040E251E4C701B60162CFCF9323
:10F47000DF93EC01CB01BA010F940A5620E030E093
:10F4800040E251E40F94EF5D20E030E0A9010F94D9
:10F49000F55C688379838A839B83DF91CF9108959C
:10F4A000CF93DF93EC01CB01BA010F940A5620E011
:10F4B00030E040E251E40F94EF5D20E030E0A9013C
:10F4C0000F94F55C688379838A839B83DF91CF9166
:10F4D00008950F940A5620E030E040E251E40F9482
:10F4E000EF5D20E030E0A9010F94F55C0C946F799A
:10F4F000CF93DF93EC01CB01BA010F940A562AE0B7
:10F5000037ED43E25DE30F94EF5D20E030E0A901C9
:10F510000F94F55C0F94685E688379838A839B837C
:10F52000DF91CF910895CF93DF93EC01CB01BA0126
:10F530000F940A562AE037ED43E25DE30F94EF5D46
:10F5400020E030E0A9010F94F55C688379838A8319
:10F550009B83DF91CF910895CF93DF93EC01CB0193
:10F56000BA010F940A5620E030E0A9010F94F55C2F
:10F57000688379838A839B83DF91CF910895CF93AA
:10F58000DF93EC01CB01BA010F940A5620E030E082
:10F59000A9010F94F55C688379838A839B83DF914B
:10F5A000CF910895CF93DF93EC01CB01BA010F9473
:10F5B0000A5620E030E048EC52E40F94EF5D20E082
:10F5C00030E0A9010F94F55C688379838A839B837B
:10F5D000DF91CF910895CF93DF93EC01CB01BA0176
:10F5E0000F940A5620E030E048EC52E40F94EF5DAF
:10F5F00020E030E0A9010F94F55C688379838A8369
:10F600009B83DF91CF9108950F940A5620E030E05C
:10F6100048EC52E40F94EF5D20E030E0A9010F9434
:10F62000F55C0C94B978CF93DF93EC01CB01BA0170
:10F630000F940A5620E030E0A9010F94F55C0F9476
:10F64000615E79836883DF91CF910895CF93DF93D3
:10F65000EC01CB01BA010F940A5620E030E0A90179
:10F660000F94F55C688379838A839B83DF91CF91C4
:10F670000895CF93DF93EC01CB01BA010F940A56A2
:10F6800020E030E04AE754E40F94EF5D20E030E002
:10F69000A9010F94F55C688379838A839B83DF914A
:10F6A000CF9108950F940A5620E030E048EC52E4E0
:10F6B0000F94EF5D20E030E0A9010F94F55C0C940D
:10F6C000C8762CEA35EC47E25EE360919F057091C5
:10F6D000A0058091A1059091A2050F94EF5D609324
:10F6E0008C1670938D1680938E1690938F160895B6
:10F6F0002CEA35EC47E25EE36091A3057091A40526
:10F700008091A5059091A6050F946956609388167F
:10F710007093891680938A1690938B1608952CEA1D
:10F7200035EC47E25EE360919F057091A005809102
:10F73000A1059091A2050F94EF5D60938C167093D4
:10F740008D1680938E1690938F1608952CEA35ECC3
:10F7500047E25EE36091A3057091A4058091A50541
:10F760009091A6050F946956609388167093891638
:10F7700080938A1690938B1608958091D10890916A
:10F78000D208A091D308B091D408809351029093ED
:10F790005202A0935302B09354020895E091980549
:10F7A000E63010F581E08E0F809398054091C908EE
:10F7B0005091CA086091CB087091CC089091CE0806
:10F7C0008091C70828E0E29FF0011124E75AFA4F20
:10F7D0002091F9163091FA163183208342835383A6
:10F7E00064837583968387830895FC01A081B1812A
:10F7F0001C92A281B3818C918F5F8C930280F381E4
:10F80000E02D90818CE0989F800D1124EBEFF6E1C4
:10F8100013AE84AF0895CF92DF92EF92FF92CF9311
:10F82000DF9300D01F92CDB7DEB76B017C0120E0E3
:10F8300030E0A9010F94035687FD1CC06DEB77E300
:10F8400086E095E3A70196010F94F55C69837A83BE
:10F850008B839C8360E2CE0101960F9435020F905A
:10F860000F900F900F90DF91CF91FF90EF90DF906E
:10F87000CF9008956DEB77E386E095EBE3CF0F949F
:10F880000A5620E030E04AE754E40F94EF5D20E0B0
:10F8900030E0A9010F94F55C0C940B7CCF92DF92C1
:10F8A000EF92FF926B017C0120E030E0A9010F9400
:10F8B000035687FD26C06DEB77E386E095E3A7014D
:10F8C00096010F94F55C6B017C0120E030E0A9010A
:10F8D0000F94035620E030E040E05FE387FF04C070
:10F8E00020E030E040E05FEBC701B6010F94F55C2B
:10F8F0000F94615ECB01FF90EF90DF90CF900D945D
:10F90000F7036DEB77E386E095EBD9CF0F940A56BA
:10F9100020E030E0A9010F94F55C0C944E7C0F942C
:10F920000A5620E030E0A9010F94F55C0F94615E67
:10F93000CB010D94F7030F940A5629EC38EC48ECF0
:10F940005EE30F94EF5D20E030E040E05FE30F9472
:10F95000F55C0F94685E862F0D944E040D94DB3891
:10F960000D94DB386FEF8091D1080D94F9366AE37E
:10F9700075EB82E00D94B8476FE375EB81E00D9471
:10F98000B84764E475EB80E00D94B84765EF72EB1F
:10F9900083E00D94B847CF92DF92EF92FF92CF931E
:10F9A000DF9300D01F92CDB7DEB76B017C0120E062
:10F9B00030E0A9010F94035687FD1BC06DEB77E380
:10F9C00086E095E3A70196010F94F55C69837A833D
:10F9D0008B839C83CE0101960F94D1020F900F90E0
:10F9E0000F900F90DF91CF91FF90EF90DF90CF902D
:10F9F00008956DEB77E386E095EBE4CF0F940A561C
:10FA000020E030E040E251E40F94EF5D20E030E090
:10FA1000A9010F94F55C0C94CB7C8091C316909156
:10FA2000C416891B8F7011F40C945D3681E0089523
:10FA300080918002882351F060919D0570919E0510
:10FA400030E020E041E081E00C94B32A089584E0A6
:10FA50000D94CC3583E00D94CC3582E00D94CC35FB
:10FA60000F940A5620E030E0A9010F94F55C0F9442
:10FA7000685E862F0D942C049091481181E08927AF
:10FA80000C94F93461E081ED98E00C9414350F94F6
:10FA9000B52D0C9466F580E090E0A0E8B0E480938A
:10FAA000511190935211A0935311B09354118FEDB3
:10FAB00092E00E9444F4E091A80580E090E0A8E480
:10FAC000B3E4E43009F44AC080E090E0A0EBB1E494
:10FAD0008093491190934A11A0934B11B0934C110C
:10FAE00080934D1190934E11A0934F11B0935011EC
:10FAF000EE0FFF0BE154FD4F808191818330910522
:10FB000049F184309105D9F1029761F480E090E0E9
:10FB1000ADEBB3E48093491190934A11A0934B113C
:10FB2000B0934C1187EC92E00E9444F41092511172
:10FB30001092521110925311109254118FED92E0C5
:10FB40000E9444F48091A8058F5F8530ECF4809387
:10FB5000A805089580E090E0ADEBB3E480934911EF
:10FB600090934A11A0934B11B0934C1180934D1177
:10FB700090934E11A0934F11B0935011D3CF80E0CA
:10FB800090E0ADEBB3E4F2CF1092A8050895CF93C7
:10FB9000DF9300D01F92CDB7DEB70F94685E0F944D
:10FBA000085669837A838B839C83CE0101960F94D8
:10FBB000B2010F900F900F900F90DF91CF910895A9
:10FBC0000F940A562AE037ED43E25DE30F94EF5DB0
:10FBD00020E030E0A9010F94F55C0C94C77DCF9232
:10FBE000DF92EF92FF92CF93DF9300D01F92CDB7B9
:10FBF000DEB76B017C0120E030E0A9010F940356D1
:10FC000087FD1BC06DEB77E386E095E3A7019601C6
:10FC10000F94F55C69837A838B839C83CE01019674
:10FC20000F94B2010F900F900F900F90DF91CF9132
:10FC3000FF90EF90DF90CF9008956DEB77E386E033
:10FC400095EBE4CF0F940A562AE037ED43E25DE3EB
:10FC50000F94EF5D20E030E0A9010F94F55C0C9467
:10FC6000EF7D0F940A5620E030E0A9010F94F55C77
:10FC70000C94EF7DCF92DF92EF92FF926B017C01AB
:10FC800020E030E0A9010F94035687FD26C06DEBFC
:10FC900077E386E095E3A70196010F94F55C6B018D
:10FCA0007C0120E030E0A9010F94035620E030E011
:10FCB00040E05FE387FF04C020E030E040E05FEB1E
:10FCC000C701B6010F94F55C0F94615ECB01FF9004
:10FCD000EF90DF90CF900D944D036DEB77E386E0CE
:10FCE00095EBD9CF0F940A5620E030E0A9010F948C
:10FCF000F55C0C943A7E0C9432DF0C9432DF0C9459
:10FD000032DF0C9432DF0C94E4DE0C94E4DE0C94CD
:10FD1000E4DE0C94E4DECF92DF92EF92FF92CF9379
:10FD2000C82F0F94CF386B017C0124EA30E74DE7F0
:10FD30005FE36091250270912602809127029091E5
:10FD400028020F94035687FD18C08AEF90E0A0E0C8
:10FD5000B0E08C0D9D1DAE1DBF1D8093430590939B
:10FD60004405A0934505B0934605C0931E02CF916C
:10FD7000FF90EF90DF90CF90089580E090E0DC015D
:10FD8000E8CFCF92DF92EF92FF920F931F930F94E1
:10FD9000CF3800911405109115052091160530916A
:10FDA00017056B017C01C01AD10AE20AF30A970118
:10FDB000860137FD11C0209113052095209313056E
:10FDC0006A547C4F8F4F9F4F6093140570931505B5
:10FDD000809316059093170581E09091130591117A
:10FDE00001C080E01F910F91FF90EF90DF90CF90C6
:10FDF00008950F9404461092FB08109274020E941A
:10FE00008836882351F08091851782FD06C083E3F0
:10FE10009EE1909371088093700861E08CE29EE10E
:10FE20000E9488380D9465014F925F926F927F9285
:10FE30008F929F92BF92CF92DF92EF92FF920F9399
:10FE40001F93CF93DF9300D000D01F921F92CDB7A6
:10FE5000DEB77C016A014901FB0190818CE0989F2B
:10FE6000800D1124982FF7012081822F880F820F97
:10FE7000880F80933617909337174115510571F10C
:10FE8000FA82E9827C836B83011121C0AE014B5F52
:10FE90005F4FB401C6010E94EF276C016D817E8126
:10FEA0008F8198856115710581059105B9F00E94D2
:10FEB0005029F70180818F5F8083853138F3CE012F
:10FEC00001960E94F57BE2CFB12C860129C08A0100
:10FED000B12C26C0452846284728B1F728960FB6EA
:10FEE000F894DEBF0FBECDBFDF91CF911F910F9170
:10FEF000FF90EF90DF90CF90BF909F908F907F907A
:10FF00006F905F904F900895B39407C0B1102EC0CA
:10FF100001151105C9F20F5F1F4F01151105A9F257
:10FF2000AE014B5F5F4FB401C6010E94EF276C0129
:10FF30004D805E806F8078844114510461047104A7
:10FF4000A9F0F0E24F16510461047104F9F2D301F3
:10FF5000C2018D97A109B1090297A105B10530F041
:10FF60004BE2441651046104710471F6F70180817B
:10FF7000482F4B0D5527551F4631510534F085301C
:10FF800020F0CE0101960E94F57B81E041145104DE
:10FF90006104710409F480E0B80EF70180818B0DD3
:10FFA0008083BB2009F496CFBA94AE014B5F5F4FBC
:10FFB000B401C8010E94EF278C016D817E818F8181
:10FFC00098850E945029EDCFEF92FF920F931F93D7
:10FFD000CF93DF9300D000D000D01F921F92CDB7F7
:10FFE000DEB77C012091CF08422F022E000C550B6A
:10FFF0008091D008833099F1843051F18CEC91E2FA
:020000021000EC
:100000005F932F939F938F938E010F5F1F4F1F93CB
:100010000F930F949A55C7010E94D8DE4FE350E02A
:10002000B80182E798E00F946A600F900F900F90EC
:100030000F900F900F902B960FB6F894DEBF0FBE67
:10004000CDBFDF91CF911F910F91FF90EF90089559
:1000500088ED91E227FDD4CF83EC91E2D1CF81EE00
:1000600091E2CECFE091DB0885E1E802F0011124B6
:10007000E558F94E868197810C94E47FE091DB0886
:1000800086E0E802F0011124EC54F74F8081918161
:100090000C94E47F0F931F93CF93DF938C01EB01BC
:1000A0009091E7162091E816921305C00F9434053D
:1000B0000E9468F5F5CF8091E61634E0839FF00149
:1000C0001124E751F94E11830083D383C2839F5FCC
:1000D0009093E7168F5F281739F08093E616DF912B
:1000E000CF911F910F9108951092E616F8CF63E912
:1000F00072E084E690E00E944A806AEB72E084E657
:1001000090E00C944A8081110C94778068EB71E048
:1001100084E190E00C944A800E942FDB0C94838051
:100120000F9419160C9483800E9422FF0C94778000
:10013000CF93DF93CDB7DEB720E2488559856F8135
:100140008E810F945C32DF91CF910895282F109209
:10015000D9088091C9089091CA08A091CB08B091A4
:10016000CC08B7FF08C01092C9081092CA081092B4
:10017000CB081092CC088091B005882331F0809193
:10018000C9088093CD081092C8088091C708181636
:10019000FCF4082E000C990B821B91092091CD08CC
:1001A000022E000C330B2817390794F097FF02C07A
:1001B00090E080E08093CD08092E000CAA0BBB0BC9
:1001C0008093C9089093CA08A093CB08B093CC0839
:1001D0008091CD086623A9F09091CE08891714F478
:1001E0008093CE082091CE08022E000C330B2C5F9A
:1001F0003F4F482F082E000C550B241735071CF4D1
:1002000084508093CE0808955F926F927F928F9270
:100210009F92AF92BF92CF92DF92EF92FF920F9395
:100220001F93CF93DF9361E081E00E94A680C0918D
:10023000CE0885E0982E9C0ED1E096E1E92E92E260
:10024000F92E882483947D2E7C1A6C2E619421E2F1
:10025000C22E22E2D22E12E01C1B33E0532E4CE6BB
:10026000A42E42E2B42EC11141C0DD23D9F0809109
:10027000CD081816BCF04091C9085091CA08609189
:10028000CB087091CC084F5F5F4F6F4F7F4F40930B
:10029000C9085093CA086093CB087093CC088F5F4D
:1002A0008093CD0880918002882341F030E020E0E7
:1002B00041E06AE272E2862D0E94B32A8091F90839
:1002C000882309F487C0C23051F48091CD08823070
:1002D00009F445C08091800281115AC0D0E0CF5FFF
:1002E0009C12C1CF83E08093C70818C0C13031F79A
:1002F0009091CD08913031F08091800281111EC023
:10030000D0E0DCCF8091C6081092C6088823A1F304
:10031000C093FA088091C808882371F3DF91CF91C8
:100320001F910F91FF90EF90DF90CF90BF90AF9013
:100330009F908F907F906F905F9008951F92FF9293
:10034000EF927F9281E0913009F080E08F930E94DC
:1003500098800F900F900F900F900F90D1CF8091B9
:10036000C6081092C608882309F4B4CF80915502BC
:1003700088258093550250928002A114B10411F097
:100380000E946C228091C808882309F4A3CFC6CFAD
:1003900081E09091CD08923009F080E09091550273
:1003A00025E032E2911102C021E032E201E048E0B2
:1003B00052E2612F0E94AE2B91CF8091C60810921D
:1003C000C608882371F0C093FA088091C808882372
:1003D00041F0A4CFC23009F082CF9091CD08923085
:1003E00061F380918002882309F478CF1F92DF9215
:1003F000CF921F9381E0923009F080E08F930E94AA
:1004000098800F900F900F900F900F9067CF2F92C2
:100410003F924F925F926F927F928F929F92AF9294
:10042000BF92CF92DF92EF92FF920F931F93CF93E1
:10043000DF934C010F94505501968401080F191F4A
:10044000C8010F94505501966801C80ED91EF801D5
:100450006080C1E0611001C0C0E0F6013080D1E0F1
:10046000311001C0D0E0AA24A3946110A12C60E057
:1004700085E00E94A6805090CE08752C9EE0E92E63
:10048000F12C252C21948A2D90E001965C01AC0E74
:10049000B11CAD0EB11C71101DC08091800288236B
:1004A000A1F0E0912402E2506AE372E2E33038F412
:1004B000F0E0EE0FFF1FE951FD4F6081718130E0E8
:1004C00020E043E0822D0E94B32AD1E0611013C0E6
:1004D000D2E011C0D2E06110D1E0D7110CC0809100
:1004E0008002882341F030E020E041E0B4018D2F0C
:1004F00085190E94B32AC1E0CD0F472C451866200C
:1005000079F0C7110BC080918002882339F030E068
:1005100020E041E0B801842D0E94B32AC2E0CD0F53
:10052000332071F0C7110BC080918002882339F00D
:1005300030E020E041E0B601842D0E94B32ACF5F75
:10054000F3E0AF16B1040CF4CF5FC71162C0809125
:100550008002882309F45AC030E020E042E067E4DA
:1005600072E2842D0E94B32AD091110593EF9E0D63
:10057000909310058EEF8E0D8093DA08209133173B
:100580002E151F0411F00CF041C020913517921761
:10059000E8F59EE3909336178093371765E470E093
:1005A00080E090E00E94502961E36D0F062E000C60
:1005B000770B880B990B0E94502960E270E080E075
:1005C00090E00E94502980917F16909180160F94A0
:1005D000F7030E942B2B6FE270E080E090E00E9416
:1005E00050290E94C17E811109C085E08D9FF001D4
:1005F0001124E651F94F8481811108C08091811640
:10060000909182160F94F7030E942B2B92E0909307
:100610008002ECE0EE0EF11C7394FAE4EF16F104A4
:1006200009F039CFCF5FC093C708DF91CF911F91F9
:100630000F91FF90EF90DF90CF90BF90AF909F9081
:100640008F907F906F905F904F903F902F90089584
:1006500082E592E20C9407828FE592E20C94078285
:1006600081E892E20C9407828CE193E20C94078279
:1006700087ED92E20C94078284E093E20C94078267
:1006800087E593E20C9407828AE393E20C94078255
:100690008AEB92E20C9407828BE992E20C94078237
:1006A0008F929F92AF92BF92EF92FF920F931F9300
:1006B000CF93DF93EC018B01E42EF22E8091F9169B
:1006C0009091FA168C179D0709F43EC020910905F8
:1006D00027FD1092090526EBC031D20709F03FC073
:1006E00084529F4B71F40F94CF386E517B4F8F4FD4
:1006F0009F4F6093990570939A0580939B05909303
:100700009C05D093FA16C093F91630E020E00093D0
:10071000C9081093CA082093CB083093CC08E09204
:10072000CE08F092C708C452DF4B21F41092120594
:100730001092980582E08093800281E08093C8083F
:100740001092AD051092A705DF91CF911F910F91E7
:10075000FF90EF90BF90AF909F908F9008952FEBF8
:10076000C432D20771F68051964B19F0C4E2DFEB28
:10077000C8CF0F94CF388090990590909A05A0909B
:100780009B05B0909C05681979098A099B0997FF18
:10079000EDCF80916E088770873041F7CFEDD3E8B9
:1007A000B0CFCF93DF93EC010E94CE7B20E040E0FE
:1007B00070E060E0CE01DF91CF910C94508320E097
:1007C00040E070E060E08EEF91EB0E94508381E0AA
:1007D000809312051092F7081092F608089520E011
:1007E00040E070E060E086EC9CE70C9450838091E0
:1007F0004B0A811114C08091850290918602019765
:1008000020917F16309180162817390744F420E094
:1008100040E070E060E089E09EEB0C9450830C9423
:10082000EF8321E020931205FC0180819181A28158
:10083000B3818093250290932602A0932702B09360
:10084000280220E040E070E060E08091C4089091D0
:10085000C5080C945083CF93DF9300D01F92CDB77F
:10086000DEB78DEC9CECACECBCE389839A83AB8364
:10087000BC83CE0101960E9411840F900F900F90BF
:100880000F90DF91CF910895CF93DF9300D01F9207
:10089000CDB7DEB78DEC9CECACECBDE389839A83DD
:1008A000AB83BC83CE0101960E9411840F900F9000
:1008B0000F900F90DF91CF910895CF93DF9300D0E9
:1008C0001F92CDB7DEB780E090E0A0E8BFE3898358
:1008D0009A83AB83BC83CE0101960E9411840F9052
:1008E0000F900F900F90DF91CF910895CF93DF93EA
:1008F00000D01F92CDB7DEB780E090E0A0E2B1E477
:1009000089839A83AB83BC83CE0101960E941184B4
:100910000F900F900F900F90DF91CF9108958FEF70
:100920008093D10820E040E070E060E085E299E942
:100930000C94508381E08093120510926E081092FF
:10094000B90520E040E070E060E081ED94E80E94AD
:10095000508386E996E29093710880937008089519
:1009600081E08093120580916E088770873051F086
:1009700010926E081092B90586E996E2909371087C
:1009800080937008809148118093A90580E00E94AF
:10099000F93420E040E070E060E082E296E80C94F8
:1009A000508380918002882341F030E020E041E0D4
:1009B0006FE670E282E00E94B32A8091B9058770E9
:1009C000873041F420E040E070E060E084E095E8AA
:1009D0000C945083089520E040E070E060E08BE1EB
:1009E00095E80E94508381E080930A058091AA05D2
:1009F000811107C084E590E290937108809370089C
:100A000008958AE590E2F8CF80918002882341F032
:100A100030E020E041E060E670E281E00E94B32A2D
:100A20008091C6081092C608882321F01092AA056A
:100A30000C94EB8408950F931F93CF93DF9300D012
:100A400000D000D01F92CDB7DEB7809180028823FE
:100A5000F1F01F9280E48F938091AA0590E00196B7
:100A60009F938F938CE490E29F938F938E010F5FFF
:100A70001F4F1F930F930F949A55B80181E490E292
:100A80000E942F2B0FB6F894DEBF0FBECDBF84E0BF
:100A90008093800280910A05811108C020E040E027
:100AA00070E060E081E695E80E9450832A960FB6D8
:100AB000F894DEBF0FBECDBFDF91CF911F910F9194
:100AC0000895CF92DF92EF92FF92CF93DF9300D001
:100AD0001F92CDB7DEB78091C6081092C608882352
:100AE00031F18091AA058F5F8093AA058034E0F0F0
:100AF00081E080930A0520E040E070E060E089E456
:100B000095EB0E9450838BE390E290937108809361
:100B100070080F900F900F900F90DF91CF91FF9082
:100B2000EF90DF90CF9008950E94EB84F2CF609118
:100B3000C9087091CA088091CB089091CC086115C2
:100B400071058105910509F43EC00F940A562DECFC
:100B50003CEC4CEC5CE30F946956209151113091C0
:100B6000521140915311509154110F94F55C6B0147
:100B70007C0120E030E040E850EC0F94035687FD04
:100B800053C020E030E040E850E4C701B6010F94C4
:100B9000555F18160CF44FC0C0925111D0925211EB
:100BA000E0925311F09254118FED92E00E9444F4C0
:100BB00082E0809380021092C9081092CA081092B5
:100BC000CB081092CC0880918002882309F4A1CF31
:100BD000C0905111D0905211E0905311F0905411E7
:100BE00020E030E0A901C701B6010F94035627E1C8
:100BF00037EB41ED58E387FF04C027E137EB41EDC8
:100C000058EBC701B6010F94F55C69837A838B8337
:100C10009C836BE2CE0101960F943502BC0184E304
:100C200090E20E942F2B75CFC12CD12C90E8E92E99
:100C300090ECF92EB1CFC12CD12C80E8E82E80E4C5
:100C4000F82EAACF80918002882341F030E020E086
:100C500041E06FE670E282E00E94B32A8091B9051C
:100C60008770873079F41092A80520E040E070E0AA
:100C700060E08BED9EEB0E94508381E08093A7059E
:100C80000C944B7D08952F923F924F925F926F92FA
:100C90007F928F929F92AF92BF92CF92DF92EF920C
:100CA000FF920F931F93CF93DF9300D000D0CDB767
:100CB000DEB71C017A8369832B833C834D835E837B
:100CC0002701380181E08093C8080E94CE7B83E031
:100CD00080938002309297052092960589819A81AF
:100CE00090939505809394058B819C81AD81BE8105
:100CF0008093900590939105A0939205B0939305EE
:100D000040928C0550928D0560928E0570928F05F1
:100D1000F12CE12CC092C908D092CA08E092CB080D
:100D2000F092CC08B092FA16A092F91690928B0528
:100D300080928A058C8D8093890526960FB6F8944B
:100D4000DEBF0FBECDBFDF91CF911F910F91FF90FE
:100D5000EF90DF90CF90BF90AF909F908F907F905B
:100D60006F905F904F903F902F90089520E040E06B
:100D700070E060E084E29FEB0C9450830E94BF36E9
:100D80000E94B8D70C94B68684E099E00F9443444F
:100D90000E94B6860D9404460E94B68682EE94E2C6
:100DA000909371088093700808950E9417340F94EF
:100DB000094581E080937B170F944B450C94B686D0
:100DC0006F927F928F929F92AF92BF92CF92DF925B
:100DD000EF92FF920F931F93CF93DF9381E0809365
:100DE000120561E00E94A680C091CE0885E0882EA1
:100DF0008C0ED1E005ED16E898EEE92E94E2F92E7E
:100E000082E0982E9C1A2CECC22E26E8D22E33EFCC
:100E1000A32E34E2B32E7D2E7C1A6C2E6194C11168
:100E200030C0DD23D9F08091CD081816BCF0409178
:100E3000C9085091CA086091CB087091CC084F5FE7
:100E40005F4F6F4F7F4F4093C9085093CA0860931C
:100E5000CB087093CC088F5F8093CD08809180027F
:100E6000882341F030E020E041E060E075E2862D2B
:100E70000E94B32ACF5F8C12D2CF83E08093C70841
:100E800023C0C13081F58091CD08813089F08091F7
:100E90008002882309F444C0DF92CF92BF92AF92C0
:100EA0007F9281E09091CD08913089F180E02FC050
:100EB0008091C6081092C608882349F30E94CC8608
:100EC0008091C808882319F3DF91CF911F910F916A
:100ED000FF90EF90DF90CF90BF90AF909F908F905A
:100EE0007F906F900895C23029F68091CD088230AE
:100EF000C9F080918002882399F01F930F93FF928D
:100F0000EF929F9281E09091CD08923079F68F9385
:100F10000E9498800F900F900F900F900F900F905D
:100F2000D0E0A8CF8091C6081092C608882309F3A4
:100F30000E94D5868091C8088823D9F2C5CF611157
:100F400060932402409311058C3008F03AC0E82FDA
:100F5000880FFF0B8827E055F8478F4F0D94EC5C06
:100F6000E387BC87C787E687CA87CD87D087DC87BA
:100F7000D387E187D687D9878CE293E821E0209355
:100F8000120520E040E070E060E00C94508384E3C0
:100F900093E8F4CF88E393E8F1CF8CE393E8EECFC6
:100FA00080E493E8EBCF84E493E8E8CF88E493E827
:100FB000E5CF8CE493E8E2CF1092FA0884E091E860
:100FC000DDCF0C94B68688E293E8D8CF80E393E82F
:100FD000D5CFCF930E9422FF0E942FDBC82F8823FA
:100FE00019F080E00F94D50E8C2F0E948380CF9152
:100FF0000C94B6860F931F93CF93DF93CDB7DEB7D4
:101000006E970FB6F894DEBF0FBECDBF282F082E07
:10101000000C330B90911F02409120028F3F39F05A
:10102000F901EE0FFF1FEF5DFD4F908141814F935E
:101030009F933F938F9386E79EE19F938F938E01BB
:101040000F5F1F4F1F930F930F949A554FE350E07C
:10105000B80182E798E00F946A600E94B6860FB6E6
:10106000F894DEBF0FBECDBF6E960FB6F894DEBF0C
:101070000FBECDBFDF91CF911F910F9108958FEFDC
:101080000C94FA878091DB080C94FA87E09198051C
:10109000EE2389F0E150E093980588E0E89FF001A5
:1010A0001124E75AFA4F628173812781468180813A
:1010B00091810C9450830C94B6862F923F924F925C
:1010C0005F926F927F928F929F92AF92BF92CF92D8
:1010D000DF92EF92FF920F931F93CF93DF9300D095
:1010E0001F92CDB7DEB761E081E00E94A68020911B
:1010F000CE082B832C83822F8B5F898389E0821B10
:101100008A8388E0782E721A87E0682E621A86E059
:10111000582E521A85E0482E421A84E0382E321A90
:10112000222E21942B8121115BC08091CD08882330
:1011300099F180918002882359F081E09091CD0847
:10114000911180E024E043E357E2622D0F945C327A
:101150008091390A8093D1088B81853009F0A1C034
:101160001092DB088091CD08853009F45CC1809134
:101170008002882309F436C211E08091CD088530C1
:1011800009F010E08091D1080F944E0400E09C011A
:1011900040E157E2642D82C08091C6081092C608D3
:1011A000882339F20E9446888091C808882309F470
:1011B000C0CF0F900F900F900F90DF91CF911F91A4
:1011C0000F91FF90EF90DF90CF90BF90AF909F90E6
:1011D0008F907F906F905F904F903F902F900895E9
:1011E0008B818130B9F58091CD088130E1F080911B
:1011F0008002882309F4ACCF11E08091CD088130C2
:1012000009F010E080917602909177020F94F70335
:1012100061E02C81621B00E09C014DE257E2812FCE
:101220000E94AE2B95CF8091C6081092C6088823E5
:10123000F1F210E000E027EE33E04AE050E066E72C
:1012400072E08DE297E20F9449348091C8088823B8
:1012500071F2AFCF8B81823009F087C18091CD08C8
:10126000823009F44EC0809180028823D1F011E0D1
:101270008091CD08823009F010E06091D70670911E
:10128000D8068091D9069091DA060E940B7C62E024
:101290002C81621B00E09C0147E257E2812F0E94F3
:1012A000AE2B80913A0A8093D1089B81963009F049
:1012B000E4C081E08093DB088091CD08863009F49A
:1012C000C7C080918002882391F011E08091CD0801
:1012D000863009F010E08091D1080F944E0400E0B0
:1012E0009C0140E157E2652D812F0E94AE2B9B812E
:1012F0009F5F9B832981291315CF8AE08093C708BC
:1013000058CF8091C6081092C608882309F4ABCF45
:1013100020E030E04AE754E46091D7067091D806A7
:101320008091D9069091DA060F94695620E030E05A
:10133000A9010F94F55C20E030E04AE754E40F94F3
:10134000F55C0F94685E1F92912C812C8CEAA82E7C
:1013500081EBB82E6B0110EDE12E17E0F12E00E0CD
:1013600010E028E13CEF4FEF5FEF67ED76E087E2BA
:1013700097E20E9443860F908091C808882309F461
:1013800072CF17CF8091CD088330C9F08091800251
:10139000882309F486CF11E08091CD08833009F0CD
:1013A00010E080918116909182160F94F70363E00C
:1013B0002C81621B00E09C0140E257E230CF80911B
:1013C000C6081092C608882309F30F94D13200EBA7
:1013D0001CE72CE231E050E040E061E876E180E299
:1013E00097E20F9449348091C808882379F2E1CEBE
:1013F0008091C6081092C608882309F4C2C00F94D1
:10140000D13202E819EC2CE830E050E040E06DE128
:1014100079E08CE197E20F9449348091C8088823E1
:1014200009F4AFC0C6CE8091C6081092C6088823C2
:1014300009F49DCE0F94D13266E378E780E197E21C
:101440000F9488358091C808882309F490CEB1CED6
:101450008091C6081092C608882309F432CF0F94F1
:10146000D13266E378E780E197E20F948835809186
:10147000C808882309F425CF9CCE2B81273091F50D
:101480008091CD088730B9F080918002882309F4DB
:101490002ECF11E08091CD08873009F010E08091C7
:1014A0003502909136020F94F70300E09C014BE067
:1014B00057E2662D19CF8091C6081092C60888237E
:1014C00019F303E118E727EE33E04AE050E065E363
:1014D00072E08BE097E20F9449348091C80888232A
:1014E00099F267CE8B81883009F062C08091CD0877
:1014F0008830D9F080918002882309F4F8CE11E079
:101500008091CD08883009F010E06091310A709127
:10151000320A8091330A9091340A0E94C87600E022
:101520009C0141E057E2672DDFCE8091C608109202
:10153000C6088823F9F261E37AE081E097E20F942C
:1015400042358091C8088823A9F233CE8091C6081D
:101550001092C6088823A1F18FED93E80E94D183F1
:101560008091C808882361F124CE8B81833009F4EF
:1015700009CF843009F0ECCD8091CD08843009F496
:1015800037CF80918002882309F48BCE11E08091BF
:10159000CD08843009F010E080911D0990911E095A
:1015A0000F94F70300E09C014CE157E2632D37CE26
:1015B0009B81993009F09BCE8091CD08893031F222
:1015C00080918002882309F492CE81E09091CD0829
:1015D000993009F080E023E046EF56E26A810F94EB
:1015E0005C3285CE80913A0A8093D10880CE5F929A
:1015F0006F927F928F929F92AF92BF92CF92DF9223
:10160000EF92FF920F931F93CF93DF93FF24F394F6
:101610008091811690918216892B09F4F12C61E05A
:1016200081E00E94A680C091CE088C2E95E0992E74
:101630009C0EAA24A39484E0E82EEC1A83E0D82E12
:10164000DC1A82E0C82ECC1A7A2C7C1A6C2E61949B
:1016500087E0B82EBC1AC111B8C08091CD0888238C
:1016600009F495C080918002882359F081E090911F
:10167000CD08911180E024E041EF56E2662D0F94F1
:101680005C3280913A0A8093D108C430E9F4A09288
:10169000DB088091CD08843009F445C18091800237
:1016A000882391F0D1E08091CD08843009F0D0E01A
:1016B0008091D1080F944E0400E09C014AED56E25F
:1016C0006E2D8D2F0E94AE2B10E000E0D5E05C2E39
:1016D00058180093D108CD131FC0F801EE0FFF1F5B
:1016E000EC5BFF4B859194919093DD088093DC082F
:1016F0008091CD088C1709F42BC18091800288233A
:1017000059F081E09091CD089D1380E023E040EDF9
:1017100056E2652D0F945C328D2F0F5F1F4FD6E080
:101720008630B9F680911D0990911E09892B19F414
:10173000FF2009F42DC1C73009F58091CD0887300D
:1017400009F417C1809180028823C1F08EEB96E8DE
:101750009F938F9387EC96E29F938F93BF9281E044
:101760009091CD08973009F080E08F930E94988087
:101770000F900F900F900F900F900F9088E0FF2424
:10178000F394CF5FC91167CF8093C7080EC08091D3
:10179000C6081092C608882309F464CF0E944688C0
:1017A0008091C808882309F45DCFDF91CF911F9104
:1017B0000F91FF90EF90DF90CF90BF90AF909F90F0
:1017C0008F907F906F905F900895C13009F05FC057
:1017D0008091CD08813009F43FC080918002882338
:1017E00009F44FCFD1E08091CD08813009F0D0E0ED
:1017F00080918116909182160F94F70300E09C016E
:101800004AEE56E2672D8D2F0E94AE2B8091390A49
:101810008093D108C33009F034CF1092DB08809157
:10182000CD08833009F46AC080918002882309F4CE
:101830004BCFD1E08091CD08833009F0D0E080918A
:10184000D1080F944E0400E09C014AED56E26D2D44
:101850008D2F0E94AE2B15CF8091C6081092C6081E
:10186000882309F4BACF0F94D1320EEA1CE72CE298
:1018700031E050E040E061E876E18AEE96E20F94D4
:1018800049348091C808882309F4A7CF8ECFC2308D
:1018900009F0BCCF8091CD088230B9F080918002F0
:1018A000882309F4EECED1E08091CD08823009F092
:1018B000D0E080911D0990911E090F94F70300E07C
:1018C0009C0146EE56E26C2D9ECF8091C608109288
:1018D000C608882319F30F94D13202E819EC2CE8DA
:1018E00030E050E040E06DE179E086EE96E20F9462
:1018F00049348091C808882389F257CF8091C6085F
:101900001092C608882309F48FCF0F94D13266E372
:1019100078E78AED96E20F9488358091C80888238D
:1019200009F482CF42CF8091C6081092C60888235E
:1019300009F4B4CE0F94D13266E378E78AED96E2EB
:101940000F9488358091C808882309F4A7CE2DCF3D
:101950008091C6081092C608882309F4CECE8AEC7E
:101960009CE80E94D1838091C808882309F4C5CEE1
:101970001CCF8091C6081092C608882309F4E2CED5
:101980000E94BE868091C808882309F4DBCE0DCF63
:1019900087E0F7CE4F925F926F927F928F929F92E5
:1019A000AF92BF92CF92DF92EF92FF920F931F936D
:1019B000CF93DF930091D10861E081E00E94A6807F
:1019C000C091CE0810E0000F111F0C5B1F4B95E07B
:1019D000592E5C0E2DEAE22E26E2F22ED3E0DC1B1D
:1019E00032EBC32E3CE7D32E4FE9A42E46E2B42EB1
:1019F00082E0782E7C1A50ED852E56E2952E81E0FD
:101A0000682E6C1A4C2E4194C11137C08091CD08BC
:101A10008823B1F080918002882359F081E0909171
:101A2000CD08911180E024E04BEB56E2642D0F9439
:101A30005C32CF5F5C12E8CF84E08093C7080CC0B3
:101A40008091C6081092C608882321F30E94468818
:101A50008091C8088823F1F2DF91CF911F910F91F7
:101A6000FF90EF90DF90CF90BF90AF909F908F90BE
:101A70007F906F905F904F900895C13059F5F801B5
:101A8000859194919093DD088093DC088091CD0836
:101A9000813081F080918002882359F21F929F92B9
:101AA0008F926F9281E09091CD08913009F474C0CB
:101AB00080E072C08091C6081092C608882351F356
:101AC0008091D108682F0F94F9368091C808882337
:101AD00009F3C2CFC23009F042C0F8018591949158
:101AE0009093DD088093DC088091CD088230D1F09E
:101AF00080918002882309F49CCFDF92CF92BF921D
:101B0000AF927F9281E09091CD08923009F080E011
:101B10008F930E9498800F900F900F900F900F90CE
:101B20000F9087CF8091C6081092C608882301F3D2
:101B30000E94B27C8091C8088823D1F28DCF809119
:101B4000C6081092C6088823C1F06091D1088FEFB3
:101B50000F94F9368091C808882379F07DCFC3307F
:101B600009F067CFF801859194919093DD088093F7
:101B7000DC088091CD08833011F3809180028823A6
:101B800009F457CF1F92FF92EF92DF9381E090917B
:101B9000CD08933009F08CCF8F930E9498800F90DE
:101BA0000F900F900F900F9044CF9F92AF92BF92E3
:101BB000CF92DF92EF92FF920F931F93CF93DF9319
:101BC00061E081E00E94A680C091CE08CC2E85E025
:101BD000982E9C0E97E5A92E96E2B92ED7E0DC1B35
:101BE00016E01C1B05E00C1B84E0F82EFC1A82E0BA
:101BF000E82EEC1A81E0D82EDC1AC11133C0809196
:101C0000CD088823B9F080918002882361F06C2D83
